:020000040800F2
:20000000F0FF01206D65060885F2000865CD0408E5650608E5650608E5650608000000002B
:2000200000000000000000000000000081F200087DF200080000000079F200086196040858
:20004000E5650608E5650608E5650608E5650608E5650608E5650608D9DC040805DE0408E0
:20006000C9DD04088DDD040851DD0408A949060899490608894906087949060865490608C2
:20008000514906083D490608E56506080000000000000000000000000000000015DD0408CE
:2000A0004D810408998104083D810408BD8104088D8104087D8104086D8104086554060847
:2000C0006D5406085954060861540608E5650608E56506083D98040881970408000000001E
:2000E0009DDC0408E5650608A10901080000000000000000000000000000000029490608F0
:20010000000000005D2406085D810408E5650608000000000000000000000000000000000E
:200120001549060801490608ED480608D9480608C54806080000000000000000000000006E
:2001400000000000000000000000000009EC0008B14806089D48060889480608C596040862
:200160004D5406085554060800000000000000000000000000000000000000000000000019
:2001800000000000E56506080000000000000000E5650608E56506080C61060001000000E3
:2001A0000E02010002000000706B0020D06B002000000000F80900081402010005000000B1
:2001C000B43E0020D46B002000000000FA0900081302010004000000CC240020DC6B002012
:2001E00000000000000A00080D1001004C000000F0680020E06B0020000000006DF5030833
:200200000400080080000000306800202C6C002000000000000000000902010001000000D5
:20022000D8670020AC6C002000000000040A0008FD010100240000007C670020B06C0020AF
:20024000000000007B630408FB01010001000000F0650020D46C002000000000C97B050890
:20026000FC01010009000000BC640020D86C002000000000D17B0508F7010100060000007B
:20028000B0640020E46C002000000000060A0008F901010004000000AC640020EC6C0020FB
:2002A0000000000025640408160215003F00000054320020F06C0020000000006D7B050826
:2002C0003400010010000000A0630020306D002000000000659402081102010008000000DA
:2002E00078630020406D0020000000000C0A0008121201000400000070630020486D002027
:2003000000000000140A000818200100320000003C6300204C6D00200000000055840508CE
:2003200012200100110000005C620020806D002000000000180A0008000201000B00000056
:20034000985F0020946D00200000000000000000FF11010006000000445F0020A06D00205E
:20036000000000005D7B0508081203000F000000505F0020A86D002000000000717B05086F
:20038000FA010100030000003C590020B86D002000000000F97B05080A8001002800000030
:2003A0001C510020BC6D0020000000006D140208061001001C00000078310020E46D00206F
:2003C00000000000557C05080202010003000000B8280020006E00200000000000000000A9
:2003E0000C0201000400000098280020046E002000000000217C0508110001000C000000B0
:2004000072450020086E002000000000FDF00308FE01010014000000E43F0020146E00207E
:2004200000000000217B0508FD0701007600000058C00020D0C000200000000081780108AE
:20044000261001000E00000058C1002048C1002000000000451C01080B3001001A00000035
:2004600024BA002098C10020000000002C0A00081F3001002400000060B90020B4C1002085
:2004800000000000480A0008050201000400000054BC0020D8C10020000000006C0A00088F
:2004A000030101000A000000A4B90020DCC1002000000000ED160108220201001C010000A5
:2004C0006CD9002024DC0020000000000D8405080C200600CC000000E4D7002040DD0020E3
:2004E0000000000065EF0308010201000B00000088D700200CDE002000000000117C05086B
:200500001B020100100000005CD7002018DE002000000000417C05081B1001000C00000042
:20052000E0C3002028DE002000000000F57E010821020100F000000060C2002034DE0020CE
:2005400000000000D9A00108231201001000000064D4002024DF002000000000700A0008D6
:20056000371001002E000000CCD6002034DF002000000000800A0008161001000600000051
:200580005CD4002064DF002000000000AE0A00082F1001002200000000DC00206CDF00201F
:2005A00000000000B40A00081E0001000900000054D3002090DF002000000000D60A00088F
:2005C0000510010006000000C8D300209CDF002000000000E00A0008F581010068000000D8
:2005E000F0C10020A4DF00200000000059910108232001001000000008D400200CE0002038
:200600000000000081150208F62101000C0000001CEC0020D4ED002000000000E80A000813
:200620001C0202001C000000C0EB002024EE0020000000004185050828200100180000004D
:20064000DCEB002040EE002000000000A5310208041201000200000094ED002058EE002065
:2006600000000000F40A00080F0201000100000090ED00205CEE002000000000F60A000852
:200680001400010004000000B8EB002060EE002000000000F80A0008012001000C000000D8
:2006A0002CE3002064EE002000000000FC0A00080EF003009E01000014E1002070EE002058
:2006C00000000000AD940208130001000400000048E7002010F0002000000000080B00082D
:2006E000010101000400000060E0002014F000200000000000000000000101000400000069
:2007000058E0002018F00020000000000C0B0008020101000300000054E000201CF00020B3
:2007200000000000A1EF03081900010005000000DCFD0020C8FE002000000000100B0008FD
:200740001A0001000E0000003CFD0020D0FE002000000000160B0008203201000A000000A3
:20076000D4FB0020E0FE002000000000899402081500100070000000B0F50020ECFE002001
:2007800000000000000000002A0008006000000024FE00205CFF0020000000003D9402082F
:2007A0002C00040010000000CCFF0020BCFF002000000000159202082B0012002400000021
:2007C00000000120DCFF002000000000E9910208292014007800000050F3002024000120FC
:2007E0000000000000000000190201001000000084F200209C00012000000000017C0508F0
:20080000030001000100000000190120141C01200000000000000000031201003D000000F5
:20082000A8180120181C012000000000240B000825201E002C0100000C160120581C0120E3
:20084000000000000000000010100100020000008C150120841D012000000000620B00087C
:20086000F821010006000000E8150120881D012000000000640B0008020001000C000000EE
:20088000F02501208426012000000000000000002902010040000000602001209026012073
:2008A000000000006A0B00080A020100140000004C1F0120F02601200000000031EF0308AC
:2008C00028020400040000004430012020320120000000003D7C05082702040004000000E7
:2008E000403001202432012000000000317C05081F020800100000009C2D01202832012098
:2009000000000000397B05081A0201003C000000442901203832012000000000C58405084E
:200920003810010001000000242701207432012000000000AA0B0008270001000400000051
:200940003C3301204433012000000000AC0B00080B1201003C000000FC340120C4470120D9
:2009600000000000B00B00080D12010014000000B04101200048012000000000EC0B000806
:200980000702010002000000AC4701201448012000000000000C00081D020200060000007F
:2009A00074470120184801200000000000000000060203000C00000080470120A04C0120CE
:2009C00000000000CD85050839000100050000008C470120AC4C012000000000E97B0508FB
:2009E00010020100010000007C8001207880012000000000020C00080000000000FF000098
:200A00000000010000000000010000000000000001010101FFFFFFFF00000001000105537A
:200A2000343131000000000200000000AE014A015E012C0164000200000001000A019A018B
:200A4000001E0A000002000000000000000100000005000001020300000000000000000060
:200A60000000000000000000008007000000000000000000000000000000000000000000EF
:200A800020003200C800D00796001400320028004C0440060005500014000F0008006400E7
:200AA0000100010005000A000000F4019600C40900001900000000000000000000000000B4
:200AC000000000000000000000000000000000000000000000000005010000000000000010
:200AE00020000301000000000000000001000000020200000000000003000023E803640058
:200B0000040A000114001E0000204030900100000000280100007E05EA05B4053200E80302
:200B2000D007000000000000000000000000000000000000000000000000000000000000DE
:200B4000000000000000000000000000000000000000000000000000000000000000000095
:200B6000010000050201F40114000000000000000000000000000000000000000000000063
:200B8000000000000000000000000000000000000000000000000000000000000000000055
:200BA000000000000000000000000000200300000000000000000000000000000000000012
:200BC000000000000000000000000000000000000000000000000000000000000000000015
:200BE0000000000000000000010000000000000000000000000000000000000000000000F4
:200C0000003C000403090412010002EF02014083045632000201020301000012010002020E
:200C2000020040830440570002010203010800FFFFFFFF00600240106002400000000000F3
:200C4000000000000B0000000000000000000000000000006002402860024001000000001C
:200C6000000000060C000000000000000000000000000000600240406002400200000000DC
:200C8000000000100D00000000000000000000000000000060024058600240030000000098
:200CA000000000160E00000000000000000000000000000060024070600240040000000058
:200CC000000000200F00000000000000000000000000000060024088600240050000000014
:200CE0000000002610000000000000000000000000000000600240A06002400600000000D4
:200D00000000003011000000000000000000000000000000600240B860024007000000008F
:200D2000000000362F000000000000000000000000000000640240106402400000000000F2
:200D40000000000038000000000000000000000000000000640240286402400100000000E6
:200D60000000000639000000000000000000000000000000640240406402400200000000A6
:200D8000000000103A00000000000000000000000000000064024058640240030000000062
:200DA000000000163B00000000000000000000000000000064024070640240040000000022
:200DC000000000203C000000000000000000000000000000640240886402400500000000DE
:200DE0000000002644000000000000000000000000000000640240A0640240060000000097
:200E00000000003045000000000000000000000000000000640240B8640240070000000052
:200E2000000000364600000000000000000000000000007D00000001000000158300081107
:200E40008300080D83000801830008FD820008098300080583000800000000D5900008B516
:200E6000AD000899900008F5AE0008AD9100088583000871830008558300083DA70008556E
:200E80008A0008D99300084D940008CD9400087D960008790F01085D8300084D830008018D
:200EA0000000000000803F41390108453E0108BD39010815100108F91101082510010841A5
:200EC000100108ED0F0108DD0F0108000000000000000009022000010104C03209040000CF
:200EE0000208065005070581024000000705010240000009026400030100C03209040000FD
:200F000001030000000921110100012226000705830308000A080B0102020201000904017B
:200F200000010202010005240010010524010002042402020524060102070582030800FF4F
:200F400009040200020A000000070501024000000705810240000009024300020100C03215
:200F600009040000010202010005240010010524010001042402020524060001070582030C
:200F80000800FF09040100020A000000070501024000000705810240000000FF0000000013
:200FA000FF0000000000000000AA550701000001AA550501000008D09D0608FF1FFF1F0561
:200FC000010905A101A1000501093009310932093309350934094009381581257F7508957E
:200FE000088102C0C0000009022200010100E0320904000001030102000921110100012232
:2010000026000705830308000A0000000000000102030401020304060708092D202D2D200D
:201020002D2D2D2D202D2D2D2D0000000000000000000000000000000000AA550B0100001D
:20104000AA5505010000AA550902000000AA5503009F0001000000C012000090C10020009C
:2010600000000068C1002000000000010000004C220708542207080000000011F00308A078
:201080008601000400000000000000000000000000000000000000000000000000000000C5
:2010A0000000000000000000000000000000004C2207085C22070800000000A5760408E817
:2010C000030000040000000000000000000000000000000000000000000000000000000009
:2010E000000000000000000000000000000000642207080000000000000000BD6003087DB6
:20110000000000FF00000000000000000000000000000000000000000000000000000000D0
:2011200000000000000000000000000000000038A807080000000000000000257103087DA2
:20114000000000FF0000000000000000000000000000000000000000000000000000000090
:2011600000000000000000000000000000000010370708000000000000000081B703087D59
:20118000000000FF0000000000000000000000000000000000000000000000000000000050
:2011A0000000000000000000000000000000006C2207080000000000000000096D0408E828
:2011C000030000030000000000000000000000000000000000000000000000000000000009
:2011E0000000000000000000000000000000007022070800000000000000001525030810F9
:201200002700000300000000000000000000000000000000000000000000000000000000A4
:201220000000000000000000000000000000004CA4070800000000058E020819CE04085FC0
:20124000760000050000000000000000000000000000000000000000000000000000000013
:20126000000000000000000000000000000000DCA70708000000000000000029EC040810AB
:20128000270000010000000000000000000000000000000000000000000000000000000026
:2012A0000000000000000000000000000000007C220708000000000000000045600408E8E8
:2012C000030000050000000000000000000000000000000000000000000000000000000006
:2012E000000000000000000000000000000000882207080000000000000000D5F303082042
:201300004E000003000000000000000000000000000000000000000000000000000000007C
:20132000000000000000000000000000000000982207080000000000000000BDF10308200B
:201340004E000003000000000000000000000000000000000000000000000000000000003C
:20136000000000000000000000000000000000A822070800000000000000001D73040840B8
:201380000D030003000000000000000000000000000000000000000000000000000000003A
:2013A000000000000000000000000000000000B8220708000000000000000071280408108F
:2013C0002700000100000000000000000000000000000000000000000000000000000000E5
:2013E000000000000000000000000000000000C0220708000000000000000071AD010810C5
:201400002700000300000000000000000000000000000000000000000000000000000000A2
:20142000000000000000000000000000000000C4220708000000000000000031710208A06B
:20144000860100010000000000000000000000000000000000000000000000000000000004
:20146000000000000000000000000000000000CC2207080000000000000000896B0408501F
:20148000C30000010000000000000000000000000000000000000000000000000000000088
:2014A000000000000000000000000000000000D4220708000000000000000059690408A0B9
:2014C000860100000000000000000000000000000000000000000000000000000000000085
:2014E000000000000000000000000000000000E0220708000000000000000041660408A880
:20150000610000010000000000000000000000000000000000000000000000000000000069
:20152000000000000000000000000000000000EC22070800000000000000002D070208A0B0
:20154000860100010000000000000000000000000000000000000000000000000000000003
:20156000000000000000000000000000000000F82207080000000000000000E99C0408A011
:201580000F000001000000000000000000000000000000000000000000000000000000003B
:2015A0000000000000000000000000000000000423070800000000000000002902020810B0
:2015C0002700000100000000000000000000000000000000000000000000000000000000E3
:2015E00000000000000000000000000000000010230708000000000000000051F00308A0BD
:201600000F00000100000000000000000000000000000000000000000000000000000000BA
:201620000000000000000000000000000000001C2307080000000000000000D5DC01081A88
:20164000410000010000000000000000000000000000000000000000000000000000000048
:201660000000000000000000000000000000002023070800000000000000002117010810C7
:20168000270000010000000000000000000000000000000000000000000000000000000022
:2016A0000000000000000000000000000000002C2307080000000000000000354C020850F1
:2016C000C30000010000000000000000000000000000000000000000000000000000000046
:2016E0000000000000000000000000000000003023070800000000000000005D20010840C2
:201700000D03000000000000000000000000000000000000000000000000000000000000B9
:201720000000000000000000000000000000003823070800000000000000001DF1030840E6
:201740000D0300000000000000000000000000000000000000000000000000000000000079
:2017600000000000000000000000000000000040230708000000000000000039EB0108507A
:20178000C30000030000000000000000000000000000000000000000000000000000000083
:2017A0000000000000000000000000000000004C23070800000000000000008505040840D5
:2017C000420F000000000000000000000000000000000000000000000000000000000000B8
:2017E00000000000000000000000000000000058230708000000000000000099F803085073
:20180000C30000000000000000000000000000000000000000000000000000000000000005
:201820000000000000000000000000000000000100000000000100E0010000FFFFFFFF01C8
:20184000017EFFFFFFFFFF080000004257020000000106425702000000010601FF0101FFC1
:20186000000000FFFFFFFF850A0208000000000000000008A80608D4E4002028E50020D53B
:20188000260208FD2402080000000070C0060851FA01080000000000000000D4BF06087545
:2018A00027020800000000000000008CBF06080000000000000000000000003CBE06080096
:2018C0000000000000000000000000F4BE0608000000000000000000000000A0BE060800DC
:2018E00000000000000000D92302080DE70020D601FF2D202D2D202D2D2D2D202D2D2D00D6
:2019000000000000000000000000000000000000000000FFFFFFFF652A0208000000000032
:20192000000000CCBD060801000000FA00000001000000010000000101000000010101000E
:2019400000000026E300200000F4010100000024E300200000F4010100000022E300200026
:2019600000F4010100000020E300200000F401010000001EE300200000F401010000001C25
:20198000E300200000F401010000001AE300200000F40101000000BD1202088112020800C5
:2019A0000000004CAA06080AE300200532010018E300206400F4010100000016E3002064EC
:2019C00000C4090100000008E30020E803D0070100000006E30020E803D00701000000049B
:2019E000E30020E803D0070100000002E300201E00B80B0100000010E3002005000F000112
:201A000000000012E3002003000A000100000000E300201E00F4010100000014E300200273
:201A2000000000D8AA0608FEE2002014006400010000000CE300203200E80301000000FC74
:201A4000E200200000C80001000000D5E2002000C80100D4E2002000500100D3E20020001F
:201A60005A0100D1E2002002000000E4AA0608582E0708602E0708AA6A00200100C4090066
:201A8000000000A86A00200100C40900000000A66A00200100C40900000000A46A00200119
:201AA00000C40900000000A06A00200100C40900000000A26A00200100C409000000009EC9
:201AC0006A00200100C409000000009C6A00200100C409000000007FE0002000C801007EF4
:201AE000E0002000C801007CE000200000FFFF0A0000007AE000200100C8000100000078DD
:201B0000E00020320030753200000076E000200582050074E0002005002C0105000000729D
:201B2000E00020055A05006FE0002000FF010071E0002002000000041000206DE0002003BB
:201B4000000000F09F06086EE0002000FF010070E0002002000000041000206CE000200365
:201B6000000000F09F060811120208A111020800000000F0AA06083CE30020EE02CA080135
:201B80000000003AE3002000C801006400000039E3002000C801006400000038E300200235
:201BA000000000FCAB060866E000200000803E0500000064E0002080C1803E050000005E81
:201BC000E000200083007D050000005CE0002080C1803E0500000057E0002000FF010052F7
:201BE000E000206400F4010100000050E000200400000008AC06084FE00020020000001C08
:201C0000AC060805E100200D00000028AC060802E100200064010000E10020320010270A39
:201C2000000000FEE000200D00000028AC0608FDE000200D00000028AC0608FCE0002002CD
:201C400000000060AC06080000000000000000000000006CAC060842E300203E000000A41D
:201C6000AC060840E300200100FF7F010000003FE3002002000000A0AD060807E10020033D
:201C8000000000B0AD060806E1002003000000B0AD0608C2E20020000A0100C0E2002000D3
:201CA00000E80301000000BEE200200000E80301000000BCE200200000E80301000000BA28
:201CC000E200200000E80301000000B2E200200000E80301000000B8E200200000E80301D0
:201CE000000000B6E200200000E80301000000B4E2002000140100D0E2002002000000C0E1
:201D0000AD0608CEE200200000F40101000000CCE200200000F40101000000CAE2002000B2
:201D200000F40101000000C8E200200000F40101000000C6E200200000A00F01000000C4B1
:201D4000E200200000A00F01000000E9E2002019640100E8E2002002000000CCAD0608E60F
:201D6000E20020E803D0070A000000E4E20020006401000A000000D9E2002000640100D828
:201D8000E2002000640100E0E20020006401000A000000DFE20020006401000A000000DE5D
:201DA000E20020006401000A000000E3E2002000FF01000A000000E2E2002000FF01000AD5
:201DC000000000E1E2002000FF01000A000000DDE2002001FF01000A000000DCE20020014D
:201DE000FF01000A000000DBE2002001FF01000A00000010E100200000F401010000000EDC
:201E0000E100200000A00F010000000CE100200000A00F010000000AE100200000A00F0199
:201E200000000008E100200000A00F010000005DE7002000C801005CE70020006401005B99
:201E4000E70020006401005AE700200064010059E700200064010058E70020FF08010057CD
:201E6000E700200164010009110208CD10020800000000D8AD060860E70020013201005F5D
:201E8000E700200100000048AE06085EE700200400000050AE060856E700200064010054AB
:201EA000E700201400E8030100000052E70020E80330750A00000050E7002000C801004FB9
:201EC000E7002000C801004EE7002000C801004DE700200032010062E70020004B01006177
:201EE000E700200400000064AE06084CE70020006401000A00000070E700200000D00701A6
:201F00000000006BE7002000C801006AE7002000C8010069E7002000C801006EE70020009E
:201F200000D0070100000068E7002000C8010067E7002000C8010066E7002000C801006CB8
:201F4000E700200000D0070100000065E7002000C8010064E7002000C8010063E7002000CF
:201F6000C80100C10E0208A90E02080000000078AE0608F9E00020005A0100F8E00020007E
:201F8000C80100F6E00020E803D0070100000000000000000000001924020814AF06085354
:201FA000544D3332463431310000006BE00020000301006AE0002000030100E50D020899CD
:201FC0000D02080000000068AF0608590D0208110D02080000000004B00608310E020849D9
:201FE0002A02080000000084B0060868E0002001030100991302086D13020800000000DCE2
:020000040800F2
:20200000B306089D0C0208590C0208000000004CB40608D10E02089D2B020800000000E82C
:20202000B40608652F0208C51302080000000090B50608210F020800000000000000001CB5
:20204000B60608FD0F0208A50F02080000000080B606089110020855100208000000002862
:20206000B70608D98B02084511020800000000B4B70608FBE2002001060100690F02083598
:202080000F020800000000B0B806080D8B0208692C02080000000020B90608218C020831A1
:2020A0002D02080000000070BA0608FAE2002001030100790E0208490E020800000000447A
:2020C000BB0608798C02080000000000000000A8BB0608E10C0208312A0208000000002833
:2020E000BC0608000000000000000000000000B4BC060879110208A92D0208000000002400
:20210000BD06080000000000000000000000003CBF060800BC00209CFF2C010000000088BF
:20212000DB0020E0150C1700000000B0D800200200000074BF06084BE000200200000080D4
:20214000BF060846E0002088136F170100000048E0002088136F1700000000EE6A00200069
:2021600000000000000000EC6A00200000000000000000EA6A00200000000000000000E88D
:202180006A00200000000000000000E66A00200000000000000000E46A00200000000000D7
:2021A000000000EC05002000000000000000001CE0002003000000D4C0060844E000208881
:2021C000136F17010000004ABC002088136F17000000003D0B02080000000000000000E4E8
:2021E000C0060851E600200100000038C106084CBC00200100000044C1060842BC00200256
:202200000000004CC1060800000000000000000000000058C10608290B020800000000003E
:20222000000000F4C1060800000000000000000000000048C20608000000000000000000C3
:20224000000000B8C206084AE0002002000000F0C2060846BC0020E0150C170000000001AF
:20226000010000AC000120FFFFFFFF0000803F0000000000000000000000000000000000D5
:20228000000000000000000000000000000000000000000000803F0000000000000000007F
:2022A0000000000000803F0000000000000000000000000000803F000000000000000000A0
:2022C000000000010000000000FA430000FA430000803F812A04080000000000000000000D
:2022E000000000FFFFFFFFFF00000000000000E02601200800000000000000D02601200895
:202300000000002000000099380108091101083138010800000000D90F0108194101088159
:20232000370108CD3301080000000000000000990F01082583000819830008259000084151
:2023400090000809900008ED8F0008D18F000851380108E51001088537010800000000B152
:202360000F0108D1330108553701082D3301080000000000000000A50F0108685E0C00FFAC
:20238000FFFFFF02010000A00F0000B80B000002FFFF01FFFF000040A407080000080205CA
:2023A0000303000000000048A40708010008020504030000000000204C07080200FE010188
:2023C00010030000000000C031070803001402000300000000000050A4070804001F0202A4
:2023E0000008000000000058A4070805001F020201080000000000FFFFFFFF1A0300000080
:20240000000000000000000000000000000000000000000000000004030904120100020093
:20242000000040830420570002010203010B01F58C0508C98C05086D8C0508097D05088937
:202440008C05082D8C0508057D0508E41A0020E58D0508058E0508D58D0508E97C050891DF
:202460008D0508498D0508D97C0508C01A002009860508F17C0508ED7C0508E57C05085138
:20248000870508E17C0508DD7C0508A0150708B5400108C5100108953F010800000000005B
:2024A0000000002D3701083D3601080000000000000000000000008D0F0108917D050885EE
:2024C0007D0508558E0508718E05083D7D0508398E05081D8E0508FFFFFFFF0100000050D6
:2024E000C30000010100001F0000001C0000001F0000001E0000001F0000001E0000001F43
:202500000000001F0000001E0000001F0000001E0000001F0000000068214C01250000E443
:20252000120708401F0708081B0020008002021F00000053544D202020202050726F647588
:202540007420202020202020202020302E3031008002021F00000053544D20202020205081
:20256000726F64757420202020202020202020302E3031EB160108E7160108DF160108C957
:20258000140108C51F0108F11F0108211F0108D5160108C5160108B5160108A5160108C19E
:2025A000140108FF010000F4010000FF0000000000040100000000000000021000000007EC
:2025C0000000000000000000000000010203040607080901000000701B0020000000000027
:2025E0000000000000000000000000000000000000000000000000000000000000000000DB
:202600000000000000000000000000000000000000000000000000000000000000000000BA
:20262000000000000000000000000000000000000000000000000000000000FFFFFFFFFF9F
:20264000FFFFFFFFFFFFFFFFFFFFFFFFFFFFFFFFFFFFFFFFFFFFFFFFFFFFFFFFFFFFFFFF9A
:20266000FFFFFFFFFFFFFFFFFFFFFFFFFFFFFFFFFFFFFFFFFFFFFFFFFFFFFFFFFFFFFFFF7A
:20268000FFFFFFFFFFFFFFFFFFFFFFFFFFFFFFFFFFFFFFFFFFFFFFFFFFFFFFFFFFFFFFFF5A
:2026A000FFFFFFFFFFFFFFFFFFFFFFFFFFFFFFFFFFFFFFFFFFFFFFFFFFFFFFFFFFFFFFFF3A
:2026C000FFFFFFFFFFFFFFFFFFFFFFFFFFFFFFFFFFFFFFFFFFFFFFFFFFFFFFFFFFFFFFFF1A
:2026E000FFFFFFFFFFFFFFFFFFFFFFFFFFFFFFFFFFFFFFFFFFFFFFFFFFFFFFFFFFFFFFFFFA
:20270000FFFFFFFFFFFFFFFFFFFFFFFFFFFFFFFFFFFFFFFFFFFFFFFFFFFFFFFFFFFFFFFFD9
:20272000FFFFFFFFFFFFFFFFFFFFFFFFFFFFFFFFFFFFFFFFFFFFFFFFFFFFFFFFFFFFFFFFB9
:20274000FFFFFFFFFFFFFFFFFFFFFFFFFFFFFFFFFFFFFFFFFFFFFFFFFFFFFFFFFFFFFFFF99
:20276000FFFFFFFFFFFFFFFFFFFFFFFFFFFFFFFFFFFFFFFFFFFFFFFFFFFFFFFFFFFFFFFF79
:20278000FFFFFFFFFFFFFFFFFFFFFFFFFFFFFFFFFFFFFFFFFFFFFFFFFFFFFFFFFFFFFFFF59
:2027A000FFFFFFFFFFFFFFFFFFFFFFFFFFFFFFFFFFFFFFFFFFFFFFFFFFFFFFFFFFFFFFFF39
:2027C000FFFFFFFFFFFFFFFFFFFFFFFFFFFFFFFFFFFFFFFFFFFFFFFFFFFFFFFFFFFFFFFF19
:2027E000FFFFFFFFFFFFFFFFFFFFFFFFFFFFFFFFFFFFFFFFFFFFFFFFFFFFFFFFFFFFFFFFF9
:202800000828000800400008232042657461666C69676874202F2053544D33324634313157
:202820002028533431312920342E312E30204A756E2031372032303139202F2032333A312D
:20284000313A3433202866376630633637383029204D5350204150493A20312E34320A2374
:2028600020636F6E6669673A206D616E7566616374757265725F69643A20424546482C2074
:20288000626F6172645F6E616D653A20424554414650564634313152582C207665727369D3
:2028A0006F6E3A2032306632663261302C20646174653A20323032312D30382D313054300E
:2028C000343A31343A35355A0A0A626F6172645F6E616D6520424554414650564634313107
:2028E00052580A6D616E7566616374757265725F696420424546480A0A23207265736F7531
:20290000726365730A7265736F75726365204D4F544F522031204230380A7265736F757222
:202920006365204D4F544F522032204130300A7265736F75726365204D4F544F5220332075
:202940004231300A7265736F75726365204D4F544F522034204230370A7265736F75726387
:20296000652050504D2031204131300A7265736F75726365204C45445F5354524950203129
:20298000204230310A7265736F757263652053455249414C5F54582031204130390A72651B
:2029A000736F757263652053455249414C5F54582032204130320A7265736F7572636520F4
:2029C00053455249414C5F5458203131204130380A7265736F757263652053455249414C8F
:2029E0005F52582031204131300A7265736F757263652053455249414C5F525820322041AD
:202A000030330A7265736F757263652053455249414C5F5258203131204130380A72657359
:202A20006F75726365204C45442031204331340A7265736F75726365205350495F53434BAC
:202A40002031204130350A7265736F75726365205350495F53434B2032204231330A7265A8
:202A6000736F75726365205350495F53434B2033204230330A7265736F757263652053502C
:202A8000495F4D49534F2031204130360A7265736F75726365205350495F4D49534F2032D7
:202AA000204231340A7265736F75726365205350495F4D49534F2033204230340A726573CD
:202AC0006F75726365205350495F4D4F53492031204130370A7265736F75726365205350E7
:202AE000495F4D4F53492032204231350A7265736F75726365205350495F4D4F5349203374
:202B0000204230350A7265736F75726365204144435F424154542031204130310A726573A3
:202B20006F75726365204144435F435552522031204230300A7265736F75726365204F53AD
:202B4000445F43532031204231320A7265736F757263652052585F5350495F435320312039
:202B60004131350A7265736F757263652052585F5350495F455854492031204331330A72FA
:202B800065736F757263652052585F5350495F42494E442031204230320A7265736F7572EF
:202BA00063652052585F5350495F4C45442031204331350A7265736F757263652052585F4F
:202BC0005350495F4343323530305F54585F454E2031204230390A7265736F7572636520B2
:202BE00052585F5350495F4343323530305F4C4E415F454E2031204131330A7265736F75BA
:202C00007263652052585F5350495F4343323530305F414E545F53454C2031204131340A13
:202C20007265736F75726365204759524F5F455854492031204230360A7265736F7572630C
:202C400065204759524F5F43532031204130340A0A232074696D65720A74696D657220419F
:202C60003030204146310A232070696E204130303A2054494D32204348312028414631294C
:202C80000A74696D657220413038204146310A232070696E204130383A2054494D31204333
:202CA00048312028414631290A74696D657220413130204146310A232070696E2041313057
:202CC0003A2054494D31204348332028414631290A74696D657220423031204146320A2384
:202CE0002070696E204230313A2054494D33204348342028414632290A74696D657220429D
:202D00003037204146320A232070696E204230373A2054494D342043483220284146322997
:202D20000A74696D657220423038204146320A232070696E204230383A2054494D3420438C
:202D400048332028414632290A74696D657220423130204146310A232070696E20423130B1
:202D60003A2054494D32204348332028414631290A0A2320646D610A646D61204144432009
:202D80003120310A232041444320313A20444D41322053747265616D2034204368616E6E05
:202DA000656C20300A646D612070696E2041303020300A232070696E204130303A20444DFE
:202DC00041312053747265616D2035204368616E6E656C20330A646D612070696E20413040
:202DE0003820300A232070696E204130383A20444D41322053747265616D20362043686182
:202E00006E6E656C20300A646D612070696E2042303120300A232070696E204230313A204E
:202E2000444D41312053747265616D2032204368616E6E656C20350A646D612070696E20C0
:202E400042303720300A232070696E204230373A20444D41312053747265616D203320437D
:202E600068616E6E656C20320A646D612070696E2042303820300A232070696E204230386F
:202E80003A20444D41312053747265616D2037204368616E6E656C20320A646D6120706992
:202EA0006E2042313020300A232070696E204231303A20444D41312053747265616D203100
:202EC000204368616E6E656C20330A0A2320666561747572650A66656174757265202D52EE
:202EE000585F504152414C4C454C5F50574D0A6665617475726520534F46545345524941B5
:202F00004C0A66656174757265204F53440A666561747572652052585F5350490A0A232007
:202F200073657269616C0A73657269616C203330203230343820313135323030203537360B
:202F400030302030203131353230300A0A23206D61737465720A7365742072785F7370698A
:202F60005F70726F746F636F6C203D204652534B595F580A7365742072785F7370695F62F1
:202F80007573203D20330A7365742072785F7370695F6C65645F696E76657273696F6E209E
:202FA0003D204F4E0A736574206473686F745F6275727374203D204155544F0A73657420C4
:202FC0006473686F745F62697462616E67203D204F46460A7365742063757272656E745F69
:202FE0006D65746572203D204144430A73657420626174746572795F6D65746572203D2005
:203000004144430A7365742069626174615F7363616C65203D203137390A7365742073798A
:203020007374656D5F6873655F6D687A203D20380A736574206D6178373435365F73706998
:203040005F627573203D20320A736574206363323530305F7370695F636869705F646574CB
:20306000656374203D204F46460A736574206779726F5F315F62757374797065203D2053BA
:2030800050490A736574206779726F5F315F737069627573203D20310A7365742067797265
:2030A0006F5F315F73656E736F725F616C69676E203D2043573138300A7365742067797236
:2030C0006F5F315F616C69676E5F796177203D20313830300A00FFFFFFFFFFFFFFFFFFFF91
:2030E000FFFFFFFFFFFFFFFFFFFFFFFFFFFFFFFFFFFFFFFFFFFFFFFFFFFFFFFFFFFFFFFFF0
:20310000FFFFFFFFFFFFFFFFFFFFFFFFFFFFFFFFFFFFFFFFFFFFFFFFFFFFFFFFFFFFFFFFCF
:20312000FFFFFFFFFFFFFFFFFFFFFFFFFFFFFFFFFFFFFFFFFFFFFFFFFFFFFFFFFFFFFFFFAF
:20314000FFFFFFFFFFFFFFFFFFFFFFFFFFFFFFFFFFFFFFFFFFFFFFFFFFFFFFFFFFFFFFFF8F
:020000040800F2
:20400000ADBE08000E02000000000B0014020000000000FF000A001302000000000100528B
:20402000000D00010001000000140504050000000000000000000504050000000000080039
:20404000000105040500000000000000000505040500000000000000001E05040500000012
:2040600000000000001F0504050000000064005200860004000000000000000000000000D3
:20408000000000000000000000000000000000000000000000000000000000000000000020
:2040A000000000000000000000000000000000000000000000000000000000000000000000
:2040C0000000000000000000000000000000000000000000000000000000000000000000E0
:2040E0000000000000000000000000000000000000000000000000070009020000002A0084
:20410000FD0100001912000000000000000018001A13000000000000000018000000000019
:2041200000000000000000000700FB0100001A0F00FC0100000000000000000000000C004A
:20414000F70100000000010000000A00F90100003E0000004500160200001001001801009D
:204160001A01FF2102002701002801002A01001202FF000000000000000000000000000073
:2041800000000000000000000000000000000000000000000000000000160034000000DCF9
:2041A0000532000000000000000000000001040E001102000000000000010101010A001282
:2041C00002010028FFFFFF380018000200000103020405060702000000000001006400DC06
:2041E000051A046C07020213001900750343080E00000100000001030A1E010100000017E2
:20420000001200020000030001000105533431310000080202001100000200000000000078
:20422000000000000000000C00FF010100000000000000150008020100151617FFFF2D2EB6
:204240002FFFFF232425FFFF0900FA0100000000002E000A00080030000000C800FA000091
:20426000000000000000000000020000029E077D00C800F4015802080078009600000122C8
:204280000006000100803E040001020028102A270000000000020026022E04D007E8030C9F
:2042A000000900020200000200000A000C020000012C020012001100000001001234567870
:2042C0009ABC000000001A00FE0100000111000000200000010000000000000000FFFF003E
:2042E0007C00FD07000061098109CD084E00CE00360096094D018909E10079018101610165
:20430000DA003300F700A701C701E70141015901EA084C00520041000100210041008801E8
:204320004B092E012F01370117012A0052005300EA00EA00EA000C01EA00EA00EA00EA0038
:20434000EA00EA00EA00EA00EA00EA00EA00EA00EA00EA00EA00EA002300EA00140026001E
:20436000010002000000000015005802D903000020000B000300AE014A015E012C016401D6
:204380000000C80001000A019A01001E0A0000022A001F0003000000000000010000000532
:2043A00000000102030000000000000000000000000000000000008007000A00050200005F
:2043C0000000000010000301000004040100A816000000002201220200000508E916D516C4
:2043E000C116AD169916851671165D16651678168B169E16B116C416D716EA164916351649
:2044000021160D16FD161117251739176C1680169416A816BC16D016E416F8161A163F16B6
:2044200064168916AE16D316F8161D17000000000000000000000000000000000000000074
:2044400000000000000000000000000000000000000000000000000000000000424F534335
:20446000414D5F4100424F5343414D5F4200424F5343414D5F4500464154534841524B000B
:204480005241434542414E440042414E44362020200042414E44372020200042414E443848
:2044A0002020200041424546523637383100320033003400350036003700380001010101EF
:2044C000010000000400000001000200030000000000000000003235200032303000353053
:2044E0003000383030004C5634004C5635004C5636004C563700D2000C0002003200006420
:204500006464000000464646410046050064CE07CE07CE070100000000000000000032005F
:2045200000646464000000464646410046050064CE07CE07CE07010000000000000000000D
:20454000320000646464000000464646410046050064CE07CE07CE070100000000000000BB
:204560000000320000646464000000464646410046050064CE07CE07CE070100000000009B
:2045800000000000320000646464000000464646410046050064CE07CE07CE07010000007B
:2045A000000000000000320000646464000000464646410046050064CE07CE07CE0701005B
:2045C0000000000000000000110001020000000000000200000000000016001B020000068C
:2045E000000000E8030000000000000000000012001B000100002100020301F40132000153
:2046000000F6002102000000223400104020000000000000000000000000000000000000BB
:2046200000000000000000000000000000000000000000000000000000000000000000007A
:2046400000000000000000000000000000000000000000000000000000000000000000005A
:2046600000000000000000000000000000000000000000000000000000000000000000003A
:2046800000000000000000000000000000FFFF000000FF1E0000FF3C0000FF5A0000FF78F4
:2046A0000000FF960000FFB40000FFD20000FFF00000FF0E0100FF2C0100FF4A0100FF006F
:2046C00000000000000000010B020D0A03050B030D0A030A0B040D0A03080B040D0A03071A
:2046E0000B030D0A03000000000000060D0100000203060000000316002302010000000034
:204700000000000000000000000000000034003700010020003200C800D007960014003260
:204720000028004C0440060005500014000F00080064000100010005000A000000F401963B
:20474000000C0016000100C4090000B40028002F0001004245544146505620363553000077
:204760000000000000000000000000000000000000000000000F001E000000000501000006
:20478000000000000C00050001002000030100006E00F5010800980864001401000A010251
:2047A0000000FF1F0000142800006E3700008000FFFFFFFF46000102000000000000000035
:2047C0000000000000000000000000000000000000000000000000000000000000000000D9
:2047E0000000000000000000000000005000C4FF00FFFFFFFF0100000005180B000016006B
:20480000230002000A0000001D000100C7FF0100000000001200F601020000000000010078
:2048200000000202000022001C0200000002011400002603000000000807010200000000E2
:2048400000010000000000001E00280002000000000002000000000000000000000000000D
:20486000000000000000080004020100000007000F020000000A00140000000300002312BB
:204880000001000200E8036400040A000114001E00A4010E000F0000009600000000002A03
:2048A0005523005A002E5A26005F002D5A00005A0032324B0000002800000000000064F409
:2048C00001900101374B000000FA00AC0D00000000320090015E01F40100000A640000C8C3
:2048E000009001960000050F00010F0114004B3200005A140B00004600AA00001400280135
:2049000000C80017190025146400000F000000000000000000003232C89602643C25050065
:204920000000009600000000002A5523005A002E5A26005F002D5A00005A0032324B000048
:20494000002800000000000064F401900101374B000000FA00AC0D00000000320090015EEE
:2049600001F40100000A640000C8009001960000050F00010F0114004B3200005A140B00B5
:20498000004600AA00001400280100C80017190025146400000F0000000000000000000046
:2049A0003232C89602643C2505000000009600000000002A5523005A002E5A26005F002D9D
:2049C0005A00005A0032324B0000002800000000000064F401900101374B000000FA00AC39
:2049E0000D00000000320090015E01F40100000A640000C8009001960000050F00010F0111
:204A000014004B3200005A140B00004600AA00001400280100C80017190025146400000FBB
:204A2000000000000000000000003232C89602643C250500000A0013000000100005320A7A
:204A40000001010000000000000A0000010000803E00000900020100006E0A010B001900E2
:204A60000000000028010014001A0000007E05EA05B4053200E803D007000010002002038B
:204A8000000364F4010064F401960076001500000000000000000000000000000000000040
:204AA0000000000000000000000000000000000000000000000000000000000000000000F6
:204AC0000000000000000000000000000000000000000000000000000000000000000000D6
:204AE0000000000000000000000000000000000000000000000000000000000000000000B6
:204B00000066002A00000000000000E803D007DC0564FF00000000E803D007DC0564FF00F9
:204B2000000000E803D007DC0564FF00000000E803D007DC0564FF00000000E803D007DCCB
:204B40000564FF00000000E803D007DC0564FF00000000E803D007DC0564FF00000000E8F9
:204B600003D007DC0564FF16002C000000E803D007E803D007E803D007E803D0072A002B78
:204B8000000000001E001E001E0005011E011E011E011E011E011E011E011E011E011E017F
:204BA0001E011E011E011E7E0029000200000010300000010100100000020110200000004C
:204BC0000000000000000000000000000000000000000000000000000000000000000000D5
:204BE0000000000000000000000000000000000000000000000000000000000000000000B5
:204C0000000000000000000000000000000000000000000000000000000000000000000094
:204C200000000000001600190200000D00000000000000001F03223F013D0007000300006B
:204C400000004300030201000000000000000000000000000000000000000000000000000B
:204C6000000000000000000000000000000000000000000000000000000000000000000034
:204C80000000000001320125000200000000000000000000000000000000000000000000B9
:204CA0000000000000000000000000000000000000000000000000000000000000000000F4
:204CC0000000000000000000000000000000000000000000000000000000000000000000D4
:204CE0000000000000000000000000000000000000000000000000000000000000000000B4
:204D0000000000000000000000000000000000000000000000000000000000000000000093
:204D2000000000000000000000000000000000000000000000000000000000000000000073
:204D4000000000000000000000000000000000000000000000000000000000000000000053
:204D6000000000000000000000000000000000000000000000000000000000000000000033
:204D8000000000000000000000000000000000000000000000000000000000000000000013
:204DA000000000000000000000000000000000000000000000000008001000010000050CC9
:204DC00000F80102000201F401140012000200000000000000000000000000000046002949
:204DE0000200000000000000000000000000000000000000000000000000000000000000B1
:204E0000000000000000000000000000000000000000000000000000000000000000000092
:204E20000000001A000A02000000004A01C800630000007D006E005A004B0014000A002800
:204E4000020000000000000A00270200000000000016001F020000FFFFFFFFFFFFFFFFFFEF
:204E6000FFFFFFFFFFFFFF42001A02000000000000000000000000000000000000000000DB
:204E800000000000000000000000000000424546480042455441465056463431315258006F
:204EA000000000000000000100070038000100000A00270000002003000042000B0201000D
:204EC00000236026C8A17A532C05C9A27B542D06CAA37C552E07CBA47D562F08CCA57E5723
:204EE0003009CDA67F58310ACEA78059320BCFA8815B33000000000000291D1E1A000D0256
:204F000001000000000000000000000000000000000000000000080007020000003C0C0037
:204F20001D0200000000000000001200060200000000010000000100000001000B003900F1
:204F4000000000000000000700100200000000008DDB0000FFFFFFFFFFFFFFFFFFFFFFFFDC
:204F6000FFFFFFFFFFFFFFFFFFFFFFFFFFFFFFFFFFFFFFFFFFFFFFFFFFFFFFFFFFFFFFFF51
:204F8000FFFFFFFFFFFFFFFFFFFFFFFFFFFFFFFFFFFFFFFFFFFFFFFFFFFFFFFFFFFFFFFF31
:204FA000FFFFFFFFFFFFFFFFFFFFFFFFFFFFFFFFFFFFFFFFFFFFFFFFFFFFFFFFFFFFFFFF11
:204FC000FFFFFFFFFFFFFFFFFFFFFFFFFFFFFFFFFFFFFFFFFFFFFFFFFFFFFFFFFFFFFFFFF1
:020000040800F2
:020000040800F2
:20800000F0B401292A4C2B4D23684FF0000694BF00270127EE626662A6626763676B47EA45
:2080200042076763EE63EC6B002A38D144F49574EC631C6824F001041C601C68E407FCD46A
:20804000490289085960D8601968EAB921F04001196019498B421DD018494FF47410C860F8
:20806000196841F01E011960596941F080015961196841F00101196022B90E4AD36A43F0B8
:208080000803D362F0BC704741F0400119600A498B42E1D14FF0746041F8500CE0E744F0DD
:2080A0001A04EC63EC6A44F00804EC62C1E700BFD01B0020002C01405864024000640240EC
:2080C0001148002302461178032902F1060216D00133062BF7D10D4AD36D052B0ED0591CFF
:2080E00003EB4303D16500EB4303032040F2EB3140F2FF32187059809A807047704703EB3A
:20810000430300EB4303F0E7081C0020D01B002070B4C3080D4CE25C00F00706B24004EB5E
:20812000D004D2B20020C6F108038B4228BF0B46C3F108052A419840C91A40EA02004FF0AE
:20814000000614F8012FEED170BC7047701C0020084AD2E9343199420AD0D118013391F8C2
:20816000D8100170C3F30A03C2F8D0300120704700207047D01B0020064AD2F8D838D2F87B
:20818000DC28934294BF4FF400600020013B9B1A18447047D01B0020012380F8513070470D
:2081A00007B501A8FFF7D4FF0028FAD09DF8040003B05DF804FB044BD3E93403984288BF9C
:2081C00003F50063181A7047D01B002001207047024BC3F8E028C3F8E4187047D01B0020EF
:2081E000024BC3F8E828C3F8EC187047D01B00207047704730B4134DD5E934239A4286BFFE
:2082000003F50064A21A9A1A0A44B2F5006F13D8A9B101444A1E013810F8014FE9188242E6
:2082200003F1010381F8D840C3F30A03F4D1C5F8D430002030BC7047022030BC7047084696
:20824000F8E700BFD01B0020212838B50C4605D022282ED0202813D0002038BD0029FBD09C
:20826000072AF9D11A4BD3F8F00893F8F41893F8F52893F8F638206021716271A371EBE718
:208280000029E9D0072AE7D1114DD5F8E4381BB10968D5F8E0089847206821796279A379E2
:2082A000C5F8F00885F8F41885F8F52885F8F638D2E70029D0D0022ACED1054AD2F8EC38B1
:2082C000002BC9D00988D2F8E8089847C4E700BFD01B0020024B0020C3F8F808704700BF9D
:2082E000D01B0020044B00200522C3F8F828C3F8EC08C3F8E4087047D01B0020704700BF74
:20830000704700BF704700BF704700BF704700BF704700BF704700BF042301480B807047E7
:208320009801002010B4074A074B92F8FC08122403F114020C8001280CBF184610465DF8C6
:20834000044B7047D01B00209C01002000487047581C002000487047581C0020034B93F850
:208360008400032894BF002001207047D01B0020034B93F88400032894BF00200120704725
:20838000D01B0020034B93F88400003818BF0120704700BFD01B0020A0B182680D4B12B16E
:2083A00007229A7070471978DA6003294FF004000CBF80214FF48071C3E901111A611A7531
:2083C00098707047034B41F2E47101225A545A70704700BF289E00200378022B10D0006920
:2083E00008B9012070470C4B1B78032B0EBF0B4B80B24FF6F773984294BF002001207047A3
:208400000549436841F650028A58B3EB422F2CBF01200020704700BF289E0020F7FFFF0F5D
:208420000378022B14D030B4104A4368006941F6480402F5C2511559096841F63C042B4010
:2084400012595B0A023801FB0030104430BC7047064B426841F6340141F630005958185800
:2084600000EB410000EB5220704700BF289E002008B5124BD3F8BC00828940F2E933028992
:20848000013B12F0020F9BB212D0FF23838140F2E9330289013B12F0010F9BB202D08089E9
:2084A000C0B208BD002BF4D145F0C0FEC0B208BD002BE4D145F0BAFEC0B2F8E7D01B002042
:2084C00070B505460E460924FFF7D2FFFF2803D1013CF9D1012070BDFE2801D0022070BD4E
:2084E000064933462A46D1F8BC0000215CF064FAFFF7BEFFFFF7BCFF002070BDD01B002038
:2085000010B51D4C0023C4F88030FFF7B1FFD4F8BC00828940F2E9330289013B12F0020F3D
:208520009BB217D0FD23838140F2E9330289013B12F0010F9BB212D08389FFF799FFFF28CC
:2085400012D1FFF795FFFF280ED10423022084F8843010BD002BDFD145F068FEEDE7002BED
:20856000E4D145F063FEE8E7D4F8003963670923002084F8843010BDD01B002070B582B067
:2085800040F040060C0E05460A0A080C95238DF801408DF804108DF800608DF802008DF8D0
:2085A00003208DF805300824FFF762FFFF2802D0013CF9D125BB1A4BD3F8BC000625838958
:2085C0006E464FF47A734FF6FF713EB316F8012B0489013BA4079BB215D593B283814FF4A0
:2085E0007A730489E40703F1FF3211D5013D8289EBD10924FFF73CFFFF2802D1013CF9D1A7
:20860000FF2002B070BD8B42E2D145F00FFEF0E793B28B42E5D145F009FEEAE7FF22D7E70F
:20862000D01B00202DE9F041684C00234FF4F0722021064604F6081084F8043960F0CBFDFC
:2086400004F6E8204FF4F072202160F0C4FD94F8C90C10B194F8CA2C1AB900252846BDE872
:20866000F08144F061F80746C4F8D40C44F030FB05460028F1D00FB12323FB800921384657
:2086800040F000FAD4F8D40C514F44F043FB94F8CA0C013840B245F033FF0223102184F82C
:2086A000CC3CC4F8D00C58F079FD798D494845F073FDD4F8D40C44F027FBFF218C2058F00A
:2086C000E5FE8046D4F8D40C44F024FBD4F8D00C042158F063FDB8F11B0F05D0D4F8D40C29
:2086E000202140F0CFF9B8E7D4F8D43C012284F804290BB12322DA80798D364845F04CFD9D
:20870000D4F8D40C44F000FB40210A2058F0BEFEFF218A2058F0BAFEC0F38013D4F8D40C33
:2087200084F8D83C44F0F6FAD4F8D00C042158F035FD94F8C83C012B3FD0022B37D0CBB3C1
:2087400094F8D93C182B08D194F8D82C7B8DA4F8DC6CA4F8DE2CA4F8E03C798D1D4845F0E2
:208760001BFD798D1B4845F017FDD4F8D40C44F0CBFA0221002058F089FED4F8D40C44F098
:20878000C9FA0421D4F8D00C58F008FD94F8E92C94F8EA3C94F8E81C84F8E41CC2F12002C8
:2087A000C3F1100384F8EB2C84F8EC3C56E708237B85C5E710237B85C2E7002EF7D094F84A
:2087C000D83C002B14BF08231023F1E7D01B0020980100209C2800202DE9F84F564B9842D1
:2087E00010D003F568530833984267D0534B0020A3F8480DA3F8540DC3F84C0DC3F8500DC4
:20880000BDE8F88F4D4C4E4E02224FF0000BC4F8F02C04F6F445D9464FF4007A4FF4807867
:20882000F26A01275A455946BB4403D0D4F8640D53F09CFB94F8682D85F82420D4F8640D6E
:20884000A5F804A04FF000724FF48031A960EA60A5F8108085F81290A5F806802F76286241
:20886000B72153F079FDD4F8F02C364B6F76934545F8283BD4DB84F8569DD4F8F01CB4F8FF
:20888000F82CD4F8003DD4F8FC0CB4F8045DC4F86C3D12FB01F203FB01F3A4F8482DB4F8B6
:2088A000FA1C294AC4F84C0DC4F8503DA4F8545DA4F84A1DC4F8442D0120A1E71F4C204ED2
:2088C0000223C4F8F03C04F6F4454FF0000B4FF4806A4FF040094FF40068F26A01275A458B
:2088E0005946BB4403D0D4F8640D53F03FFBD4F8641D94F8682D296285F824204FF400311F
:208900004FF00062C5E90212A5F804A0A5F81090A5F80680AF74FFF7D3FB28466F7653F0D6
:208920006DFCD4F8F02C094B45F8283B9345D4DB84F8567DA1E700BF1971EF00D01B002051
:208940009801002078920608D0920608A4920608F8B51A4C94F8703D002BFBD159B30144FE
:208960004E1E451ED4F8DC28D4F8D81815F8017F531CC3F30A038B422CBF4FF40060002062
:20898000C91A22440144012982F8747DC4F8DC380FD1012040F0C4FDD4F8D838D4F8DC1856
:2089A0008B4294BF4FF4006200225B1A1344012BEFD0B542D6D10020F8BD00BFD01B0020DC
:2089C00010B5094CD4F8F838084611465BB1D4F8F838052B07D1002AD4F8003903DDFFF7C7
:2089E000B7FFD4F8003910BDD01B002010B590F85010002380F8503081B10B4CD4F8F828A7
:208A000072B1D4F8F828052A0CD13C30D4F80039FFF79EFFD4F80039012010BD0120FCE740
:208A20001046FAE71846F8E7D01B0020002280F85120DBE790F85020531C0244DBB280F838
:208A4000503082F83C1090F851200AB1132B00D9CCE770472DE9F04143794F4C002B14BFFF
:208A60000122002284F8B02003D184F88430BDE8F08190F8018008F1FF3676B2054630462B
:208A80000F4645F03DFD0223C4F8BC0084F8B8302B78002B5BD1ED78002D4CD14FF4807134
:208AA000D4F8BC00C4F8C05058F078FB4FF47A7040F036FDD4F8C00044F02CF9D4F8BC00AA
:208AC0000A2683894FF6FF714FF47A73FF270289950719D587814FF47A730289D20703F1AA
:208AE000FF3524D5013E8289F1D12C4B0289920713D5028912F080020FD1D4F8001984F86A
:208B0000782001236167B0E7013B9BB28B42DED145F08CFBD4F8BC00E7E7013BE6D194F8A4
:208B2000782084F88430531C84F878309FE7ABB28B42D2D1ECE7284643F0F6FD054608B11C
:208B40001E23C380092128463FF09CFFA6E706EB86063E44414696F90320002041F054F8CD
:208B6000064630B140685AF047FBB36884F8CE3018B9002384F8C4308DE7094A431E02EB86
:208B8000431317210022C4F8C8305AF047FB012384F8C4307FE700BFD01B0020A1860100F9
:208BA000C80100202DE9F04FCF4ED04D86468C4617460FCE05F27C442DED068B0FC40FCE53
:208BC0000FC496E807008BB095F8B234059784E80700CDE906EC042B00F24981DFE813F023
:208BE000A801470142010500B8019FEDC18ADFEDC18AC149C5F89814C049C14BC14AC5F845
:208C000094140599002918BF134638EE887AF5EE006AC6EE879ABC4EC5F8A034A6F1150321
:208C2000039306F1C0080027DFEDBF7A9FEDB79A28EE278AB0EE67AA079BBB4200F00C8144
:208C4000039B13F8014B039307F1010B5FFA8BF3002C00F08081002203E00132152A00F02A
:208C60007A8102EB42014FEA420918F80100A042F3D12944049391F88D15002900F0738152
:208C800020463FF0E5FC824600683FF085FC9AF805103FF0FDFC90F800C0BCF1000F40F07B
:208CA0005A8105EB09014FEA141909F1FF39049B81F8CD350322B9F1040F81F8CC2504F0ED
:208CC0000F0000F2FF80924C04EB4901B1F8B0C04CFA00F111F0010100F02881012101FAF4
:208CE00000F0013800EA0C00A14404935DF0C6FA99F8BCC0DFF82CE2049B60440EEBC00CD2
:208D000003228CF807308CF806205EF83000C6F814C000F13F4303F57E0304EB93240121FD
:208D200094F8C4309AF8082003F01F045B09032B01FA04F100F0D380042B00F0CB80022B87
:208D400000F0C380BCF804300893B3FA83F3C3F11F03C3F3CC0100EB810103F007030C6A01
:208D60009B004FF00F0C0CFA03FC24EA0C040C620C6A02FA03F323430B62022308A90993C0
:208D80000BF0DAFC059B002B76D0B5F8B034D5F8781807EE903AF8EEE77AFCEEE77A17EEAD
:208DA000900AB1FBF0F202F57F42FF32120CB1FBF2F295F8B214B2FBF0F0042983B272D070
:208DC00007EE902AF8EE676A66EE887A29EE677A95F8B30406990091A8EEA67A019051468D
:208DE0003046C6ED027A86ED037A36F07FFF002F64DD7368D5F8D024934261D0012F5DD0CB
:208E0000D5F8E82493425BD0022F57D0D5F80025934255D0032F51D0D5F8182593424FD0E4
:208E2000042F4BD0D5F83025934249D0052F45D0D5F84825934243D0062F3FD0D5F86025D3
:208E4000D31A18BF01235F460122082F3374727406F118067FF4F0AE2E480BB0BDEC068B0D
:208E6000BDE8F08F9FED2C8AF0EE488AC1E69FED2B8AF0EE488ABCE6B0EE690A5EF038FB10
:208E8000FCEEC07A4FF6FF7317EE902AD5F87818B1FBF2F21A44120CB1FBF2F295F8B214EC
:208EA000042918468CD107EE900A07EE102AF8EE677AF8EE476A67EE8A7A87E70123C2E71A
:208EC0000023C0E7C6F814C05CE7154B5C6C2143596437E7124B1C6B2143196332E7104B54
:208EE0001C6C214319642DE7FC920608C82C0020ACC5A737ACC5A73691F10308116404089A
:208F0000B5EC0308056404089431002000007A447892060844310020282930386F1203396A
:208F200000380240C03200206F12833A716129E71FED038A0D4A0E4BC5F89824C5F894343E
:208F400000220123CDE90532F0EE488A094B5CE69FED098AEEE7094A064BC5F89824C5F8CA
:208F6000A034002079E70B68FFDE00BF91F1030811640408056404080000000005EE03080D
:208F8000104B70B5D3F87848054600680E4664080BF0D6FAB4FBF6F1B1F5803F03D3012C8A
:208FA000FAD96408F6E72246284689B23FF0EEF90549064B0B6028460022BDE870403FF050
:208FC00005B900BFC82C0020A83D0020EDFD010810B5044C04480A4621460AF02BF920466C
:208FE00010BD00BFB03D00206421070810B5044C04480A4621460AF01DF9204610BD00BF2A
:20900000B03D00207421070810B5044C04480A4621460AF00FF9204610BD00BFB03D002086
:209020008021070810B5044C04480A4621460AF001F9204610BD00BFB03D00208C210708B9
:2090400010B5044C04480A4621460AF0F3F8204610BD00BFB03D00209821070810B50C4C2F
:2090600094F8CD200023C4F8803012B1094AC2F8F03059F053FA20B10423022084F8843018
:2090800010BDD4F800396367092384F8843010BDD01B0020C03D002070B50D4D95F8843023
:2090A000042B04460E460AD0082B06D1EB6F83420CD0FFF7D3FF022801D0012070BD0823C8
:2090C000C5E91F4685F88430022070BD022070BDD01B002070B54379234C002B14BF012331
:2090E000002384F8B03003D1002384F8843070BD1E4D002195F9F720032040F085FD00286F
:20910000F2D0466830465AF077F884F8CC000028EAD095F8F530003B18BF0123304684F8AC
:20912000CD305AF049F90AF035F838B994F8783084F88400013384F8783070BD59F0D8FABA
:2091400040B194F878300022013384F8783084F8842070BDD4F8002984F87800012362674D
:2091600084F8843070BD00BFD01B0020C03D002010B559F0BDFA58B10B4C94F8783001331E
:20918000DBB2072B84F8783003D9002384F8843010BD09F0FFFF0028F7D0D4F8003963673B
:2091A000012384F8843010BDD01B00202DE9F041874C94F8B050002D00F0F88094F8842018
:2091C000844F0226531E082B41D8DFE803F037399E4068501540050059F0A0F9002840F083
:2091E000EC80636FD4F80029FA3393422CD2FFF7BFFF94F88420E5E759F090F90028F0D0D2
:20920000D4F880300022012B84F8782040F2D980E16F94F8CD00013B0131C4E91F1310B12E
:209220006C4BC3F8F020082284F88420A2F10805B5FA85F56D092846BDE8F08184F884603F
:2092400059F06CF9002841D194F88420531EDBB2022B09D8D4F80039616F5B1AC82BE5D9EF
:20926000FFF786FF94F88420042ADFD1E3E7236B002BDBD1E66ED4F800396367072284F86E
:209280008420002ED2D0D4E91821236F0120B047DAE7636FD4F8001964338B42C6D2D4F87A
:2092A0002C80B8F1000FF4D159F038F90028A0D0E66E84F87880042384F88430002E7AD0DC
:2092C000D4E91821236F4046B047BDE758F0CCFD0028B9D197F8F930002BA3F10203B3FAF9
:2092E00083F314BF022201225B0984F8792084F87A3058F0B9FD00287FF479AFD7F8483136
:20930000C4F88830032384F8843058F0ADFD00289AD1304BC4F8800093F82C61B3F82E0155
:20932000D3F830E1D3F830C1D3F83071D3F8302184F88E6093F83411A4F88C0093F835618A
:2093400084F8922093F83501D3F83821C4F89420B3F83E81B3F83E2184F89310B3F83E11FD
:20936000C2F30B1343EA182303F00F0301F00F024FEA1E6E4FEA1C4C3F0A360900F00F00BE
:2093800003F5FA63042184F8990084F88FE084F890C084F8917084F89860A4F89A3084F8B4
:2093A0009C2084F884102846BDE8F08184F884502846BDE8F08105463DE7042384F88430C3
:2093C00039E7FAD1FFF74AFE94F88420531E3EE7D01B0020C03D00202DE9F8431A4C94F833
:2093E0008460042E0546894690461F4608D0082E02D00020BDE8F883FFF782F80228F8D17F
:20940000D4F8C00043F080FC94F87A3093B969021120FFF7B3F898B9D4F80039C4F8609050
:209420000522C4E91B87656684F8842063670120BDE8F88329461120FFF7A0F80028EBD0AF
:2094400009F07EFED5E700BFD01B002070B51E4C94F88430042B06460D4608D0082B22D176
:20946000E36F83422DD0FFF74BF802281BD1D4F8C00043F049FC00213720FFF77FF8294631
:209480001720FFF77BF8B0B994F87A306BB971021920FFF773F870B90823C4E91F6584F85B
:2094A0008430022070BD012070BD31461920FFF765F80028F0D009F043FE09F07DFE03209F
:2094C00070BD022070BD00BFD01B00202DE9F043694D91B006460F469046994695F884306F
:2094E000042B0DD0082B07D1EB6FB34200F0C080FFF706F80228F1D0012011B0BDE8F083FD
:20950000D5F8C00043F000FC95F87A30002B40F09E8071021820FFF731F8002840F0A2809B
:2095200095F88440FEF7A4FF082C0CBFFC22FE22D5F8BC00818940F2E9330189013B11F05D
:20954000020F9BB24FD093B2838140F2E9340389013C13F0010FA4B276D0838995F8C430F1
:20956000002B48D001A80AF013FED5F8BC30D5F8C82095F8CE10506803970C334022029393
:2095800000234906CDE9083304920B934FF4806206930A934FF400730792019105930AF066
:2095A00035FED5F8C83001A958680AF003FED5F8C830D5F8BC2059680B6843F001030B600A
:2095C00093889BB243F002039380012206230020C5E91B892F666E6685F8682085F884307B
:2095E00011B0BDE8F083002BA7D144F01FFE95F8C430002BB6D1D5F8BC00BE4683894FF48F
:2096000080724FF47A744FF6FF71BEF1000F19D01EF8013BB0F808C0013C1CF0020FA4B259
:2096200017D09BB283814FF47A74B0F808C01CF0010F04F1FF3311D0013A8389C5D0BEF1A2
:20964000000FE5D1FF23E5E7002C80D1CDE7314660E78C42DED144F0E9FDB6E79CB28C4218
:20966000E3D1F8E709F06CFD09F0A6FD032044E7FEF7FEFEFC225BE7D01B00202DE9F04F5A
:20968000A44C94F8B06087B0002E00F0D68194F88420DFF88892DFF888829F4F4FF6FF75E9
:2096A000531E082B00F29580DFE813F0A700D1006B0193008200090014019300FF0094F800
:2096C000C430002B40F03E82D4F8BC00236E94F868E0828903EB0E2C4FF480714FF47A73F7
:2096E000BCF1000F00F0B7811CF801AB0289013B92079BB240F1EE811FFA8AF383814FF49C
:209700007A730289D20703F1FF3A40F1EB8101398289E5D10EF1010E5FFA8EFEBEF1020F80
:2097200084F868E052D1D4F8BC00838940F2E9330289013B12F0020F9BB200F0C7810023DE
:20974000838140F2E9330289013B12F0010F9BB200F0B4818389838940F2E9330289013B3F
:2097600012F0020F9BB200F0A5810023838140F2E9330289013B12F0010F9BB200F09481D3
:209780008389FEF775FE00F01F00052800F0A18209F012FDD4F86CA0BAF1000F00F0CC812F
:2097A0000022236F616E0120D04794F8842077E7206E4FF40071FEF783FE012800F0A4816A
:2097C000022800F0A881002800F0EF8194F88420531EDBB2022B00F23A81D4F80039616FE1
:2097E0005B1AC82B00F22F81A2F10806B6FA86F67609304607B0BDE8F08FD4F8C00043F003
:2098000083FA00210846FEF7B9FE824609F098FCBAF1010FDAD10023D4F8C00084F8793021
:2098200043F072FA40F2AB110820FEF7A7FE052800F08581012800F0118109F081FC94F809
:209840007920002A00F04282022384F88430D4F8C00043F059FA94F87930022B0CBF4FF0BE
:20986000804A4FF0000A00213720FEF787FE51462920FEF783FE824609F062FCBAF1000FB4
:20988000A4D194F87930022B00F0A48184F87AA0D4F8C00043F038FA00210920FEF76EFEAA
:2098A00000283FD009F04CFC90E74FF0080AFEF7DFFDFF2800F02082BAF1010AF7D1636F8E
:2098C000D4F80029FA33934280D209F075FC94F88420E5E6FEF7CCFDFF284FF0080A06D0CE
:2098E000BAF1010AEBD0FEF7C3FDFF28F8D1D4F880300022012B84F8782040F20382E26F6C
:2099000008210132013BC4E91F2384F884100A466AE700BFD01B0020006402400F640240EA
:2099200000600240C5481021FEF7CAFD83460028B8D101217F20FEF7EBFB01288246B1D102
:2099400058460221FEF7E4FB002800F0A0810128A8D116213A20FEF7DBFB01308002C4F8CC
:20996000880009F0EDFBD4F8C00043F0CDF900210A20FEF703FE002840F06481032384F8D9
:209980008430102102A8FEF79BFD00287FF41EAF9DF815309DF816109DF810209DF809004B
:2099A0009DF80AC01B01DBB243EA111303F5FA63A4F89A30DDF8113001F00F0184F89C1054
:2099C0001BBA110902F00F024CEA002084F8981084F899209DF808109DF80B20C4F89430F9
:2099E000039BC4F89030A4F88C0084F88E1084F88F2009F0A5FB94F87A307BB9D4F8C00051
:209A000043F082F94FF400711020FEF7B7FD824609F096FBBAF1000F7FF457AFD4F8BC00FE
:209A2000042157F0BBFB002204233046C4F8802084F8843007B0BDE8F08F304684F8846008
:209A400007B0BDE8F08F09F0B7FB94F88420042A7FF4CAAECDE64FF0FF0A47E6D4F8BC0087
:209A60004FF0040E838902A94FF47A734FF0FF0C028992073CD5A0F80CC04FF47A73028910
:209A8000D20703F1FF3A3AD5828992B209B101F8012BBEF1010EEBD19DF80B30AB2B04BFA0
:209AA000022384F87930C8E6002B7FF462AE44F0BDFB66E6002B7FF451AEF8E7002B7FF4AE
:209AC00042AE44F0B3FBD4F8BC0044E6002B7FF42FAEF6E7AB427FF409AE44F0A7FB94F831
:209AE00068E017E61FFA8AF3AB427FF40AAEF4E7013B9BB2AB42BBD144F098FBCCE71FFA03
:209B00008AF3AB42BBD1F7E7636FD4F8002964339342BFF45BAE09F013FB09F04DFBD4F86E
:209B20006CA0BAF1000F07D000221046236F616ED04794F88420B3E594F88420B0E584F88F
:209B400079A07AE6D4F8C8305968DB69494594BF4046384613F0005F00F08B80D0F804C0F5
:209B6000DFF8DCE003EA0C0C1CEA0E0F3FF43CAE03EA0E03C3600B68D4F8BC0023F00103DA
:209B80000B600389D90703D583890389DA07FBD403899B07FCD503891906F9D4838823F039
:209BA00002031B041B0C8380BFE5019009F0C8FAE56E019884F87800042384F88430002D03
:209BC0003FF417AED4E91821236FA84794F88420531EFEE5D4F8C00043F096F851463A2054
:209BE000FEF7CCFCD4F8BC1082468B894FF0040E4FF47A7302A84FF0FF0C0A89920728D596
:209C0000A1F80CC04FF47A730A89D20703F1FF3B2AD58A8992B208B100F8012BBEF1010E24
:209C2000EBD1BAF1000F0DD109F08AFA029B1BBAC3F3807384F87A302AE600BF701C002097
:209C40007D0F7D0F09F07CFA09F0B6FA94F8842026E5013B9BB2AB42CFD1084644F0E6FA21
:209C6000BAF1000FEED1DFE71FFA8BF3AB42CBD1F3E7D0F800C0DFF8ACE003EA0C0C1CEAB5
:209C80000E0F3FF4B1AD03EA0E03836073E704212C20FEF73DFA032183464E20FEF738FABC
:209CA0000C21034636200193FEF732FA019B421C02339A400AFA0BFAA2FB0A01420A42EAF1
:209CC000C152C4F8882009F03BFA4CE684F884208AE5E56ED4F800396367072284F88420B3
:209CE000002D3FF481ADD4E91821236F0120A84794F88420531E6CE509F022FA042384F894
:209D0000843076E508D0042384F8843009F018FA94F88420531E5CE5FEF7F2FB02287FF499
:209D200055ADBFE57D0F7D0F2DE9F04FC14C94F8581183B00546C1F34001D4F8600142F03C
:209D4000EFFF94F85811D4F85C01C94301F001016F1E42F0E5FFFBB20193002D00F0D080A7
:209D6000B54EDFF8DC82B54D4FF01009D4F8600142F0BAFFD4F85C0142F0B6FFB4F86831E4
:209D8000002B40F04E8194F86A11D4F86C0142F0C7FF4FF0FA0A4FF47A710120D8F80430CB
:209DA000C3F30803002B40F00F81EFF31183002B40F00A81D6F80029D5F808C0D6F8003908
:209DC0009A42F7D1D4F890319C45F3D8D4F88C7101FB07F3A3EB0C03B3FBF7F301FB023282
:209DE000D8F80430C3F30803002B40F0AB80EFF31183002B40F0A680D6F80039D5F808B095
:209E0000D6F80079BB42F7D1D4F89071BB45F3D8D4F88C7101FB07FCACEB0B0CBCFBF7FC7E
:209E200001FB03C39B1AB3F57A7FD9D3BAF1010AB4D1D4F8600142F057FFD4F85C0142F013
:209E400053FFB4F86831002B40F0DF8094F86A11D4F86C0181F0010142F062FFFA204FF40E
:209E60007A714FF0010CD8F80430C3F30803002B40F08980EFF31183002B40F08480D6F8DF
:209E80000029D5F808E0D6F800399A42F7D1D4F890319E45F3D8D4F88CA101FB0AF3A3EB7E
:209EA0000E03B3FBFAF301FB0232D8F80430C3F3080343BBEFF311832BBBD6F80039D5F8D3
:209EC00008B0D6F80079BB42F7D1D4F89071BB45F3D8D4F88CA101FB0AFEAEEB0B0EBEFBBE
:209EE000FAFE01FB03E39B1AB3F57A7FDDD30138B9D1019B5F1EFBB2FF2B01937FF436AFE3
:209F000003B0BDE8F08FEFF3118A89F31288AF682B68DB0344BFC4F888C1AF68D6F8003929
:209F2000D4F888E15FFA8AFA8AF31188D4F88CA1734401FB0AFEAEEB070EBEFBFAFE01FBEA
:209F400003E3D0E7EFF3118E89F31288D5F808B02B68DF0344BFC4F88801D5F808B0D6F838
:209F60000039D4F888C15FFA8EFE8EF31188D4F88C71634401FB07FCACEB0B0CBCFBF7FCCD
:209F800001FB03C34EE7EFF3118E89F31288D5F808A02B68DA0344BFC4F888C1D5F808A0D1
:209FA000D6F80039D4F888215FFA8EFE8EF31188D4F88CE11A4401FB0EF3A3EB0A03B3FB49
:209FC000FEF301FB023270E7EFF3118C89F31288D5F808E02B68DB0344BFC4F88801D5F839
:209FE00008E0D6F80039D4F888215FFA8CFC8CF31188D4F88C711A4401FB07F3A3EB0E0348
:020000040800F2
:20A00000B3FBF7F301FB0232EAE6D4F88431002B3FF424AFD4F87031C3F800A084F881A190
:20A020001CE7D4F88431002B3FF4B3AE3FF038FBAFE600BFC03D0020D01B002010E000E02F
:20A0400000ED00E02DE9F04FBD4CBE4E94F85811D4F86001DFF8F482BB4D83B0C1F340012A
:20A0600042F05EFE94F85811D4F85C01C94301F0010142F055FE052301934FF01009D4F8D0
:20A08000600142F031FED4F85C0142F02DFEB4F86831002B40F04C8194F86A11D4F86C01CB
:20A0A00042F03EFE32274FF47A710120D8F80430C3F30803002B40F00F81EFF31183002B39
:20A0C00040F00A81D6F80029D5F808C0D6F800399A42F7D1D4F890319C45F3D8D4F88CE11C
:20A0E00001FB0EF3A3EB0C03B3FBFEF301FB0232D8F80430C3F30803002B40F0AB80EFF3CA
:20A100001183002B40F0A680D6F80039D5F808B0D6F800C96345F7D1D4F890C1E345F3D887
:20A12000D4F88CE101FB0EFCACEB0B0CBCFBFEFC01FB03C39B1AB3F57A7FD9D3013FB5D1F7
:20A14000D4F8600142F0D0FDD4F85C0142F0CCFDB4F86831002B40F0E08094F86A11D4F8DC
:20A160006C0181F0010142F0DBFD32204FF47A710127D8F80430C3F30803002B40F08B8022
:20A18000EFF31183002B40F08680D6F80029D5F808E0D6F800399A42F7D1D4F890319E4521
:20A1A000F3D8D4F88CA101FB0AF3A3EB0E03B3FBFAF301FB0232D8F80430C3F3080343BBB5
:20A1C000EFF311832BBBD6F80039D5F808B0D6F800E97345F7D1D4F890E1F345F3D8D4F854
:20A1E0008CA101FB0AFEAEEB0B0EBEFBFAFE01FB03E39B1AB3F57A7FDDD30138B9D1019B84
:20A200005F1E17F0FF0301937FF439AF03B0BDE8F08FEFF3118A89F31288D5F808B02B6847
:20A22000DB0344BFC4F88871D5F808B0D6F80039D4F888E15FFA8AFA8AF31188D4F88CA1DB
:20A24000734401FB0AFEAEEB0B0EBEFBFAFE01FB03E3CEE7EFF3118E89F31288D5F808B02D
:20A260002B68DB0344BFC4F88801D5F808B0D6F80039D4F888C15FFA8EFE8EF31188D4F8B9
:20A280008CE1634401FB0EFCACEB0B0CBCFBFEFC01FB03C34EE7EFF3118E89F31288D5F8EA
:20A2A00008A02B68DA0344BFC4F88871D5F808A0D6F80039D4F888215FFA8EFE8EF31188DE
:20A2C000D4F88CE11A4401FB0EF3A3EB0A03B3FBFEF301FB02326EE7EFF3118C89F3128896
:20A2E000D5F808E02B68DA0344BFC4F88801D5F808E0D6F80039D4F888215FFA8CFC8CF360
:20A300001188D4F88CC11A4401FB0CF3A3EB0E03B3FBFCF301FB0232EAE6D4F88431002B4A
:20A320003FF423AFD4F870311F6084F881711CE7D4F88431002B3FF4B5AE3FF0B1F9B1E609
:20A34000C03D0020D01B002010E000E000ED00E00E4B30B4DB68427801780D4CDB43C3F358
:20A360000223C3F10403DBB202FA03F360181B0101F01F050122490903F0F003AA4080F818
:20A38000003344F8212030BC704700BF00ED00E000E100E000F01F0240090123032803FA77
:20A3A00002F304D004280CD0022805D07047074A116C0B4313647047044A516C0B435364BC
:20A3C0007047024A116B0B43136370470038024000285FD00368374A2DE9F04103F13F4408
:20A3E00004F57E0402EB9422012492F8C42002F01F055209032A04FA05F456D0042A4FD0A4
:20A40000022A48D08588B5FA85F0C0F11F00C0F3CC0603EB860600F0070082000F24306AB2
:20A42000944020EA04003062306A01FA02F20243002132624FF0010E0A464FF0030C022710
:20A440000EFA02F838EA050002F101021CD118680CFA01F420EA04001860186807FA01F677
:20A4600006431E609E6826EA04069E6098689860586820EA0800586058685860D86820EAB3
:20A480000400D860D868D860102A01F10201D7D1BDE8F0817047084A556C2C435464B1E792
:20A4A000054A156B2C431463ACE7034A156C2C431464A7E77892060800380240002861D026
:20A4C0000368384A03F13F4101F57E0102EB91222DE9F04192F8C42002F01F0452090121BF
:20A4E000032A01FA04F158D0042A51D0022A4AD08588B5FA85F2C2F11F02C2F3CC0403EB08
:20A50000840402F00702216A92000F20904021EA00012162206A0C2101FA02F20243002101
:20A52000226208464FF0010E4FF0030C02270EFA00F838EA050200F101001DD11C680CFAF1
:20A5400001F224EA02041C601E6807FA01F434431C609E6826EA02069E609E6816439E6090
:20A560005C6824EA08045C605C685C60DC6824EA0202DA60DA68DA60102801F10201D6D1E1
:20A58000BDE8F0817047084A546C21435164AFE7054A146B21431163AAE7034A146C2143C5
:20A5A0001164A5E7789206080038024058B183884FF00042B3FA83F332FA03F303D0024910
:20A5C0000A6813430B607047003C0140134B0268196821EA02011960596821EA02015960BC
:20A5E00019680A431A609968026821EA02019960D96821EA0201D9604179102907D001F15D
:20A60000804303F59E3319680A431A607047996811439960D9680A43DA607047003C014065
:20A62000002864D0F0B58388B3FA83F3202B0A4685B00446C3F11F0143D02D4D2D4E05EB05
:20A6400081037718C3F89421002197F8CC703EF019FAB4F804C02268274CBCFA8CFCCCF1E2
:20A660001F0303F0FC0101F1804101F59C3103F0030398004FF00F0E02F13F438A680EFAF6
:20A6800000FE22EA0E0203F57E038A60C3F38723834088684FF0004222FA0CF203433D44C8
:20A6A0008B6002A8626101234FF400618DF80E300292ADF80C10FFF789FF95F8D431F02B37
:20A6C00001D805B0F0BD3E44F02196F8DC308DF8043003224FF4807301A885F8D4118DF86E
:20A6E0000520ADF80630FFF733FE05B0F0BD7047C03D002078920608003C014010B4B8B13B
:20A700000D4CD4F8DC31102B05D15DF8044B052100203EF09FBC03EB4302224482F8E1117E
:20A7200001210B4482F8E00182F8E211C4F8DC315DF8044B704700BFC03D0020C078202167
:20A74000DCE700BF2DE9F04FDFF87CA32DED028B9AF824120022CAE98522CAE9872297B09E
:20A76000CAF8102219B19AF825228AF810229AF826221AB19AF827228AF81F229AF82A226D
:20A780001AB19AF82B228AF81A229AF828221AB19AF829228AF815229AF82C3205935A1E14
:20A7A000D3B257B204937B1C00F0AA80BC4ABD4E52F83780029602EBC70200231279019321
:20A7C00008EE102A1D463446994626783946304644F032F983463046BBF1000F1ED041F082
:20A7E000A3FFEA1D1321D2B220B14FF0000E827180F807E03EF046F9207844F047F94FF0D0
:20A80000070309F1010223714FF0010384F802906070CDF804B05FFA82F9E3700135042D75
:20A8200004F10504D1D118EE100A029ECDF80C90FFF7B0FD9C499D4A4868024042F440324E
:20A840004A600FB9019B5BB9994C4820FFF7A2FD204602215AF01CFEA26842F00102A260C6
:20A860009148934A4168BAF82E4241F400014160516821F480515160916B21F4401141F499
:20A8800080119163D16841F46001D160956B85F44011C1F3015101EB81011F2000FA01FCBF
:20A8A00025EA0C0C112505FA01F141EA0C019163D16841F0E061D160956BC5F30151C1F186
:20A8C0000401C9B201EB810188404FF0120C25EA00000CFA01F108439063E4B1BAF8301297
:20A8E000CAF83842A1B1BAF83222CAF83C1262B1019B7048521A90FBF2F2CAF840226BB92A
:20A9000017B0BDEC028BBDE8F08F6B4A1288EFE76A4A1188E7E76A4A1488DFE7404603999E
:20A920005AF0B6FD5F4B012003F114090723F278441CE4B252B375783279A5F10A0101EB8A
:20A94000410105EB450C092D03FA01FE03FA0CFB02FA01F140F28E80D8F80C2022EA0E0EEC
:20A9600041EA0E01C8F80C10421E02EB82021F21062801FA02FC05FA02F261D8D8F8341049
:20A9800021EA0C010A432046C8F834200536B145CDD1D8F80820049942F40072C8F80820E4
:20A9A000D8F8082042F48072C8F80820D8F80820574442F00102C8F8082097F934220220D7
:20A9C0003FF022F9044600289AD0406858F014FC059A062158F022FC606809F017FC07A8A2
:20A9E00009F0D6FB039EA368364A0793012E8CBF4FF48060002000230D9008F14C054FF4BD
:20AA00000060089509920A934FF480720C930E904FF4003360680B9607A94FF40055CDE9B2
:20AA20000F52119309F0C6FB6268136843F001031360D8F8083043F08043C8F808305FE72C
:20AA4000C11FA0F10D0201EB81014FF01F0E02EB82020C280EFA01FC0EFA02F005FA01F107
:20AA600013D8D8F8302022EA0C0211432046C8F830108BE7D8F8101002FA0CF221EA0B0B7A
:20AA800042EA0B02C8F810206EE7D8F82C1005FA02F221EA00010A432046C8F82C2075E712
:20AAA0005C930608D03F002000230140E030FCFF00200140803801002E7AFF1F2C7AFF1F57
:20AAC0002A7AFF1F04400020C03D0020F8B5264E00EBC00406EB8404D4F85052002D36D049
:20AAE00094F861C20CF0FF07BCF1000F2FD149004FF0010CC9B284F8621284F8632284F86C
:20AB000065C284F8667284F864C284F861C284F86072AA88C4E99A33940502D50127384669
:20AB2000F8BD2B88D9050CD44FF4805301E0013B10D02A889205FAD42B889BB243F480739B
:20AB40002B80AB889BB243F44073AB80E6E700273846F8BDB6F8B83201339BB2A6F8B832ED
:20AB60005AF04CF8DBE700BFC03D002070B44D4A92F8BA3203EB430002EBC000590090F8B9
:20AB8000BC0203281DD8DFE800F00E1F024FC81802EBC000D0F8C04204B3013CC0F8C0429D
:20ABA000002070BC704792F84863002E63D03E4C002001E086425ED0258801308C34002DB0
:20ABC000F8D0012070BC7047C81802EBC000D0F8C042002CE1D1022480F8BC42194402EB8E
:20ABE000C10191F8C8020138C0B281F8C802B0BB2E4892F8B057D0F83002D1F8C4420133E3
:20AC000003F00303421E0326AB42224481F8BC62B2FBF0F4C1F8C042D3D090429CBF04F1B7
:20AC2000FF34C1F8C042CCE7194402EBC101D1F8C00290BB92F8B0178B42C2D0013303F0BA
:20AC40000304A14282F8BA42BBD004EB440302EBC3020223C2F8C00282F8BC32B2E7134B21
:20AC6000D3F83022012002F2E73370BCB3FBF2F3C1F8C03270470D480B44D0F8301202EBCC
:20AC8000C302012001F51C530F3370BCB3FBF1F382F8BC02C2F8C03270470138C1F8C0021A
:20ACA00000208FE7C03D00201041002098010020064B93F8B127002AFBD141F21432044947
:20ACC0009B5801F10C001B68184700BFC03D0020744500202DE9F84F3249DFF8D4B091F830
:20ACE000F91001240229074619461046CBF82C404FF000022C4C1D4618BF7F02FDF780F9E9
:20AD00002A4B63626B02A362E36A40F2FF5943F093034FF400704FF48A62E3620121C4F8E2
:20AD20003890A0601020E26057F0EAF9012D40F251434E46C4F83890CA4640F252488EBF7A
:20AD40004FF0120998464FF011090A25C4F838A00121A7604846C4F80C8057F0D1F9034646
:20AD60004FF0000C40F2774201213720A6632BB900231846CBF82830BDE8F88FA663C4F8AA
:20AD800008C0E26057F0BCF9013DA6630028EFD015F0FF05DAD10346CBF82C50CBF8283028
:20ADA000BDE8F88FC03D0020002C014000E1F505D01B00202DE9F843184C94F88460042EA0
:20ADC0000546894690461F4608D0082E02D00020BDE8F883FEF742F90228F8D101234A4627
:20ADE00028460021FFF776FF50B1FEF7C1F9E56E002DECD00022236F616E1046A847E6E7D8
:20AE0000D4F80039C4F860900522C4E91B87656684F8842063670120BDE8F883D01B00200A
:20AE20002DE9F84F2F49DFF8C49091F8F9101E4602292D4B07464FF0010418BF4702012E99
:20AE400040F259481C6398BF4FF48B683B469346474640F2FF55B0468CBF4FF0190A4FF0C4
:20AE6000180A0A241E4640F2FF53C9F838300121C9F808605046C9F80C7057F041F9034689
:20AE80004FF0000C40F2774201213720C9F83850A3B9584641460122FDF7B2F84646134A8F
:20AEA000134B536276029662D36A43F09103D3620D4B002108469962BDE8F88FC9F838509F
:20AEC000C9F808C0C9F80C2057F01AF9013CC9F838500028DDD014F0FF04C4D1024B1C63DF
:20AEE000BDE8F88FC03D0020D01B0020002C014000E1F5052DE9F047374C82B005460E4615
:20AF00001746984694F8840004280CD0082806D1E36FAB4207D0FEF7A1F80228F2D0012026
:20AF200002B0BDE8F087DFF8B8A02666DAF8F0906566C9F34F210F294FEA592223D8D4F88C
:20AF400080300193FBB194F8CD00E0B1B9F5005F13D0224831464FF4007248445EF0DAF8E5
:20AF600009F50072C2F34F211029CAF8F0204FEA522202D0019B012B21D192B2013A174E14
:20AF8000AD1A0B4600E0012332462846062601250021E766C4F8708084F8685084F88460AF
:20AFA000FFF73EFF0028BBD0FEF7E2F8E66E86B12846236F616E0022B0470320B0E7E26F5E
:20AFC000013B01320421C4E91F2384F884100220A6E70320A4E700BFD01B0020286E002001
:20AFE000C03D002070B52E4D95F82042022C84B01AD0012C02D0002004B070BD95F9244265
:20B00000631CF8D0032CF6DC0091134695F825120246204659F086FF0028ECD0204604B0C0
:20B02000BDE870405AF04AB8D5F8283213B11C689B886383D5F82462B38940F2E93433895D
:20B04000013C13F0020FA4B219D084B2B48140F2E9343389013C13F0010FA4B21BD0B3891D
:20B06000134630460A46002159F0A6FCD5F82832A3B11A689B881383012004B070BD002CC1
:20B08000DDD13046CDE9021243F0D0F8DDE90212D5F82462E4E7002CDBD1F2E70120ABE76B
:20B0A000B84E002010B50278022A044613D0012A01D0002010BD2D4B90F9040083F86022E7
:20B0C000421CF6D00328F4DC0A4603F518736179BDE81040FAE4836813B11A689B885383A7
:20B0E0006368988940F2E9321889013A10F0020F92B225D089B2998140F2E9321989013A72
:20B1000011F0010F92B22BD09A899A8940F2E9321989013A11F0020F92B21ED001229A81ED
:20B1200040F2E9321989013A11F0010F92B20ED09B89A368BBB11A689B881383012010BDEE
:20B14000002AD1D1184643F071F86368DDE7002AE8D1184643F06AF8EBE7002AD8D1F8E740
:20B16000002ACBD1EEE7012010BD00BFB84E002010B50C4C94F82032022B11D1D4F8280261
:20B1800041F0C8FDD4F8280208B12123C38001213DF078FCBDE810400348082142F0FCBF6A
:20B1A00010BD00BFB84E0020D850002073B50D4E05460C46FF230A46014630468DF807308A
:20B1C00043F01CF901230DF1070245F08001304643F0D8F89DF80700031B5842584102B02E
:20B1E00070BD00BFD8500020094B93F8B234042B08D9053B032B08D801231A4600B1037050
:20B200001046704700230122F8E700231A46F5E7C82C0020F0B40D6800240CE0BCF1050F9F
:20B2200018D8A0F137030A2B14D104EB840415F8010B03EB4404A0F13003DEB2092EA0F157
:20B240006107A0F1410CF0D9052FE7D8A0F157030A2BEAD00D601460F0BC70479FED737A55
:20B2600007EE901A20EE070AF8EE677A27EE800AFDEEC07A17EE903A2033402B00F2C780BF
:20B28000DFED6B7AB4EEE70AF1EE10FAF0EE407A0CDD9FED686ADFED686AB0EE677AB4EEE3
:20B2A000E67AF1EE10FA77EEC67AF6DC9FED637AF4EEC77AF1EE10FA0CD59FED5E6ADFED58
:20B2C000606AB0EE677AB4EEE67AF1EE10FA77EE867AF6D49FED5B7AF4EEC77AF1EE10FA9E
:20B2E00000F38D809FED587AF4EEC77AF1EE10FA44BF9FED527A77EE677A27EEA76ADFED51
:20B30000535A9FED537ADFED536AA6EE257A67EE865AE6EE076AB6EE007AE5EEA67A27EECB
:20B32000877ADFED486A70EE267ABDEEE76A16EE103A2033402B67D8B4EEE60AF1EE10FACE
:20B340000CDDDFED3C5A9FED3C6AF0EE676AF4EEC66AF1EE10FA77EEE57AF6DCDFED376AC3
:20B36000F4EEE67AF1EE10FA0CD5DFED325A9FED346AF0EE676AF4EEC66AF1EE10FA77EE30
:20B38000A57AF6D4DFED2F6AF4EEE67AF1EE10FA40DDDFED276A76EEE77A67EEA75A9FED13
:20B3A0002B5A9FED2B6ADFED2B6AA5EE856A27EEA55AE5EE866AB8EE006AE5EE267A67EE55
:20B3C000867AC7EE206A0023836143610362C361B7EE006A76EE865A76EE666A86EE257A60
:20B3E00067EE277A66EE876AC0ED017AC0ED037A80ED007A80ED027AC0ED046A70479FED92
:20B400000C7A77EE677A78E7DFED137AD9E79FED127A86E7DFED0C6AF4EEE67AF1EE10FAF6
:20B4200044BFDFED066A76EEE77AB6E727D4D236DB0F4940DB0FC940E4CB1641DB0F49C009
:20B44000E4CB16C1DB0FC93FDB0FC9BF92E741B99730083C15A82ABE000000002DE9F04198
:20B460008C4C82B094F861320190002B40F00C8194F88432B4F88622DFED876AB4F8888221
:20B48000A4F8988207EE103A07EE902AB8EEC76AB7EE007AB4F88222F0EE475A4FEA4805BD
:20B4A000E6EE665A9542B8BF1546A6EE267AAEB20122F8EEE77AA4F89A6267EEA67AC4ED93
:20B4C000A35A84EDA47AC4EDA57A84F86122002B00F0D680DDED017A9FED700AF8EE677A8E
:20B4E000ADB280EE270A5CF049F86D00B0FBF5F5012DB8BF0125EDB2B0FBF5F39BB2074628
:20B5000084F89C5200EE103ABBEEED0A84EDA80A5CF034F8624BDFED636AB8FBF0F0A3FBD7
:20B520000737FF0807EE907AF8EEE77A022886EEA77AB8BF02205C4984F8A40200239FEDB2
:20B540005B1A9FED5B6ADFED5B1ADFED5B5A9FED5B2ADFED5B2A9FED5B3ADFED5B3A9FEDF3
:20B560005B4A84EDAA7A07EE903AB8EEE77AF0EE467AE7EE017AFDEEE76A16EE902A203291
:20B58000402A7AD8B4EEE17AF1EE10FA0CDDDFED506A9FED507AB0EE675AB4EEC75AF1EE43
:20B5A00010FA77EEE67AF6DCF4EEE57AF1EE10FA0CD5DFED476A9FED487AB0EE675AB4EE13
:20B5C000C75AF1EE10FA77EEA67AF6D4F4EEC67AF1EE10FA49DD74EE677A67EEA76AF0EE5A
:20B5E000624AE6EE824AF0EE430AE6EEA40AB7EE007A27EEE65A77EE677AB6EE007AE5EEA7
:20B60000207A67EE877A0133202BE1EC017AAAD107EE905AF8EEE77AF7EE006A86EEA77AEE
:20B620002E4B2F4AC4F8483903F12801A833C4F844191020C4F854392021142384F8A55761
:20B64000A4F84009A4F8501907EE906AF8EE677AA4F84C3982ED007AC2EDAC7AC2EDAD7A95
:20B66000C2EDAE7A02B0BDE8F081F4EEE37AF1EE10FA48BF75EEE77AAFE7F6EE007AC2E79B
:20B68000184A82F8343225E794F89C52B4F89A62BEE700BFB84E00200AD7233C002474498F
:20B6A000ABAAAAAADB0FC941645100203C8C4F3EDB0FC93F0100F840DB0F49C092E741B932
:20B6C0009730083C15A82ABEDB0FC9BFDB0F4940DB0FC940E4CB1641E4CB16C16493060851
:20B6E00060560020980100200848002302461178022902F1060204D00133062BF7D1002030
:20B70000704703EB430300EB43007047081C002010B50021094C82B00846C4F8741A34F0EC
:20B72000C7FA074B0193042304F678200DEB0302062142F0EDFD02B010BD00BFB84E002005
:20B740005475C52A70B5461E00F13105344614F8011F601E801BFF29C0B201D034F0A8FA91
:20B76000AC42F4D1A02051F0EFF90121022034F09FFA0E4D40F2E93401E0013C05D042212C
:20B78000284642F077FD0028F7D16221074842F071FD1321242034F08BFA2520092134F07F
:20B7A00087FABDE87040A02051F0CEB9305900202DE9F04F2DED108B034697B00433159309
:20B7C000DFEDCACA149002238A4613928B461293149C4FEADB0604EB461202EB061031010F
:20B7E000A6EB86034FEAC60806EB4605CDE9000100EBC303043108F10400119620442144E2
:20B800002C01C6EBC60C0394EC00119D04944FEACC0405946C0106EB860E0294159D009C37
:20B8200003EB46174FEACE0E02EBC6064FEACB094FF0000C51ED01AAD3ED001A92ED007ADB
:20B8400094ED005A96ED004AD7ED007A15ED012A50ED016A32EE07BA76EE840A7AEE855A13
:20B8600031EEA70A3BEE256A70EE804A76EEC46A36EE244A36EE646A05ED014A82ED006AEC
:20B88000D0ED00BAD6ED012AD3ED019A95ED00AA92ED016A97ED013A91ED00CAD4ED014ABF
:20B8A0007BEEE23A36EEE19A32EE472A73EEE98A3AEE464A39EE279A78EE838AB0EE428A82
:20B8C000A9EE6C8ADC44E24573EEC33AB0EE441AA8EEEC1A76EEE77A33EEA97A7CEE643A8D
:20B8E00077EEA17A3AEE066A7AEEC51A3CEE24AA74EECC4A39EE833A35EE6A5AF0EE639AD3
:20B90000F0EE48AAE7EE2C9AA8EEAC4AE7EE2C4AE7EE6CAAF0EE418AB0EE427AB0EE612ACE
:20B920007BEE656A7BEEA22A76EE4A5AA9EE2C7AA7EEAC2AA7EEAC5AE7EEEC8A32EE83BAA7
:20B9400076EEC3BA35EEE09A75EEC07A36EE0A6A76EEE26A36EE0BAA76EE836A77EEA07ADB
:20B9600034EE423A77EE290A36EE4B6A7BEEA22A39EE000A73EEAA3A78EE244A37EE697A31
:20B9800031EE055A71EEA85A32EE044A85ED00AA82ED016A4D4441ED012A4A44C4ED006AD1
:20B9A00081ED000AC4ED017A494440ED010A4C4487ED007AC6ED003AC3ED004A80ED003A12
:20B9C00087ED014A484486ED015A4F44C3ED015A4E444B443FF62EAF119B072B40F2C78125
:20B9E000029D149E019B03980499059A083575190C330E95354608F108080EF10804EB1844
:20BA000008300831083246442C1928186918AA18079305F10C030D960C940B900A91099276
:20BA200008934FF001084FF0000E129B9E44139B03EBCE0303EBCE02109302EBCE0303EBCD
:20BA4000CE01029101EBCE0101EBCE0505EBCE06D6ED007A0F93AEEB8E03019106EB0313A4
:20BA600003EBCE07D3ED01AACDED067A019BD5ED007A97ED01BACDED057AD3ED007A029B37
:20BA8000CDED047AD3ED007A0F9BCDED037A07EBCE0CD3ED007ADCED01BACDED027A0CEB9C
:20BAA000CE01D2ED007A109A009101EBCE00014691ED01DACDED017A0099D2ED007A91ED64
:20BAC00001CA00EBCE0000EBCE0494ED01EAD0ED01DACDED007ADDE90776DDE90954DDE9C1
:20BAE0000B01DDE90D23C44602E000BFF304353F94ED009A90ED00FA91ED006AD5ED007A78
:20BB0000D3ED006A57ED014A92ED005A56ED013A96ED00AA35EE060A73EEA65A39EE278A7C
:20BB200034EE8F7A70EE082A75EE87EA35EE465A3EEEA26A73EEE63A06ED016AD1ED019A43
:20BB4000D2ED01FAD4ED016AD3ED011A95ED013AD0ED018A97ED004A3FEEE96A35EE491A4B
:20BB600076EE660A31EE271A3AEE612A75EE677A70EE830A3FEEA95A74EECF9A77EE897A4C
:20BB80007AEE211AB0EE42AA74EE68FAA0EEECAADC44E24535EEC77AB0EE639A74EE285A66
:20BBA00038EEC44AF0EE698AA1EE6C9AE7EEAC8A36EE436A7FEE644A36EE266AA0EEAC2ADC
:20BBC000F0EE4A0AE7EEEC0AE7EEAC4AF0EE687AF0EE498A36EE833AE6EE6C8AE1EE2C3A4C
:20BBE000B0EE6F1AA6EE2C1A71EEE56AA6EE2C4A71EEA55A75EE031A7EEEE22A37EE43FAD4
:20BC000075EEE1EAB0EE686A76EEC08A39EE044A7FEE86FA76EEC86A33EE816A38EE888A9C
:20BC200073EEC13A37EE457A2CEE2E1A3FEE055A22EECC9A9DED03FA70EE266A33EE077A49
:20BC4000AFEE221AAFEE2E9A7AEE244A9DED01FA79EEA09A25EE4BAA72EE670A37EE822A00
:20BC60006BEE087AAFEE08AAEFEE057A2DEEA63A9DED05FA67EE6D8AAFEE073AEFEE268A03
:20BC800066EE6A2A9DED00FA2AEEA00AEFEE202A6EEE02EADDED060A23EECE5AE0EEA3EA99
:20BCA0002BEEA98ADDED023AAFEE060AA3EE848A24EE6B7A6DEE246A9DED044A2FEECD6ADA
:20BCC000A0EE825AA3EEA97AE4EE2F6AA4EE246A75EEA15AC6ED005A83ED001A83ED019ABB
:20BCE0004E4447ED017A87ED00AA4B4480ED003AC0ED018A4F4482ED000A4844C2ED012A05
:20BD0000C5ED00EA85ED015A4A44C1ED006A81ED016A4D4484ED008A84ED017A49444C44A6
:20BD20003FF6E6AE0E9B08330E930D9B08330D930C9B08330C930B9B08330B930A9B083352
:20BD40000A93099B08330993089B08330893079B08330793119B08F1010843457FF465AE1F
:20BD6000129BDDF844B0DB009BB2129330E517B0BDEC108BBDE8F08F30B5044683B000BF1B
:20BD8000806840F0C1FF4CF2050301AA6946ADF800306068032300258DF8025058F00CFE1A
:20BDA000A06840F0B7FF00BF9DF8060003B030BDF0B5BE4FBE4885B0242200215DF00BFAF5
:20BDC00097F8856A002E3AD1BA4C3546D4F8443D5BB39B6A4BB3B848984783682BB303889A
:20BDE000DFF8CCC2013B9BB26046664600213778032F06F106061BD001310629F7D10022C8
:20BE00000178022900F1060000F0A5800132062AF6D1E16D052908D0481C02FB01C2E0658B
:20BE200002200021938010705180284605B0F0BD062303FB01414B8F013B9BB2DFE797F86A
:20BE4000840A07F68C23C7F8883A10B9994C0025BCE740F069FC0446C7F8940A40F038FF0E
:20BE600005460028F2D0013E022370B287F88C3A42F046FB0028E9D0C7F8900A0CB1202315
:20BE8000E380204609213CF0FDFDD7F8883A894C986840F03FFFD7F8883A1021586855F0EE
:20BEA0007DF9864BD7F8882AC4F8642D93E803000123009032208DF8041084F8683D002609
:20BEC0003DF02EFB052302AA6946D7F8880A8DF80A608DF8096042F097F99DF80A009DF855
:20BEE00009109DF80B20764B000240EA01401043984200F0AE8032DCA3F5F11398425ED03E
:20BF000042DD704B984252D00233984262D14FF400724FF48073A4F8482DA4F8543DB4F834
:20BF2000542DB4F8483D120202FB03F300204FF48071B3F1807FC4F84C2DC4F8503D84F857
:20BF4000560DA4F84A1D7BD85F4BC4F8443D012284F85D2D3AE7062101FB02C260E75B4B23
:20BF6000984234DC053B984234DD594B0344032B77D801A252F823F0BFBF0008AFBF000848
:20BF8000A1BF00080FBF0008A3F52203013B984267D051DD4F4B984209D00133984219D1E6
:20BFA0004FF48073A4F8483DA4F8543DB7E780224FF48073A4F8482DA4F8543DAFE7402251
:20BFC0004FF48073A4F8482DA4F8543DA7E7424B9842E5D00023A4F8483DA4F8543DC4F816
:20BFE0004C3DC4F8503DFCF7F7FB034600287FF4EDAE9DF80B009DF80A209DF80C100002F9
:020000040800F2
:20C0000040EA0240354A0843904232D0A4F8483DA4F8543DC4F84C3DC4F8503DFCF7DCFB70
:20C02000064600287FF4D2AE97F8840A40F07CFB42F092F83546C9E6294B9842B0D0C9E771
:20C040000123D4F8640D84F85C3DB72150F084F97AE74FF480621023A4F8482DA4F8543DDE
:20C060005DE720224FF48073A4F8482DA4F8543D55E71C4BC4F8483D4FF4003140234FF0CC
:20C0800000620126A4F8543DC4F84C1DC4F8502D84F8566DFCF714F8074884F85D6D50F079
:20C0A000ADF8114BC4F8443D90E600BFB84E0020081C0020D01B0020142900208C9406080D
:20C0C0001640E0001720C200789206081940EF00EABF10FF17BA20001870EF0021AAEF00F7
:20C0E0001860010000040008A49206082DE9F041C84BC94EC94DCA4C0822C3F88820336BAF
:20C1000082B043F0010333630746884628464FF4C05240F202336946CDE9002308F00CFB54
:20C120006B6AC049C4F8981A23F470436B626B6ABD49C4F89C1A43F420436B626B6ABB498F
:20C14000C4F8A81A23F470236B626B6ADFF820C3B74A01F5807143F42023C4F8B01A6B62A6
:20C16000736C01F5007143F48043C4F8EC1A7364736BA1F5F071C4F8B41A41F27C0041F2A5
:20C18000840143F0800344F80080675073634FF0A041A84EC4F8A41AA74FA84BC4F8F0CA2C
:20C1A00001F5366104F58455C4F8B86AC4F8F47AC4F8BC3AC4F8F81A0123A14F2F604FF0B6
:20C1C000020EACF5E46CA6F5A066A1F5CC6184F8A0EAC4F8ACCAC4F8646B84F8A33A994FF6
:20C1E000536106F58076C4F8281B84F8AA3B1946954B964AC4F8306B0CF5C07CA036C4F8F5
:20C200003C7B934FC4F838CBC4F8403B0CF5D45C03F56953C4F8446B4FF050260020DFF893
:20C220005482DFF854E2C4F8682BC4F86CCB02F5A0420CF5A04CC4F8707BC4F8743B07F505
:20C24000A047A3F54853C4F8786B04F69826C4F87C2BC4F8847BC4F8A43BC4F82C8BC4F885
:20C2600034EB0246C4F880CB334684F8AC0B402783F81C21A3F822210132042AC3E94970E1
:20C2800083F81D1183F81F01C3F8300103F12803EED1002211463346402083F87423A3F891
:20C2A0007A230132042AC3E9DF0183F8751383F87713C3F8881303F12803EED14FF0A04396
:20C2C00064489A6822F001029A60DA6842F04002DA6007F0EFFA94F8A13A0022212161F3B2
:20C2E00017420BB142F4801294F89B1AD4F8A43A01299A6300F0E780DA68D4F8A47BD4F8FF
:20C30000A80AC2F3076121F0600141F0400161F31F620021DA603960026861F3CC22026093
:20C3200094F8A32A012A00F0BB8010214A4807F013FE494807F0F6FDD4F8A81A94F8997ADB
:20C3400000224FF0FF300A614A618861CA616FB306F11400DFF824E100EB87009446BF000F
:20C360004FF0FF085EF8042F1368002BACBF00234FF0904370451360C2F810C0C2F80880B4
:20C38000F0D106F1500335483B444FF0000CFF2750F8042F1668002EACBF00264FF0904658
:20C3A00098421660C2F810C09760F1D10B6994F89B0A43F4807301280B6161D0D4F8A42ABB
:20C3C000274C0023936100284FF0FF336FF0804151615360516114BF00231023946143F4AE
:20C3E00070139069296843F4605343F00803034393619368096843F0010393608847194B05
:20C40000194ADA606846194B0093FDF7A1FF02B0BDE8F08100E100E0003802400000024001
:20C42000B84E0020080401004000400100080050003C014040090050400B00506009005086
:20C44000D0030020A0050050C005005000100050003000505C59002050590020A059002048
:20C460000008008000ED00E00005FA0543020001200B00502005005060050050645900209B
:20C48000D4F8A42A144B0B6314486FF0804100234FF0FF34936151615460516190619EE7A2
:20C4A00001680F4A0F4F41F003010160802159629F62C3F80421E022C3F80821C0F24002AF
:20C4C000C3F80C2131E79A6822F03E0141F02A0161F307029A600FE7030181000008008053
:20C4E000A00040008000200010B51A4C14F86A0CC0B9194B83F8B100C3F8B40014F8673CE8
:20C50000012B05D0022B21D054F8643C1BB910BD124B44F8643C12495B68BDE81040A1F191
:20C520000C00184740F000F914F8682C0A49003A18BF012281F8B120C1F8B4000028DDD0B4
:20C540001F22C28020213CF09DFAD7E7054B44F8643CE0E7B05F0020D01B00201004002035
:20C56000505F0020EC03002099B10A6B824216D9154B53F8242C914221D34C3991421ED360
:20C580000B6B9842F9D38B6B9842F6D80B46184670470D4B53F8241C0A6B904212D30B68F9
:20C5A0000BB9F4E70A6B90420B4602D38A6B9042EDD951F84C3F002BF4D1184670470023E6
:20C5C000184670470A46D8E7B05F00202DE9F047CC0143D10346224A43F8082B4FF0FF3247
:20C5E0004260022418467E26DFF8788058F8209C2644013E051D49466FF070474FF0010ADC
:20C6000008E0A3421CD0631C45F8043C321B1C460435CAB10B6BA34202D88B6BA34204D21C
:20C620002046FFF7A1FF014690B10A794B6B002AE7D1A34204D0E6D245F8042C631CE5E732
:20C6400045F8047C631CE1E748F8201CBDE8F08745F804AC321B631C4946D8E78026C3E7E7
:20C66000F8FFFF0FB05F0020036870B55E6A26B133460522BDE87040184704460D464E1DFB
:20C6800000E023689B68204698470028F9D0236815F8011B1B6820469847B542F1D170BD94
:20C6A000036870B55E6A26B133460822BDE87040184704460D4601F1080600E023689B68E9
:20C6C000204698470028F9D0236815F8011B1B6820469847B542F1D170BD00BF2DE9F047B6
:20C6E000164D0746002015F9139CA5F10C0684B007EB010805F5257504464FF0B60A33685E
:20C70000ABB193F83830142B11D0B9F1FF3F01D04B450CD1002269463046CDE90244CDE98B
:20C720000078ADF808A08DF80E4034F07DF8E036B542E4D104B0BDE8F08700BFB05F002048
:20C740002DE9F743124E0124A02318255FFA84F8FF2B14DCD6F89402E9B2C1F11C02827252
:20C760005F1C026880F80B80DBB20093C1F11B01D2F8189000234246C9B2C8473B46013D7D
:20C78000E6D10134052CE0D103B0BDE8F08300BFB05F002010B50A4C94F8B102003818BFA9
:20C7A0000120FBF73FFF50B1064904F5267041F063FC04F5267010F067FA04F5267010BD6D
:20C7C000B05F00209494060870B4447941BB03684FF400524FF40076202502213CBB1A8C59
:20C7E00022F001021204120C1A841A8B188C22F0F30280B2120420F00A00120C014342F00C
:20C80000010241F001011A8319841A8B22F00C021204120C1A831A8B92B270BC1A837047A9
:20C8200000220368164615461146002CD7D0042C21D0082C38D0198C21F480510904090C80
:20C8400019849C8B1D8C45F6FF7040F6FF4128402140024342F4805241F4807199831A8455
:20C860009A8B22F440621204120C9A839A8B92B270BC9A8370471A8C22F010021204120C23
:20C880001A84188B198C89B240F6FF4221F0A00102400D4342F4807245F010051A831D840C
:20C8A0001A8B22F44062B3E71A8C22F480721204120C1A84998B1A8C21F0F30192B20904E1
:20C8C00022F42062090C324342F4807241F0010199831A849A8B22F00C02C4E738B50F4DE8
:20C8E0000446006807F02CFED5F87828204652084FF6FF713BF04AFD20460021FFF764FF31
:20C9000041F2E403064AEA5005F5875120460022BDE8384004313BF059BC00BFC82C0020B4
:20C9200021CE01082DE9F0479AB0DDE9226ADDF8909004460D461746984602E020683DF0B2
:20C94000C3F920683DF0C8F90028F7D10146642201A85CF040FC264B8DF80450CDF85CA0AC
:20C960000293002D40D0AB1E012B3FD9042D14BF002203221F4B0396D3F800398DF80520DC
:20C980001E440123CDE9059404968DF85B3037B14246394607A85CF0BDFB8DF85A80164EB3
:20C9A00096F8029300231893B9F1000F19D196F80103642202FB006001A900F541705CF0D2
:20C9C000A9FB012386F8019386F80233236843B143463A46294620461AB0BDE8F04712F0C5
:20C9E00089B81AB0BDE8F0870522C3E70222C1E770620020D01B0020B05F00200C480D4B9B
:20CA0000D0F8841310B40C4CC0F874338A1E2231B0F89E331B01A4FB03C3DB08A3F5B063B9
:20CA200022F8023F9142F3D15DF8044B704700BFB05F002075200208CDCCCCCC70B5084C72
:20CA4000251D2E4614F8010B34F0AEF828B1037805F8013BB442F5D170BDFF23F8E700BF08
:20CA6000706300202DE9F0471D4F012607F10805B2464FF03C094FF0000817F8010B3FF0D1
:20CA800053FE044690B180F80690C671FB7803F07F02012A18D013F0800F20460DD185F828
:20CAA000048040F031F985F805802C600136052E05F10805E1D1BDE8F08785F804A040F07E
:20CAC00029F985F805A0F0E71B0605D4012120463BF0D8FFFB78DEE740F01CF9F6E700BF9E
:20CAE000786300202DE9F04FDFF8E491DFF8E4A183B009F10C05012419F8018BB8F1000F86
:20CB000000F0C0804FEA1817013F042F08F00F0200F2BB800AEB4703B3F8B00040FA02F608
:20CB200016F0010600F0C38001239340013B1840574459F0A3FB97F8BC305F4E184406EB33
:20CB4000C00604236E61F471B371002303E00133152B00F09780594903EB43025F00895CF6
:20CB60004145F4D1564B1A4492F88D15002900F0A08040463BF06CFD804600683BF00CFD8A
:20CB800098F805103BF084FD0378002B7AD14C4B3B44042283F8CD4583F8CC25002E58D0C8
:20CBA000336898F8080003F13F4202F57E020AEB9222012792F8C42002F01F015209032A7D
:20CBC00007FA01F169D0042A62D0022A6AD0B6F804C0BCFA8CF2C2F11F02C2F3CC0103EB79
:20CBE000810102F007020E6A92000F27974026EA07060E620E6A90403043002208624FF08E
:20CC0000010B11460BFA01FE3EEA0C001CD118680326964020EA060018601F68022090400C
:20CC2000384318609F6827EA06079F6098689860586820EA0E00586058685860D86820EA93
:20CC40000600D860D868D8600131102902F10202D8D11C4B1C4AB3F8F013B3F8F233009137
:20CC6000002001340190B2FBF3F328469BB24146E4B233F03BF80123092C6B7405F11805C2
:20CC80007FF43AAF03B0BDE8F08F00266E615CE70E4F3A6B0A433A6399E70C4A176C394368
:20CCA000116494E7094A576C394351648FE76E614BE70B68FFDE00BFC032002054320020FF
:20CCC000C82C0020B05F002040420F0000380240A46300207892060870B5044684B04FF4E1
:20CCE000004035F0F5FB80B300234FF4E131032590F904000293CDE900151A464FF400413B
:20CD000035F047FC124BC3F8C004F0B1012C40F6980208BF4FF496620E480F4DA3F8CC24F2
:20CD20004FF461710D4AC3F8D8040A2683F8C444C3F8C864A3F8CE14A3F8D014C3F8D45477
:20CD4000C3F8DC24012004B070BD0020FBE700BFB05F0020BDCE0108E9820108DD820108B6
:20CD60002DE9F041214E224F96F8FF3487F8583106F2FC4607F5AE7500244FF0050816F8EC
:20CD8000010B20BB28600134032C05F10405F6D197F85811D7F85C01C94301F001013FF0A8
:20CDA000BFFF97F85811D7F8600181F00201C1F340013FF0B5FF97F85811D7F8640181F0A4
:20CDC0000401BDE8F041C1F380013FF0A9BF3FF0ABFC013401212860E3B210B180F80680A3
:20CDE000C37128683BF04EFECEE700BFB05F0020C03D00202DE9F0412A4C2B4DB4F80465EE
:20CE0000A5F8686182B0EEB994F800053FF08CFC94F80125C5F86C01003A18BF012285F8FE
:20CE20006A2148B194F802152B22002914BF11210121C2803BF026FE002002B0BDE8F041F5
:20CE400040F0E4BE94F80085002240462B213BF06FFC074640463FF067FCF8B1F7B12B2262
:20CE6000C5F88401C280397AFDF7B2FA4FF000080E4AB2FBF6F3C3F34F0000909BB2394645
:20CE8000CDF8048005F5B870A4F8066532F02EFFD5F87031C3F8008085F8818102B0BDE852
:20CEA000F08100BFB05F0020C03D002040420F002DE9F84F254C94F8143584F8083504F213
:20CEC0000B57002604F5A5645FFA86FB0BF101085FFA88F8012117F8010F42460E448A4625
:20CEE0003BF026FC4FF00009054640B3387804F80E9C04F80D9C04F80FBC04F810AC44F8A9
:20CF0000045C3FF011FC18B180F806A080F80780297AFDF75DFA0E4A002128463BF036FA5F
:20CF20000C4B23600C4B221D21462846C4E901393BF04CF9697928684A4632F06BFE082E92
:20CF400004F11C04C0D1BDE8F88F00BFB05F002040420F004DFC030881EA030870B52C4C19
:20CF60002C4B94F84006C4F8383600220221C4F8F825C4F8FC25C4F80026C4F83426A4F8AF
:20CF80003C263BF0D5FB002841D0234B0268054603F1C000597C11B159688A422BD01833BA
:20CFA0008342F7D1002394F84006C4F8245584F818353FF0B9FB08B10223C380297AFDF756
:20CFC00007FA2846154A00213BF0E0F9144A1549C4F828150026111F2846134BC4F82C356A
:20CFE000C4F830653BF0F2F8697928683246BDE8704032F00FBE138D0C490D4A9BB2D2F83A
:20D0000078280133B2FBF3F381F89C32CAE770BDB05F002000FFFF009431002040420F00E1
:20D02000DC640020A9EA030849EC030898010020C82C00202DE9F04FDFF80CB3B64E85B0C1
:20D040000D460446C0220BF2CC40002101955CF0C2F896F87836002B76D096F87936002B76
:20D0600000F091809BF8C034012B00F0B680022B00F09580A94DDFF8D4A29BF8B6740FCDC8
:20D080000AF5477403940FC40FCD0FC495E807009BF8B234A24DCAF834533D1E18BF012530
:20D0A000072B84E8070086F8815600F20A81042B00F21481DFF89882CDF808A0A8F1150334
:20D0C00000259A46019B5FFA85F909F10107FFB2AB423A464FF0030129DD1AF8014B2046AB
:20D0E0003BF026FB034620461C4613B33FF01CFBC8F8140018B14FF003038371C7719BF826
:20D10000B3349BF8B224002B00F0E680E37983F0010349462046013556F020FA48B14FF0A8
:20D120000103082D88F8113008F11808CAD1039B08E0DDF808A07B4B7B4ACAF84033CAF8BC
:20D1400038230023C6F87C36D6F87C3663B10022019883F82C00012183F82D101A6383F819
:20D160002E2005B0BDE8F08F704D714C0FCD0FC40FCD0FC495E80700A4F1200384E8070001
:20D18000C6F87C36EDE79BF8B4240199003A204618BF0122FBF706FDC6F87C06D4E79BF829
:20D1A000B634002B3FF466AF9BF8B234082B14D15A4DDFF898A15A4F0FCD0AF547740394F4
:20D1C0000FC40FCD0FC495E80700012384E80700CAF8347386F8813676E0564D019BC6F8C1
:20D1E00084360FCD544CDFF868910FC40FCD0FC49BF8B63495E80700003B18BF01239BF8DD
:20D20000B25486F881360027A9F1150384E8070086F8C4566434029386F882760AE03FF033
:20D2200073FDE368C9F81430082F04F1200409F118094DD0D6F88436BB4249DD029B13F853
:20D24000018B029340463BF0A7FA054640463FF06BFA9BF8B32495F8078082460AB188F07D
:20D26000010808F0010596F88126013586F880560AB188F0010850463FF02AFD00283DD08B
:20D28000504640F001FD6901013741F0090161616060C4F80CA084F81080FAB2BAF1000F91
:20D2A00005D04FF003038AF806308AF8072050463BF0E8FB18F0010F5046B0D13FF02AFDCA
:20D2C000AFE7082B7FF4F6AE1C4BC6F88836F1E61948C6F87C0637E7E3791AE79BF8B5341C
:20D2E000174AC6F88826012B05D0022B06BFB7FA87F35B09002386F88C36DBE60A4B11490C
:20D30000084AC6F860360123C6F85C16C6F8682686F88236DDE700BFB05F0020109506082C
:20D320009DF30508056404080D640408E4940608406600203C950608F46500204D640408FD
:20D340007D64040811640408C82C0020C03D002094310020F8B56E4F97F8980397F899533A
:20D360003FF0E2F960B12D23C380202104463BF089FB0A203BF0B6FF204640F07BFC18B9DD
:20D38000D7F8C837DA0000D5F8BD013D092DFBD897F89743D4B9402035F09AF80028F3D01C
:20D3A00090F9043097F86D13092BC8BF143B3B440A2993F8CC4700F09D8093F8D83797F811
:20D3C0009623002A08BF1C46002CDDD020463FF0ABF90546002800F085802D23C380012112
:20D3E0003BF050FB012108463FF0A2FC2B68AA881A833C203CF094F8002101203FF098FCFF
:20D4000097F89933002B4CD0424C00261FE02B68AA885A833BF066FF94F85811D4F85C0167
:20D4200001F001013FF07CFC94F85811D4F86401C1F380013FF074FC2B68AA881A8378205E
:20D440003BF050FF97F8993301369E4229DA94F85811D4F85C01C94301F001013FF060FC35
:20D4600094F85811D4F8640181F00401C1F380013FF056FC7820002DC9D178203BF032FF07
:20D4800094F85811D4F85C0101F001013FF048FC94F85811D4F86401C1F380013FF040FC42
:20D4A000CDE797F89733ABB997F89833002B7FF46BAF97F89A33012B7FF466AFD7F8C8370B
:20D4C00013F080537FF460AF87F89933BDE8F8404AF05CB932203CF023F8284600213BF02A
:20D4E000D1FAE1E701213BF0CDFA012108463FF01FFC7EE7D7F8F0375B057FF545AF09F0AF
:20D500007BFD00287FF440AF002C7FF45FAF3BE7B05F0020C03D0020094BD3F8F407D3F809
:20D52000F827D3F8FC37904202DC114602460846984204DD9A42B8BF1A46104670477047FF
:20D54000B05F0020124A02F5006030B419C89842D2F80C18D2F8102802DC1D460346284662
:20D56000914202DC15460A4629468842A8BF08469342B8BF1346844202DB22460446104611
:20D58000984203DD9C422046B8BF184630BC7047B05F00200B6810B414681B1B03605468DE
:20D5A0004B681B1B43608B6892685DF8044B9B1A836070472DE9F047041E0D4612DB092C1B
:20D5C00026DC824A0B468248A0FB0410C00800EB8000A4EB40000021125C1A705970284661
:20D5E000BDE8F08764422D23092C01F8013B24D8764A774BA3FB0403DB0803EB8303A4EBA6
:20D6000043030020D35C48700B702846BDE8F0876F4B632CA3FB04264FEAD60621DC6B4AE0
:20D620000B466B49A1FB0601C90801EB8101A6EB4101515C03F8011BC5E7654A632CA2FBE5
:20D6400004364FEAD60637D8604A614BA3FB0603DB0803EB8303A6EB4303D35C01F8013BDD
:20D66000C7E7A3FB0627B4F57A7F4FEAD7070DD2564A0B465649A1FB0701C90801EB810126
:20D68000A7EB4101515C03F8011BCAE7A3FB072842F20F7294424FEAD80836D84B4A0B46DC
:20D6A0004B49A1FB0801C90801EB8101A8EB4101515C03F8011BDDE7A2FB0637B4F57A7F19
:20D6C0004FEAD7070CD2414A414BA3FB0703DB0803EB8303A7EB4303D35C01F8013BB4E768
:20D6E000A2FB073842F20F739C424FEAD80821D8364A374BA3FB0803DB0803EB8303A8EB13
:20D700004303D35C01F8013BDEE7324AA3FB080994424FEAD90921D82C4A0B462C49A1FBAD
:20D720000901C90801EB8101A9EB4101515C03F8011BB5E7274BA2FB08099C424FEAD90951
:20D7400021D8224A224BA3FB0903DB0803EB8303A9EB4303D35C01F8013BCAE71E4AA3FB01
:20D76000090394424FEAD30A21D80B461849174AA1FB0A01C90801EB8101AAEB4101515C3B
:20D7800003F8011BCAE7144BA2FB09029C424FEAD20A13D80E4B0D4AA3FB0A03DB0803EBB0
:20D7A0008303AAEB4303D35C01F8013BCAE70A22BAFBF2F049F0DCFA0346D7E70A22BAFB39
:20D7C000F2F049F0D5FA0146E4E700BFB0210708CDCCCCCC9F8601003F420F0070B4344827
:20D7E00090F81438A3F13001092957D800F61404224600F6230012F8015FA5F1300109293D
:20D8000004D88242F7D1002070BC7047141B022C4ADD2848002101E010F8013B01EB8101F5
:20D8200003EB4103161A303B022E044603F0FF01F2DC214B03FB01F1A2424FF000030DD978
:20D8400003EB830314F8016B5B00303B3344A24203F0FF03F4D1194800FB03F32E2D06D07E
:20D860001748A0FB032301EB930070BC7047013204200024157804EB8404303D6400092DA0
:20D8800000F1FF30A4B202D82C44A4B2013210F0FF00EFD1642202FB0433E1E700211D467A
:20D8A00000F614020B46D9E7064C0021C4E700BFB05F0020C56700208096980040420F00B4
:20D8C000ABAAAAAAC467002038B504460D460A460068FF215BF07FFC21682944216038BDC0
:20D8E00083B50C461646054633F0CCF9204633F0C9F90021204B0846002E08BF1E463FF062
:20D9000017FA002101203FF013FA28463CF0E4F9B0B1012100203FF00BFA28463CF0D4F9C3
:20D92000074620463CF0D4F90028FAD0394620463CF0D6F93846B047002108463FF0F8F965
:20D9400020463CF0C9F90028DFD0012100203FF0EFF920463CF0B8F90146284601913CF08D
:20D96000B7F901990028F8D028463CF0B9F9002108463FF0DDF9C8E719F10308F0B5002321
:20D980000B604B608B60CB600B610268DFF88CC089B004ADC2F385572E4647FA03F0C00778
:20D9A000344604D513F80C0004F8010B26460133062BF2D11748C2F303240444002394F82F
:20D9C000F84233708DF8184000F5407CC2F305370DF1190647FA03F0C007344604D513F875
:20D9E0000C0004F8010B26460133062BF2D100233370C2F3834406ABCDE90134084602F061
:20DA00000F0305490095C2F303124DF09BFE09B0F0BD00BF78920608D82107086895060821
:20DA200070B5094CD4F82428054662B10026D4F824082D21013640F0F3FEAE42F7DBBDE8CB
:20DA4000704042F017B970BDB05F00202DE9F04F5FFA81F9002185B00746084616463FF014
:20DA600067F9002101203FF063F93EF03BFE022E0AD0042E44F6C01818BF4FF49648B9F122
:20DA8000070F07D900200CE0B9F1FF0F4FF41648F5D10326CD4D95F828382BB90020C5F874
:20DAA0002C0805B0BDE8F08F032EC94C0DD0A144002299F8B70403213AF03AFE0028EDD078
:20DAC000C4F8C008C3799A07E8D441F2DB0395F82808E654002203213AF02AFEC4F8C40CFD
:20DAE0000028DBD04FF48061BA4BC4F87C38C4F888180323C4F88C1841F2CC01A4F8803884
:20DB00000023635441F2C8014FF0010A24F801A041F2D401B04A635041F2D80102F148002C
:20DB2000635241F2DA01C4F89008032E02F24C406354C4F88488C4F8A838C4F89C38C4F8B6
:20DB40009838C4F89408C4F8A438C4F8A03891460ED0D4F8C0B89BF804003EF0E5FDC4F815
:20DB6000BC08584612F054F85146484612F064F832203BF0D5FC002E60D1D4F8C48CD8F8D9
:20DB8000000006F0DDFC4046944A22213AF0FEFB9349944B0B60324640463AF017FBD4F8C0
:20DBA000C088D8F8000006F0CBFC8C4A4FF6FF7140463AF0EBFB31464046FEF705FE41F247
:20DBC000E403894AE25009F66801324640463AF0FDFAC5F82C984FF0060A022E12D0D5F823
:20DBE0002C083CF079F868B1012100203FF0A0F8D5F82C083CF070F80146002840F09E80E0
:20DC00003FF096F838463CF067F888B1012108463FF08EF84FF0050B4FF0000838463CF0A0
:20DC20005BF80146002840F0928001203FF080F8042ED4D005203BF073FCCEE7012E09D1C5
:20DC4000D4F8C40C4146FBF79BF9D4F8C008FEF745FEBEE7022E09D1D4F8C00811F0C7FF45
:20DC6000D4F8C40C4146FBF78BF9B2E7032E5DD14FF0000A41F2DC0351465C4804F803A0DE
:20DC800040225BF0A8FA8DF80FA0DFF864A19DF80F30072B09D95048012111F0CDFFD4F8EA
:20DCA000C40C4146FBF76CF993E79DF80F3003EB430304EBC30393F8DD3483B39DF80F30D9
:20DCC00003EB430304EBC303D3F8E0343BB39DF80F30234493F8B70408B3002203213AF0E2
:20DCE00027FD8346D8B111F082FF9DF80F309AF8002003EB430304EBC30305EBC201D3F83F
:20DD0000E034C1F830389BF80730DB0748BF012302F1010248BF81F834388AF800209DF8DE
:20DD20000F300133DBB28DF80F30B0E7042E7FF450AFD4F8C00811F05AFF81E7D5F82C088D
:20DD40003BF0C2FF014638463BF0CAFF50E738463BF0BAFF95F87E3801468BB9242803D197
:20DD60004FF0010385F87E38012E04D1384601913BF0B6FF0199D5F82C083BF0B1FF4DE78F
:20DD8000012B06D14D280CBF0223002385F87E38EAE7022B06D13C280CBF0323002385F8FB
:20DDA0007E38E1E7032B25D10A2802D985F87E88DAE7042385F8710885F8708885F8738866
:20DDC00085F8720885F87E38CEE700BFB05F0020C82C0020809506084435002040420F0015
:20DDE000A83D0020C5FC01083DCD0108E0670020A43D0020042B09D195F8723885F87F0895
:20DE0000434085F8723885F87EB8ADE7052BABD195F8703895F8719895F872084B4509D228
:20DE20005A1C2B44484085F8720885F8702883F8741899E78842B9D195F87F3885F87EA8A7
:20DE4000F42B91D1B9F1000F8ED12421384685F87E983BF045FF4D2138463BF041FF3E21AE
:20DE600038463BF03DFF494638463BF039FFF42138463BF035FFF42138463BF031FF032E3C
:20DE80001BD0D4F8C008437901689D080223AB40DB439BB20B828D892B408B8100792021EA
:20DEA00011F094FED4F8C0084A4649463AF08EF9D4F8C038186806F043FB0022D4F8C40C35
:20DEC00011463AF083F9D4F8C43C186806F038FB0120E6E5114A013002EBC000F0B4D0F83F
:20DEE0003CC30F4E002333603361336233633364336533663367BCF1000F0DD090F8387323
:20DF000057B13F0100240CEB04030FCB35191034A74285E80F00F6D1F0BC70477892060884
:20DF20003068002038B50F4C94F8071901F03F018B1C024601F10A0584F8053984F8025983
:20DF400004F5106084F8032908311DF0A7F9254485F8FE0894F802391C44000A84F8FF082A
:20DF600038BD00BFB05F002070B51D4C0968D4F82C591C4ED4F82849D6EDA87ADFED1A6A92
:20DF8000491B00EE901A0168F8EEE00A091B60EEA70A00EE101A20EEA07AB8EEC00A1C4617
:20DFA000A0EE007AB1EE400AF1EEC77A67EEA67AFCEEE77AC2ED007A4DF0B6FC9FED0B7A67
:20DFC000DFED0B7AE0EE077AFDEEE77A17EE902A002ABCBF02F50C42A032226070BD00BF6C
:20DFE000B05F0020980100202C7D8E3FA00CB34500A00C4638B50B4C00250122802120469A
:020000040800F2
:20E0000034F052FA30B194F9040034F081FA08B1006838BD0135062D04F10C04EDD100201D
:20E02000F7E700BFF068002038B5041F00F1080554F8043FD81780EA430017F0ADFCA542FB
:20E04000F6D138BD2DE9F041D14CDFEDD27AD4F88C3994F8250A07EE103A2DED028BB8EEB0
:20E06000478A28EE278A002840F0CA80D4F8302A94F8241A94F8413A002A19DD07EE902AA0
:20E08000DFEDC56AF8EEE77AC3F1640386EEA77A00EE103AB8EEC00A20EE070A29B920EED7
:20E0A000000ADFEDBE7A20EE270A59F067FA80B2B4F8263AA4F8260A834200F0A18094F8FD
:20E0C0009079B74EDFEDB78A4FF00008002594F8443A2B41DB0714D594F8243A002B7FD113
:20E0E000B4F8263A07EE103A002F00F0FA80B8EE477AC8EE877A77EE887A88EE277A86ED2D
:20E10000027A0135042D06F12406E0D194F8295AB4F82C6A002D40F0E780002F5CD194F84D
:20E12000403A84F84D5A84F84C3A002E54D0002D52D007EE906A0123B8EE678ADFED997A16
:20E1400084F84E3A9D42C7EE888A28D0022D43D1D4F88C199448B0EE480A44F0A7FD94F839
:20E160004D3A012B00F00F81022B35D1D4F88C198E48B0EE480A44F099FD94F84D3A012BF9
:20E1800000F0FC80022B27D1B0EE480ABDEC028BD4F88C198648BDE8F04144F087BD854A6C
:20E1A000D2ED007A78EEA76A134687EEA67A002143F8041F83ED017A78EEA76A002187EE4A
:20E1C000A67A996083ED037A77EEA88A002287EEA87A1A6183ED057ABDEC028BBDE8F08133
:20E1E000B4F8263AD4F88C1900EE103A301DB8EE400A002F6FD144F059FD94F8907980E738
:20E2000094F89079002F3FF45CAF94F8295AB4F82C6A002DE0D0D4F8482A94F82A3A92F816
:20E2200083201343D8D1D4F8302A94F8413A002A64DD07EE902ADFED586AF8EEE77AC3F16C
:20E24000640386EEA77A012D00EE103AB8EEC00A27EE000A5FD059F091F980B2A4F82C0AC7
:20E26000002F78D08642B7D00028B5D094F84D3A002BB1D007EE900AB8EE678ADFED497AB7
:20E28000012BC7EE888A4DD0022BA5D1D4F88C194548B0EE480A44F0F3FB94F84D3A012B7C
:20E2A00069D0022B98D1D4F88C194048B0EE480A44F0E6FB94F84D3A012B57D0022B8BD1A2
:20E2C000B0EE480ABDEC028BD4F88C193848BDE8F04144F0D5BB301D44F0D2FB94F89079AA
:20E2E0000FE7C6F8048002E7D4F8482A94F82A3A92F8832013437FF410AF94E70023A4F8E0
:20E300002C3A002F7FF468AF94F8403A84F84D5A84F84C3A60E720EE000ADFED207A20EEE0
:20E32000270A98E7234A1346F3EC017A78EEA76A87EEA67A83ED017AD2ED007A78EEA76A66
:20E3400087EEA67A83ED037A77EEA88A87EEA87A83ED057A40E794F8403A84F84D5A84F852
:20E360004C3A00283FF438AF0646E2E6114AD2ED007A131DE8E70F4A131DDDE70D4AD2EDCB
:20E38000007A131D20E70B4AD2ED007A131D13E7B05F0020BD37863500409C45CDCC4C3CF4
:20E3A0004069002083F9223E006A0020246A0020486A00206C6A0020F8B5214C1D270E4606
:20E3C000054684F8D87A1DF08FF800201DF02EF808201DF02BF80E201DF028F838461DF0FF
:20E3E00025F804201DF022F804201DF01FF800201DF01CF830201DF019F800201DF016F883
:20E4000030461DF013F800201DF010F81DF058F804F6D9201CF05EFF234670B194F8D92A67
:20E4200062B994F8DA2A302A00D03AB993F8DB2A22B993F8DC3A2B700120F8BD0120FCE793
:20E44000B05F0020104B034410B5044693F8100410F0D2FE0D4800EB44040A23B4F9EC1A05
:20E46000B1F5FA6FA8BF4FF4FA61B1F57A7FB8BF4FF47A71A1F57A71BDE81040B1FBF3F13E
:20E480000920C9B210F0E6BE78920608B05F00201D4991F81428A2B3F0B4002605463346DF
:20E4A000304637461BB991F814482D2C23D02E2A19D0CA1800EB800092F81448A4F1300229
:20E4C000092A4FEA40009CBFA0F13002A0180E2B14D80133CA1892F81428002AE2D106B125
:20E4E0004042F0BC70470133002DF8D0CA182A4482F81478DDE701231E46EBE70020F0BCCE
:20E5000070470020704700BFB05F00201FB503AC8DF80C30009400238DF80D300FF0B6F914
:20E5200004B010BDF8B50546262025F0C5FE134C0146F8B9D4F8100B90F838301E3B012B91
:20E5400001D93BF0CDFB0E4F0026AE420ADBB4F8343B0133A4F8343B0A4BD3F80039C4F827
:20E56000443BF8BD17F8011BD4F8100B3BF0B8FB0136EAE7002384F8423BEDE7B05F002050
:20E58000C46A0020D01B002010B58021044604F077FE2046002104F073FE2046BDE81040C2
:20E5A00005F0AEB92DE9F041B14C94F85B3BC4F8480B82B088465A2B00F2B980DFE813F010
:20E5C000CC00B700B700DC00B700B700B700B700B700B700B700B700B700B700B700B70091
:20E5E000B700B7000F01B700B700B700B700B700B700B70033017400B700B7007400B7005B
:20E60000B700B700B700B801B7006201B700B7007C00B7000902B700B700B700B7005B001F
:20E62000B700B700B700B700B700B700B700B700B700B700B700B700B700B700B700B7006A
:20E64000B700B700B700B700B700B700B700B700B700B700B700B700B700B700B700B7004A
:20E66000B700B700B700B700B700B700B700B700B700B700E40194F85C3B9B0700F16982EE
:20E68000B4F8623BD4F85D2BD4F89C1B5BBA9BB212BAD0188842C4F8A83BC4F8A42B03D974
:20E6A00004F0AEFD002854DB0020A4F8940B0546284602B0BDE8F08194F8A03B002B40F0C6
:20E6C000FF8094F9583B002B31DAD4F8903B08469B689847002840F01E82B4F8620BD4F8C1
:20E6E0005D2BD4F89C3B40BA80B212BA15189D42C4F8A80BC4F8A42B07D904F081FD002877
:20E7000027DBD4F8A42BD4F8A80BD4F8983BD4F8546B03FB00F003FB02F20225B042C4F8FE
:20E72000A42BC4F8A80B84F8A05B00F0CF8094F86C3B5A1CD2B204EBC30305204FF400514A
:20E74000042A84F86C2B83F8700BC3F8741B00F0A0814FF0FF35ABE7D4F8543B002BE6D1E5
:20E76000D4F8903B08469B6898470546002840F0D281A4F8940B9BE73E4B002203F112016D
:20E7800003F8012F8B42FBD13B4994F8963B94F86C0B70250D7098424FF00C05CD7110D077
:20E7A00004EBC300013390F8705B8D70B0F8740BDBB2042B40BA888114BF84F8963B84F8A1
:20E7C000962B94F85F3B12229342A4F8942B98BFA4F8943B0025284602B0BDE8F08194F845
:20E7E0005C3BDA0700F13E81D4F8903B94F85F0BDA6901EBC10102EB81010A79531D83424C
:20E8000028BF0346A4F8943B002BE3D0013B1A489BB201331944034411F8012D03F8012D5C
:20E820008342F9D1D6E7154E154F35460823073EC5F10700A4F8943B002202E092F83024D0
:20E840001D462B46B54203F8012900EB030217FA82F2F3D1D4F8903B4046DB689847002828
:20E86000B8D0AB7863F07F03AB70002520E700BFB05F0020278E0020288E00202F8E00205B
:20E8800078920608D4F8903BC74A5B680846111D98470546002840F03E81D4F89C3BC34A88
:20E8A000D4F8981B013B180E1070180C09BAD37050701B0A082093705160A4F8940BF7E6F4
:20E8C000D4F8A86BD4F8A42BD4F8983BD4F8905BB2FBF3F24FF48057BE4228BF3E462D69BB
:20E8E000B249A4F8947B4046B6FBF3F39BB2A8470028C0F2BC803346AC4AD4F8480B8121D3
:20E9000004F0F2FCD4F8A42BD4F8A80BD4F8B43B3244851B9E1BC4F8A42BC4F8A85BC4F86B
:20E92000B46B002D7FF456AF032384F8A03BBFE69E4E0027334606F10C0203F8017B9A420D
:20E94000FBD1D4F8903B40465B686A4601A998470546002840F0E980019BBDF80020013B19
:20E96000190E52BAF3713171190C1B0A71710820B371022172810C23BDF80220F0703172C7
:20E980007272A4F8943B93E6894E8A4F30460823073EC0F10705A4F8943B002202E092F863
:20E9A000382418460346864203F8012905EB030217FA82F2F3D1D4F8903B4046DB689847EA
:20E9C00000283FF407AFF37863F07F03F37000256EE694F8A03B002B61D194F9583B002BFB
:20E9E000FFF6A5AED4F8903B08469B689847002840F09180D4F8903B4046DB689847054615
:20EA0000002840F0BA80B4F8623BD4F85D2BD4F89C1B5BBA9BB212BAD0188842C4F8A83BC5
:20EA2000C4F8A42B00F29F80D4F8981BD4F8540B03FB01F302FB01F28342C4F8A42BC4F8A2
:20EA4000A83B7FF474AEB3F5805F28BF4FF480530121D4F8480B554A84F8A01B9BB204F062
:20EA60006DFD25E607235449A4F8943BCEE694F86C3B5A1CD2B204EBC30304204FF4885119
:20EA8000824284F86C2B83F8700BC3F8741B7FF460AE002384F86C3B4FF0FF3508E6D4F86B
:20EAA000A86BD4F8900BD4F8983BD4F8A42B4569B2FBF3F2B6F5805F28BF4FF4805608468A
:20EAC000B6FBF3F339499BB2A847002862DBD4F8A42BD4F8A85BD4F8B43B3244AD1B9B1B63
:20EAE000C4F8A42BC4F8A85BC4F8B43B2DB9D4F8480B294604F076FDDAE5B5F5805F28BF17
:20EB00004FF48055ABB2D4F8480B284A012104F015FD0025CCE594F86C3B5A1CD2B204EBD5
:20EB2000C30302204FF468510AE694F86C3B04EBC3020133DBB202204FF46851042B82F892
:20EB4000700BC2F8741B22D084F86C3B4FF0FF35AEE594F86C3B5A1CD2B204EBC3030520CF
:20EB60004FF41051ECE504F04BFB0028FFF6F1ADD4F8A42BD4F8A83B56E794F86C3B5A1CFB
:20EB8000D2B204EBC30302204FF41C51D8E584F86C7BDEE594F86C3B5A1CD2B204EBC303A5
:20EBA00004204FF440716BE7486B0020288E00202F8E002078920608A096060810B51C2008
:20EBC0003DF0B2FD1121044639F05CFF20463EF09BF8C8203AF0A4FC2046BDE810403EF0F7
:20EBE00099B800BF08B500203DF09EFD054BC3F8BC0B08B12A23C380BDE80840402139F0CE
:20EC000041BF00BFB05F00202DE9F04FB34CD4F8A43A5A69D2078BB002D50BB0BDE8F08F7B
:20EC20005A699B6912EA030AF7D0CAF307431AF4002F009340F00281009B5D0743D41AF093
:20EC4000020F5FFA8AF503D0D4F8A43A02225A61BAF1000FC0F211821AF4006FCAF3072708
:20EC600040F084812E0708D59D4B9E48D3F8B0329847D4F8A43A08225A61ED0600F1E98116
:20EC8000F80600F1A981B90600F12E81009BDA0609D5934B9348D3F8C0329847D4F8A43AA4
:20ECA0004FF480125A61009B9B06B6D58C4B8D48D3F8C4329847D4F8A43A4FF400125A61F7
:20ECC0000BB0BDE8F08FD4F8A82A9369D26913401FFA83FBBBF1000FB1D0DFF80882CDF834
:20ECE0000CA045464FF0000909E05FEA5B0B09F1010908F1040805F1280500F0DA811BF07B
:20ED0000010FF2D0D4F8A81A5FFA89F708694A6B04EB8703FA40D3F8B03AD2019B68D2B2D2
:20ED200002431A40D007D3B216D54B6BD8F81820012000FA09F023EA00034B63684B6948F9
:20ED4000D3F8A832012191603946984794F89B6A012E00F0FE8101231A0703D5D8F8182049
:20ED600008239360DE0603D5D8F8182010239360580603D5D8F8182040239360990703D57F
:20ED8000D8F81820022393601A06AED5D5E94C60D5F82431D8F818C0311A8B42DCF8182058
:20EDA00028BF0B46033392B2B2EB930F9DD9D4F8A82A323704EB8703CDE901989046994668
:20EDC000B04238D2BEB3D5F8241194F89B3AD5F82821371AB94228BF394601F1030E4FEA5F
:20EDE0009E0E83B98FB20337BF10D9F8A0AA0AD0013352F8040BCAF800009F42F8D1D5E935
:20EE00004C60D5F82821DCF8183008440A44B042C5F82821C5F834010AD195F81C11D8F82B
:20EE20003420012707FA01F122EA0102C8F834209BB29E45C4D3DDE9019856E7D4F8A83A2F
:20EE40009D69DB691D402D0C3FF4F6AE04F69826DFF88CB0B046B146002708E06D0807F1C7
:20EE6000010706F1040608F128083FF4E5AEEB07F4D5F9B204EB8102D4F8A83AD2F8EC2A34
:20EE800092685B691A40D007D3B218D594F89B0A726D01239842936007D11269D8F87C333E
:20EEA000C2F312029B1AC8F88C33DBF8A4324846984794F89B3A012B00F0598101239A0723
:20EEC00002D5726D022393601B07C7D5DBF8AC3248469847736D08229A60BFE7B84E0020B8
:20EEE0009801002050590020D4F8A83AD4F8B01A9A680868C2F34102022A08BF03224FF08B
:20EF0000000514BF65F30A0062F30A0008605A6842F480725A6006A805F0C0FBD4F8A42A54
:20EF2000D4F8A80AD368C049079D6FF38D23D3608068C0F34100014491F84014032900F00C
:20EF4000D180BA49BA480126294484F89A6A81424FF04006A4F89C6A00F217810E2161F350
:20EF60008D234FF40051D36051618FE6B14B94F8AA2BD3F8B832B04800218DF817108DF897
:20EF800017209847D4F8A81AD4F8A42A94F8A23A88684FF400615161002B3FF463AEC3074C
:20EFA0007FF560AE94F8AD3B012B7FF45BAE9DF81730032B7FF456AED4F8A43B9F491A681D
:20EFC00042F001021A601A6842F003021A600B6943F006030B6145E6D4F8A82A96485368D1
:20EFE0004FF0000823F001034146536004F0B4FF94F8996A414656B1914BFF2203EB86063E
:20F0000053F8045FD86BAA609E428260F8D1D4F8A83A89484FF0FF329A614FF00112DA61F3
:20F020000B2262F3070162F30708C3F8148019611A686FF30A121A6004F062FCD4F8A42AB3
:20F040007C4B7D48D3F8B4324FF480515161984719E6D4F8A43A9A6922F010029A611A6A7F
:20F06000C2F34340022802F00F0146D0062823D09A6942F010029A6102E694F8A23A3BB177
:20F08000D4F8A42B136823F0030161F307031360D4F8A82A67495368D1F8BC12664823F011
:20F0A000010353608847D4F8A43A4FF000425A61D2E5DDF80CA0C2E5D4F8685B41F26400DF
:20F0C00001EB81012E68265004EBC1012E68D1F8240E41F26805C2F30A1202446651C1F84D
:20F0E000242EC5E700214FF4007084F89A1A0921A4F89C0A61F38D2333E747F6F070104295
:20F10000B6D001EB8100C2F30A1204EBC00002F1030C5FEAAC0CD0F8185ED4F868EB4FEAE3
:20F12000810818BF002006D00130DEF8006045F8046B8445F8D1414404EBC101D1F8185E5F
:20F14000D1F8240E15440244C1F8185EC1F8242E8EE7B9F1000F7FF4FEAD94F8A93B042BF0
:20F160007FF4F9AD344804F0CBFB3346F4E5002F7FF4A4AE94F8A92B052A7FF49FAE48461D
:20F18000019304F0BDFB019B99E62E48A5F57401A1F51051814203D80D2161F38D23E0E602
:20F1A00029492A482944814203D20C2161F38D23D7E62748A5F18C71A1F54341814203D8BE
:20F1C0000B2161F38D23CCE6224923482944814203D20A2161F38D23C3E62049204829445C
:20F1E000814203D2092161F38D23BAE61D48A5F1B771A1F55851814203D2082161F38D2382
:20F20000AFE6194919482944814203D2072161F38D23A6E6164917482944814234BF0621D1
:20F22000052161F38D239CE678920608401E1BFF3F420F00980100205059002000ED00E0B3
:20F2400064590020DFC810002013FBFE20D61300FF69180000D3CEFE40771B00C05BB3FE28
:20F26000C091210040AC2700C01D6AFE40E13300803C36FEE09C4100704700BF704700BFD7
:20F28000704700BF704700BF2DE9F0414FF0FF35324A33482C46002304E001330B2B02F1FB
:20F2A000100215D0917A0429F7D103F5B17100EB0111C979CF07F0D4661C116801D0A942AD
:20F2C000EBD21C4601330B2B0D4602F11002E9D1631C02D10120BDE8F081214D04F5B1777B
:20F2E00005EB07139988F1B9DFF880802601AB1958F8642C1B4916691B4A41F2186001EBB8
:20F30000442118580023B047D0B1022808D141F2CC6205EB0717AB58013B0121AB50B97185
:20F320000020BDE8F081DFF8448005EB041358F8642C41F21860D268185826019047D6E705
:20F3400041F2CC6205EB0717AB580321B97141F2D061013B0124AB506C54BCE744B40020B2
:20F36000289E0020409E002089F30008B05F0020044B41F2E472995C09B901219954012235
:20F380005A707047289E002038B5174D174B41F2D0640020285504E001300B2803F1100300
:20F3A00014D053F80E4C8C42F6D11C78032CF3D16AB10F4B03EB40239A4201D0FFF7D8FF68
:20F3C00000F5B17005EB00100123837138BD41F2CC6100F5B1736A5805EB03130420013272
:20F3E00098716A5038BD00BF289E00204EB40020409E002038B5134B00209C7B14B11D68C4
:20F400008D4205D001300B2803F11003F5D138BD72B10D4B03EB40239A4210D0FFF7A8FFFD
:20F420000A4B00F5B17003EB00100123837138BD064B00F5B17003EB0010827138BD022CDB
:20F44000ECD1EDE740B40020409E0020289E00202DE9F84F12F0020E9B4606D028B9FFF726
:20F4600087FF02252846BDE8F88F804C41F638056559002D5BD14FF0FF367D4FB146B046C1
:20F48000B24600253B68984200F0B68097F80EC0BCF1000F5BD0BCF1010F15D105F5B17C9E
:20F4A00004EB0C1C9CF807C01CF0010F0CD11CF07E0F09D15FEADC1340F0A880D7F808C047
:20F4C000D44501D2E246A94601350B2D07F11007D8D1751C04D1B8F1FF3F00F09F8046461B
:20F4E00041F2C86806F5B17754F80850013544F8085004EB061C41F21C694FEA07184CF8B3
:20F50000095044F8085041F2186904EB07154FF000084CF80900C5F8048004EB0715AD7939
:20F52000042D9CD8DFE805F01A330F334D0004F5C25741F63C063F68A65907FB0565A84207
:20F5400099D3FFF715FF00252846BDE8F88F2E4601350B2D07F1100794D1BAE712F0010C70
:20F5600070D104EB0710D51090F80780BBF1030F65F3C71880F8078062D94FF6FF708345A5
:20F580005B4628BF03469BB204EB07108380BEF1000F16D004EB061303F5B0531833987B3F
:20F5A00004280ED041F2C8654FF0040C60590130605141F2CC65586083F80EC063590133A2
:20F5C0006351500705D504EB0710C37943F00103C371D30608D504EB0714E379C3F3450280
:20F5E000013262F34603E371224B012503EB46260E602846BDE8F88F05F5B17704EB0716C3
:20F600004FEA071CB67986B92E4669E7A84601350B2D07F110077FF435AF5AE7B9F1FF3F71
:20F6200018BF4E467FF45CAF8DE741F2C8682E4654F80850013544F8085044F80C506CE73D
:20F640006346A1E70C4B0B4953F8643C0B4AD3F8088001EB46210023C04700283FF473AF41
:20F6600004EB07140223A371FCE600BF289E002040B40020409E0020B05F0020F5F300088F
:20F68000F0B5124D2B7841F63002022B0BBF070AC0F3D417C4B200F07F04A85883B00E4644
:20F6A00000230122384401A9FFF7D2FE01280AD12B78022B019B16BF53F8243033F81430C5
:20F6C00023F07043336003B0F0BD00BF289E002010B5144602070B4610D50B4941F2C472B1
:20F6E000581C8B58834204D305D100232360012010BDFFF73DFE2060012010BD2146184649
:20F70000BDE81040BCE700BF289E00202DE9F0414268C2F308030B44B3F5007F82B0044609
:20F720000D4657D390F91A30591C0AD0304A03F5B17302EB0313FF21DA796FF30002DA716F
:20F74000817694F91B305A1C0FD0294A03F5B17302EB0313FF20DA79C2F34501013921EA41
:20F76000E17161F34602DA71E0762378022B37D01F4A02F5C2531B68B5EB432F4FEA43287D
:20F7800024DC41F648036768D6583E407342AB421CDCAB19434511D32169207E01AAFFF7D9
:20F7A00097FF012812D16768236963614744019B2361A5EB0801BF1B67608D192046F8F7A8
:20F7C0000BFE20B93D446560012000E0002002B0BDE8F08115444560012002B0BDE8F08131
:20F7E000616801202944616002B0BDE8F08100BF289E002070B5154604460E46FFF786FFEB
:20F8000050B994F8280028B9022384F82830C4E90B5670BD022070BD1DB12046A847012083
:20F8200070BD012070BD00BF10B4D0E9011390F91A208B4238BF0B46511C83600AD0144B9C
:20F8400002F5B17203EB0212FF21D3796FF30003D371817690F91B305A1C0FD00C4A03F509
:20F86000B17302EB0313FF24DA79C2F34501013921EAE17161F34602DA71C4760022436A69
:20F880005DF8044B4261426011460361B2E700BF289E002038B544220021114859F09BFCD9
:20F8A000104B41F602011A784FF6FF745C52022A41F2E87118BF032203F5C05041F64C0577
:20F8C0005A5441F60C0441F6010203215D5900F8181910211D519954FFF7A6FF012038BDB9
:20F8E00010B60020289E00202DE9F041B1F904300F2B82B00C461646054632D02846F8F753
:20F900008FFD95F91B80B8F1FF3F074633D02D4B41F2186203EB08118A58904211D11833EE
:20F9200003EB4823A188013109B203EB4113A18028463360F8F774FD2060012002B0BDE89C
:20F94000F081FFF715FD2846F8F746FD28B100230120336002B0BDE8F081002002B0BDE89F
:20F96000F0814FF40071FFF7D1FE0028F5D04FF6FF73A380C2E72846F8F72EFD0028E2D1CA
:20F980000FB9FFF7F5FC38460023112201A9FFF75FFD0128D7D1019B0B4A9A1A48BF02F277
:20F9A000FF12B2F5B05F4FEA622106D24FFA81F885F81B80002BB5D1C5E7FFF7D9FC019B4E
:20F9C000F6E700BF289E0020409E002030B50446C06983B010B9012003B030BD0D4600231C
:20F9E000032201A9FFF734FD0128F5D1B4F92030002B03DAFFF7BCFC0220EDE7019A012DB0
:20FA00004FEA431102EB431303D0022D12D1E5255554A268DA612278032A04D100221A77EA
:20FA20005A779A77DA77626A5A83C2F30F429A8203B030BDE268DA61EDE700BF10B50378D0
:20FA4000023B012B0446037E02D913F0060F5AD198063AD494F91A30591C0AD02D4A03F513
:20FA6000B17302EB0313FF21DA796FF30002DA71A17694F91B305A1C0FD0264A03F5B1736D
:20FA800002EB0313FF20DA79C2F34501013921EAE17161F34602DA71E076237E1B070BD57F
:20FAA0001C4841F2C873C35C072B01D0FFF760FC41F2C8730022C254E26A0023237084F8DC
:20FAC0002830FAB1BDE81040104700231249E0691A018A58904206D001330B2BBAD01A015C
:20FAE0008A589042F8D10B4A03F5B17302EB0313DA79C2F34501013921EAE17161F3460294
:20FB0000DA71A7E710BD0121FFF760FF0128F9D1237E9DE7289E002040B4002030B102785B
:20FB200022B190F828201AB1002070470120704710B5D0E90142A242C16238BF224603215D
:20FB4000826080F82810FFF779FF012010BD00BF2DE9F04FDFF868918A4699F80010DAF890
:20FB600000300229174683B0834641F6300240F08B8059F80250DEB2A6EB030805EB132536
:20FB8000B8444FF480729044BB4208F1FF38B8FBF2F875D2A844032906EB0704A4EB0304A5
:20FBA0000CBF80224FF48072944228BF1446A8EB050366B994422CBF0A220B2201A92846A0
:20FBC000FFF746FC012809D003B0BDE8F08F0B2201A92846FFF73CFC0128F5D199F8002001
:20FBE000DAF80010022A01F1010321D0A64210D2019906F18042013A081F00EB840001EB36
:20FC0000820242F8043F824203F10103F9D1DAF80010A61B7318BBF1010FCAF800301BD096
:20FC20009F4205F101052BD999F800100026B2E7A642EED2DDF804C006F10042013AACF131
:20FC4000020000EB44000CEB420222F8023F904203F10103F9D1DCE7BB42E1D199F8003016
:20FC6000022B21D004F18044019B013C4FF0FF3243F82420DAF800309F4205F10105D3D85B
:20FC8000012003B0BDE8F08F59F8022003F07F060329C3F3D415A6EB03081544B84414BFF2
:20FCA0004FF4807280226EE704F10044019B013C4FF6FF72584623F8142003B0BDE8F08F8C
:20FCC000289E00202DE9F04190F838300446032B51D8DFE803F002323B462D4BC0681978C6
:20FCE000E76A03F5C252032911680CBF80264FF4807601FB06F141F2C47C00EB412041F273
:20FD0000A87841F2AC7E53F80C20E06053F80E0053F808502261A5EB4125A0EB41219019A4
:20FD200043F8085043F80E1043F80C00C4E90C205FBB6262012384F8383016480021FFF75C
:20FD400045FE012811D1022384F83830626B04F130010120FFF7FCFE012806D1032384F8A6
:20FD6000383000212046FFF731FE431EDBB2012B02D9BDE8F081022094F82830062B04BF6A
:20FD8000002384F82830BDE8F081921B2263D1E7289E0020C8B500202DE9F04FDFF8248118
:20FDA00098F80060012887B08CBF00230123032E02930C460B68154639D0022E62D14FF4CC
:20FDC00080724FEA1329DFB201920138012823D8012203929D421AD9384E06F1880A06F1AB
:20FDE0001C0B32681AB1DBF8001099424ED0DAF8000000234844092205A9FFF729FB0128FE
:20FE00001FD002280FD020B123689D42E9D82560032007B0BDE8F08F87B1FFF7A9FA022078
:20FE200007B0BDE8F08F022007B0BDE8F08F80220192C3F3D41903F07F07C6E7019A0392BC
:20FE4000C8E7DDE902C1059ADDF804E098F80030022B14D0032BE6D152F8273023F07043F5
:20FE6000B3FA83F35B0963450F44236823D00B4477452360EAD309F101090027C5E732F836
:20FE80001730EDE74FF480720192D2E70C490968013A02EB41224902B2FBF1F203991344A7
:20FEA000B3FBF1F201FB12320AB10B449B1A9D42236096D8ABE7AB42ABD3A8E7D0B50020B1
:20FEC00068B60020289E0020F0B5104D2B7841F63002022B0BBF070AC0F3D417C4B200F0E4
:20FEE0007F04A85883B00E4600230322384401A9FFF7AEFA012807D12B78022B019B0CBFB4
:20FF000023F8146043F8246003B0F0BD289E00202DE9F04390F83C30002983B0044614BF97
:20FF200002210021042B7BD8DFE803F0030C3C476900FFF74BFD012870D1626B002A75D161
:20FF400084F83C00404EDFF80881404D4FF6F7771DE01FFA80F9B94594BF4FF000094FF054
:20FF6000010901A9B9F1000F46D1FFF789FB0128494650D1206BFFF7A7FF01284BD1019BA2
:20FF80002A682363013B934228BF13462B603378206B032BDDD1404594BF4FF000094FF0FC
:20FFA0000109DEE7426B04F130010020FFF7D0FD012833D1032384F83C30234BE16A41F295
:20FFC000C47003F5C2521D581268195041F2A87741F2AC76D8596D1A995902FB05F200EB59
:20FFE000422501EB422203F5BD500021DD519A51FFF7ECFC012811D1042384F83C3094F887
:020000040801F1
:200000002830042B04BF002384F82830A36B8BB120469847012003B0BDE8F0830228FAD12F
:2000200094F82830042B09D00220F4E7022384F83C30B8E7012003B0BDE8F083002384F8A0
:2000400028300220E7E700BF289E00206CB60020F7FFFF0F38B590F834300446052B46D8FC
:20006000DFE803F01F033F101963006B4FF0FF31FFF72AFF01283AD1E06A002839D103230A
:2000800084F8343000212046FFF7A0FC01282ED1042384F8343094F82830082B2DD0012003
:2000A00038BD41F63803224DEA5800F1300102320120FFF771FE012824D00238C0B201285A
:2000C00015D8052384F8343094F82830082B04BF002384F8283041F2E5730122EA5402204C
:2000E00038BDC06A216BFFF7EFFE0128C7D0002038BD022384F83430F4E7002384F82830C6
:20010000012038BD05F5C252E3681168D4E90B2003EB412341F644016850C4E9033002B9EE
:200120006062012384F83430A0E7014DCCE700BF289E00202DE9F04F436883B0C3F30808D3
:200140001646002A00F0E180714B05468946A3F1180B4FF0000AC8F5007495F91A70B442B3
:2001600028BF3446791C28462ED0F8F759F90BEB071341F218629B58984205D0FFF7F8F897
:20018000504603B0BDE8F08F614B03EB472022464946404458F0BEFF002221462846FFF784
:2001A00029FBA2440028EBD02B7E1B0706D5594B2A691B689A4201D3FFF7DAF8361BA14444
:2001C0004FF00008C7D1DBE7F8F706F9002849D12846F8F725F96968C1F308032BBB21F448
:2001E000FF7323F0010303F50072AB689A422CBF062207222B7E03F00C030C2B1CD00023F0
:2002000001A9FFF725F90128BAD10198404BC31A48BF03F2FF13B3F5B05F4FEA63224FD2C7
:2002200057B2AF760028B2D1AAE72B7E03F00C030C2B4FF00702E2D19BF800C0364BBCF1F6
:20024000030F1B680CBF4FF0800C4FF4807C03FB0CF34FEA432C0CF1FF3C0CEA0101A3EBD1
:200260005123CDE72B7E1A072ED59BF800102A4B95F828201B6803290CBF80214FF480714D
:2002800003FB01F3062A4FEA43233FF479AF23490868834230D891F83D30002B7FF470AFE6
:2002A000002A7FF46DAF6B6985F83820062185F82810EB622846FFF705FD012888D05FE786
:2002C000FFF756F80198ACE7154B1A78002A7FF457AF95F82820002A7FF452AF082185F800
:2002E000342085F82810D3F85F206B692846C5E90B32FFF7AFFEE0E741F2E57301225046D0
:200300000BF8032003B0BDE8F08F924638E700BF409E0020ECB5002068B60020D0B5002088
:200320000DB600202DE9F04390F8384083B00546032C00F2A180DFE804F0021A8B0BFFF76E
:2003400089FE012811D002280BD1032385F838302B6C002085F82800002B00F0898098479C
:200360000224204603B0BDE8F08385F838002B78022B79D0414A6F6841F64803D3581F40EA
:20038000C7F34F272846F8F74BF8DFF8F48006463F1A0AE0D8F800305A1E91454AD2FFF753
:2003A000B5F908B9FEF7E4FF0136022201A900233046FFF74DF8BC1901281FFA84F94FF446
:2003C00000724FF000010446CBD1019858F003FFEB694FF400712846002BDBD06B68002B58
:2003E000D8D1019B4FF020324FF02E0C1A605A6083F800C0C3F807204FF0100E6C6A1A62AE
:200400005A6283F820C083F821C0C3F8272083F80BE0EA6B5C83C2F30F4CC4F30F4483F838
:200420002BE05A879C82A3F834C0D8F800305A1E9145B4D3C3EBC353590201F5007128465A
:20044000FFF764F908B9FEF793FF022385F838302B6C002285F8282063B1284698470124F3
:20046000204603B0BDE8F0836F68C7F34F2789E7022476E7012474E7002472E7289E00206E
:2004800068B600202DE9F04F90F8303089B00446042B00F2A880DFE813F0A900B2000500EB
:2004A0008A00E800C64D41F61003EB5C002B40F09A80C44F04F11C09B84607F1380BBA464B
:2004C00001AE324649464046FFF70EFA012840F03F810198002800F021810378E52B01D01A
:2004E000002BEED1B84A821A48BF02F2FF12B2F5B05F4FEA622380F06F811B01B34A134424
:200500009A7B042A0CD041F2C86104266A5801326A5041F2CC615A609E736B5801336B50AA
:2005200041F60202AB565E1C09D003F5B17305EB0313FF26D979AE546FF30001D97141F6AD
:2005400003016B565A1C0ED003F5B17305EB0313FF26DA796E54C2F34501013921EAE17194
:2005600061F34602DA712022002158F034FE2346019A53F8311F58685060116019899B7A80
:2005800093721181019B627EDA7205A846F0BAFCBDF81430002B40F0578144F28172019974
:2005A00003200A82CB810A83CB8284F83000237E980600F1D0802046FFF736F92369002BF8
:2005C00000F0D580237E03F0F70213F00403227640F0DB80122A00F0E180002384F8283098
:2005E0002046E36A984709B0BDE8F08F7548FFF71BF94FF6FF720123228484F83030714FA9
:2006000004F11C0501AE04F13109324629463846FFF76AF901282FD00228E4D1684D41F635
:200620000202AB56591C09D003F5B17305EB0313FF20D979A8546FF30001D97141F60301F0
:200640006B565F1C0ED003F5B17305EB0313FF20DA796854C2F34501013921EAE17161F34A
:200660004602DA71042384F830300020E36A2070984709B0BDE8F08FDDF804800B22494616
:200680004046B8F1000F00F0AD8098F80030002B00F0A88058F0CBFD0028B6D1B8F8141069
:2006A000B8F81A304A4A43EA014312686362D8F81C30A3605202B3FBF2F102FB113109B1FF
:2006C00013445B1AE36098F80B303D4D637641F60202AB565E1C09D003F5B17305EB03132C
:2006E000FF20D979A8546FF30001D97141F603016B56581C0ED003F5B17305EB0313FF2051
:20070000DA796854C2F34501013921EAE17161F34602DA71032384F8303048E73B782D49F7
:20072000022B4FF0090250469CD00B78002B99D1C1E905330A708BF800304A6B0B7351F89D
:20074000143CC1E90132FFF7EDFD01283FF4B9AE022887D047E7E0690023112205A9FEF7D8
:2007600077FE01283FF427AF09B0BDE8F08F237E19077FF532AF124A41F2C873D15C0029BF
:200780007FF431AF0721D15427E70023E26AA16884F828302046FFF72DF824E7626AE06ABD
:2007A000A0630421C4E90233C4E90B2284F83C30636384F8281063622046FFF735F812E7AC
:2007C000289E002010B60020409E002040B4002068B6002038B60020FEF7CAFD01986FF03B
:2007E0000F038BE6294D41F60202AB56591C09D003F5B17305EB0313FF20D979A8546FF385
:200800000001D97141F603016B565A1C0ED003F5B17305EB0313FF20DA796854C2F34501F2
:20082000013921EAE17161F34602DA71237EDF067FF518AF1648FEF7F7FF4FF6FF72022355
:20084000228484F830302EE6124B05A9B3F9C02B02A846F0ABFB9DF80C309DF80D609DF872
:200860000A509DF80B20BDF808109DF80E00DB0243EA461342EA4512A1F2BC7143EA5003C8
:2008800042EA41229BB292B289E600BF289E002010B60020B05F00202DE9F04390F82830E6
:2008A000013B83B00446082B41D8DFE803F048054D525865406A4300384B4668056B41F60B
:2008C000480103F5C2525F5813683740EA19B2EB432F4FEA432816D258E02169207EFEF727
:2008E000F7FE012823D1256B666823696361A5EB08053D444644F61B019B6660A8452563A8
:200900004F46236142D82046F7F766FD01AA81460028E2D06668A368E26A9E4238BF1E4641
:200920000023A66084F828300AB12046904703B0BDE8F083FFF7F6FC03B0BDE8F083FFF74E
:20094000A1FD03B0BDE8F083FFF778F803B0BDE8F0830021FFF7DCFA03B0BDE8F083012123
:20096000FFF7D6FA0128E2D10023216C84F828302046FFF7D3F8DAE7FFF7A4F903B0BDE87E
:20098000F083FFF767FB03B0BDE8F0832046F7F723FD0028BFD12E446660BCE7289E0020D4
:2009A00010B5114C94F8A23A23B9104B4FF480225A6110BD0E4A136823F00603136054F063
:2009C00055FE94F8A23A002BEFD0D4F8A83A9B68DB07EAD5D4F8A42B136823F0030161F39F
:2009E00007031360E1E700BFB84E0020003C014010ED00E02DE9F04704460D469046002192
:200A000044221E46089F58F0E6FB01234FF6FF722676628384F828302B782E2B4CD02E4681
:200A200004F1310A307804F1390968B12E280BD042F03EFEC0B20AF8010BCA4506F1010662
:200A400007D030780028F1D120200AF8010BCA45F7D130782E2808BF707804F1380908BF5E
:200A6000013604F13B0A58B142F022FEC0B209F8010FD14506F1010607D030780028F3D1A8
:200A8000202009F8010FD145F7D118F0100F14BF0323012384F819802370E7622B782E2BF6
:200AA00026D16B7823BB0323204684F83030FFF7E9FC2046BDE8F0876B78002BAFD1114BCF
:200AC00041F2F47241F60C0041F2F0719A5818585958E26041F601026062A1609A5C627686
:200AE00041F2E8729B5C2370E7622B782E2BD8D00023204684F83030FFF7C4FC2046BDE8CC
:200B0000F08700BF289E002008B50121032003F02FFB72B64BF034F82DE9F04FCD4CDFF8C6
:200B200040938DB000270090651C04F6CD3A54F80B0C002800F0FE8039F0CEF80646002810
:200B400000F0D281D9F8003944F8073CE0260023A4F10B0B04F8033C7E4354F80B0C39F06D
:200B6000BBF8002800F0E68054F80B0C39F0ACF814F8023C5A1E80460B2A0DD8DFE812F0A9
:200B80001F003A004600530083009B00E3001601350140017201890124280CD0009A3AB922
:200BA00095F88A29824240F07A81012204F8032C0D2BD2D186E0012304F8023CCDE7002342
:200BC0004D28C4F8C53084F8CD3084F8CE3004D0582808D004F8023CBFE7022204F8022CA2
:200BE00084F8C430B9E7032304F8023C022384F8C430B2E704233C2804F8023C0BD0B8F10E
:200C00003E0F0CD0002304F8023CA6E70A233C2804F8023CF3D1002304F8013C9DE701232E
:200C200004F8013C99E7D4F8C500AB190344421CC4F8C52003F8018C94F8CD00022A88EAE1
:200C4000000184F8CD1088D12378C02BDAD86278FF2A08D1052BD5D9012384F8C430072331
:200C600004F8023C79E7A4F8C12000229342C4F8C93014BF0523062384F8C320C4F8C5208D
:200C800004F8023C69E7D4F8C500AB190344421CC4F8C52003F8018C94F8CD00D4F8C93089
:200CA00088EA00019A4284F8CD107FF456AF062304F8023C51E794F8CD308342A2D10D2388
:200CC00004F8023C14F801CCBCF1000F40F0ED80614B08940FCB04AE86E80F00D4F8C93092
:200CE000D4F8D100ADF82CC023440993B4F8C130ADF8283094F8C3308DF82A3001238DF822
:200D00002E30324603AB08A9CDF80CC032F052F848B1049B059394F8C420504B0493314658
:200D200058462FF081FD039E002304F8023C002E40F0D2800137032F04F1E0047FF4F7AE6F
:200D40000DB0BDE8F08FD4F8C500AA190244431CC4F8C53002F8018C94F8CD2094F8CE00AE
:200D6000019388EA0202414684F8CD2046F0B4FB019B84F8CE00072B7FF4EFAEB4F805308B
:200D8000C02B3FF63FAFB4F80320A4F8C120A27884F8C32000229342C4F8C93014BF0823D6
:200DA0000923C4F8C52004F8023CD6E6014694F8CE0046F091FB94F8CD3084F8CE0088EAC8
:200DC0000303D4F8C50084F8CD30AB190344421CC4F8C52003F8018CD4F8C9309A427FF45D
:200DE000BCAE092304F8023CB7E694F8CD30434084F8CD3094F8CE3083427FF403AF56E750
:200E0000D4F8C500AA190244431CC4F8C53002F8018C94F8CE000193414646F05DFB019B02
:200E200084F8CE00052B7FF498AEB4F80120B4F80330A4F8C120227884F8C3200022934266
:200E4000C4F8C93014BF0B230C23C4F8C52004F8023C82E6AF5F0020BC96060880800120BB
:200E6000D01B0020014694F8CE0046F035FB84F8CE00D4F8C500AB190344421CC4F8C5207B
:200E800003F8018CD4F8C9309A427FF466AE0C23A0E694F8CE3083427FF4B4AE0FE7232888
:200EA00004BF022204F8032C82E6BCF1010F4FF0000602D004F8026C3CE7D4F8C9300894F6
:200EC0002344099308A8B4F8C130CDE90A66ADF828302EF0C3FCEDE754F80B0C2FF0D2FE9C
:200EE00054F80B0CB04725E714F8033C002B3FF421AFD9F8002954F8071C521A632A7FF63C
:200F000019AF012B2FD0022B7FF414AF54F80B3CC5F8C43BC5F8C83BC5F8D03B402385F8C4
:200F2000D43B95F8AF3285F8D50B0122003B85F8C22B0E4AC5F8CC2B18BF01230C4885F837
:200F40001C3CC5F824A8C5F818AC3EF097FE4FF4005031F0E7FD07483EF086FE85F81D6CCD
:200F600085F81E6CE6E6FFF7CFFD00BFA9630408E72107081D220708034B93F8240000386B
:200F800018BF0120704700BF301C0020202301480B80704768040020642301480B8070470B
:200FA00088040020432301480B807047EC04002010B5074CD4F8C800FF2807D0054951F843
:200FC000042BF7F741F9FF23C4F8C830002010BD6804002080B60020EAE700BF08B5D0F800
:200FE000E4355B6A9847002008BD00BF08B5D0F8E4351B6A9847002008BD00BFD0F8E43509
:2010000010B504461B689847D4F8E8359B689847002010BD08B5D0F8E435DB6903B1984732
:20102000002008BD08B5042290F81211D0F8E83580F8131180F81221DB689847002008BD0A
:2010400010B5D0F8E83504461B699847032384F81231002010BD00BF0B0630B41CD401EBD7
:20106000810200EBC202002300EB810582F8741382F8753301241A4604FA01F16D6D61F3E4
:201080001F4201696FF3CF332B60CB6923EA0203002030BCCB61704701F07F0101EB81047F
:2010A00000EBC404012200EB8105002384F81C1184F81D2102FA01F11A46AD6961F30F029A
:2010C000DFE700BF10B581210446FFF7C5FF20460121FFF7C1FF024B0020187010BD00BF61
:2010E000506B002010B581210446FFF7B5FF20460121FFF7B1FF82212046FFF7ADFFF7F7F3
:20110000E9F8002010BD00BF38B50D4604468321FFF7A2FF29462046FFF7E4FF002038BDBA
:20112000F0B416460A063AD401EB810500EBC5052824002204FB0104022B85F87413C5F80A
:201140007C6385F8773385F8752304F55D7448D0154600EB8107012202FA01F17F6D61F373
:201160001F45D7F800C01CF4004F11D1E488204946F0805242F4004242EA834204F00F04EE
:201180001C4B42EA845211400CEA0303194339600269D3692B430020F0BCD361704701F0E7
:2011A0007F0101EB810500EBC5052824012204FB0104022B85F81C11C5F8246185F81F312F
:2011C000A5F8221185F81D2104F58E740CD0002500EB8107012202FA01F1BF6961F30F0574
:2011E000BFE722711546B4E700252571F0E700BFFF87CC13007833EC002310B519460446E2
:201200004022FFF78DFF8021204600234022FFF787FFD4F8E835A078012284F812215B684C
:201220009847002010BD00BF70B44B78012B26D00B784A6900EB83035C6D25682369D2B10E
:201240008A684A6102F07F0223F4002323F07F0342F4002213432361C378012B04BF0B69DF
:201260006361C5F3076363F07B0363F31F652560002070BC70478A6802F07F02E4E782693A
:201280004C691568136944B38E68B4428CBF06F07F0404F07F0423F4002323F07F0344F47B
:2012A000002443EA040388BF4E611361C378012B1DD0C5F3076464F07B0464F31F651560D2
:2012C000002BD5D14B69002BD2D002690878516B012383400B435363CAE723F4002323F02C
:2012E0007F0343F400231361C378012BE1D10B780C6900EB8300C5F30763816963F07B0342
:2013000063F31F654C610020156070BC704700BF2DE9F0434B78012B30D00B784C6900EBB4
:2013200083035E6D356837691CB38B681C44013CB4FBF3F4C4F3090203FB02F3C3F31203AA
:201340004B61144643EAC44363F31C073761C378012B04BF0B697361CB78012B44D0C5F395
:20136000076363F07B0363F31F6535600020BDE8F0838A680124C2F31203E3E791F80080D7
:201380004E6900EB880EDEF818C0DCF80050DCF8107076B3D1F80890384A06EB0904013CA8
:2013A000B4FBF9F402EAC444C6F312022243CC7807F060473A43012C174649D0CCF8102075
:2013C000C278012A55D00269516B03FA08F30B435363C5F3076363F07B0363F31F65CCF8CF
:2013E00000500020BDE8F0834B7973B345F00055B5E707F0604747F40027CC78CCF81070CD
:20140000C378012B2FD0012CE3D102699268D20554BF45F0005545F08055C5F3076262F02F
:201420007B0262F31F65CCF80050002B9ED1B0B203308010DEF8D04098D0CA6852F8041B9A
:20144000216001339842F9D190E745F0805586E764F35E77CCF81070C378012BD5D10A6955
:20146000CCF81420D1E70A69CCF81420012CB0D1CBE70B69CCF81430ABE700BF0000F81F0D
:201480000E4BDA68D20310D4DA68D1060FD4DA68D20510D4DA6812F0E00F0AD1DB6813F0AB
:2014A000020F14BF0820092070470120704706207047072070470220704700BF003C024097
:2014C00000207047002070477047704730B1044B93F90C000028D4BF00200120704700BFB6
:2014E00080B6002008B5FFF7F1FF50B1054A537B927B5B0003F00203002A18BF43F001033D
:201500000B6008BD80B6002008B5FFF7DFFF10B1014B1B690B8008BD80B6002070B5FFF762
:20152000D5FF78B1084A958A65B196690023B3421C4607DA02EB44040133A48BAC42DBB2BA
:20154000F5D30B7070BD00BF80B6002008B5FFF7BDFF10B100230B70137008BD0420704715
:2015600028B1034B93F9CC00003818BF012070476804002008B5FFF7F3FF50B1054B93F9F7
:20158000CC20012AC3BF93F8CF30C3F340030B60002008BD6804002008B5FFF7E1FF18B1F7
:2015A000024B93F8CE300B7008BD00BF6804002070B5FFF7D5FF38B10E4C94F8CF30DB072B
:2015C00003D500230B70137070BD0B4D94F9CD3095F82C6093FBF6F301330B7094F9CD402A
:2015E00095F82C1094FBF1F301FB134301331370EAE700BF6804002080B60020032070475A
:2016000070B50A4A92F8303006255E1CB6FBF5F405FB146492F83150AC4205D002EBC3032F
:20162000C3E90D0182F8304070BD00BF80B60020002230B504461046914200DC30BDA35C82
:201640000825584010F0800F4FEA400318BF83F0D503013DD8B2F5D10132EDE710B5D9B1B4
:201660000E4B586E814217DCB2B1DB6A9A4213DC0B4C013A013903FB012184F8DA1004F1DB
:20168000D6000521FFF7D4FF062184F8DB0004F1D600BDE81040B3E710BD00BF80B60020CB
:2016A00068040020024B93F868300B600120704780B60020024BB3F86A300B8001207047A0
:2016C00080B60020024B93F86C300B700120704780B6002000230B70012013707047003866
:2016E00018BF012070470120704770470023038083708380C3800372704700BF074A92F807
:201700006D3092F86E100133DBB2994282F86D3004BF002382F86D30704700BF80B60020A8
:20172000F8B5774C236F83B1764B1B6893F82E305BB1754B94F87420A3FB0013012A4FEA45
:2017400093132FD0022A08D002B1F8BD6F4B9842FBD9012384F87430F8BDA26F64329A4294
:201760003CD894F86D3004EB031393F88C20FF2A06D067490132012083F88C2081F8DC0071
:20178000FFF7BCFF634B1B780122092B84F87420DBD1B4F80E31604A01339BB2A4F80E3153
:2017A0005380F8BD5D4D94F86D105A48A3678C2303FB015300789A70002384F88A3004F171
:2017C00080050A2202230928E56784F88B2084F87430BAD1504B01311980F8BD94F88A2093
:2017E00094F88B309A42B0D104F17F0004F18805002310F8012F082153405A0013F0800F4C
:2018000008BF5B0082F0070214BFD3B2DBB20139F3D18542EDD194F889209A4239D194F81C
:201820006D6094F8875094F88830B4F88300B4F8852094F881C004EB061743EA052394F8FA
:20184000825087F88C1040BA52BA81B292B245EA0C202F4DC7F890101BB294F98010C7F83F
:201860009420032E4FF00102A7F88E00A7F8983087F88D1085F8DC2008D8264A12780C2A08
:2018800029D00D2A02D1244B23F81610FFF736FF5FE794F86D3004EB031393F88C20FF2A96
:2018A00006D01B490132012083F88C2081F8DC00FFF724FF174B1B780122092B84F87420A9
:2018C0007FF443AFB4F80C31134A01339BB2A4F80C319380F8BD1249124A897E0E4803EB39
:2018E000830303EB830349089B0093FBF1F382FB0312DB17C3EBA20320F81630C6E700BFEF
:2019000080B600202C660020D34D62103F4B4C0068040020A9280020AC2800201041002075
:2019200078310020676666660A4B93F88A1093F88B2091420DD010B493F88A20DC6F511C34
:20194000D2B2C0B2C9B283F88A10A0545DF8044B7047704780B60020FD2870B522D0F02851
:2019600004D0EF2822D00224204670BD114D0320052641282E444FF0000405F1010580F09B
:2019800080030DD0042B0BD9FFF7E6FF2044B542C4B2E9D015F8010B412880F08003F1D138
:2019A0000420F3E7044D0B200426E2E7034D0C200626DEE7F49B0608F09B0608FC9B060872
:2019C0000E4BD3F81421B3F91001530707D400EB8000400080B200F5C87080B27047084B76
:2019E000084A9B6B323382FB0312D817C0EBA20080B200F5C87080B2704700BF80B60020FF
:201A0000D8500020676666660C4AD2F82C3130B41C68D2F824515D6019810025611C19604F
:201A20009D812070D2F82C31D2F824111A685A604FF6F67230BC19609A81704780B600205C
:201A40000E4B30B4D3F8D022C3F8D42203F5D87503F5307403F5987003F5E0710132C3E9D2
:201A60004A54C3E96C0030BCC3E9B011C3F8D022C3F82001C3F82411704700BF80B6002012
:201A800000B583B00268084B8188CDF801203222D3F8D832ADF805108DF80020684698479D
:201AA00003B05DF804FB00BF80B600205E2810B511D05D2805D00D4BBDE81040D3F8DC325E
:201AC00018470A4CD4F8DC329847D4F8DC323D20BDE810401847054C5D20D4F8DC32984786
:201AE000D4F8DC323E20BDE81040184780B6002070B5094E0546D6F8DC325E200C469847B2
:201B0000D6F8DC3228469847E0B2FFF7CFFFC4F30720BDE87040C9E780B6002003682DE98C
:201B2000F041002B3D4D3E4F3E4EB8BF5B42A5FB0321890D07FB0137C7EB0717BF0096F8E1
:201B4000E63285FB0725FA170446C2EBA555002B57D101EB810101EB810105EB810109B263
:201B6000DFF8BC801320FFF7C3FF2F4908FB057581FB0531ED17C5EBA11109B21B20FFF76E
:201B8000B7FF2368254D002BB4BF53214E212320FFF7AEFF636896F8E62283EAE376A6EB73
:201BA000E376A5FB0631890D08FB0168C8EB08184FEA880885FB08354FEAE873C3EBA5555E
:201BC0002ABB01EB810101EB810105EB810109B21220FFF78DFF124B134903FB058581FBA6
:201BE0000531ED17C5EBA11109B21A20FFF780FF6368002BBDE8F041B4BF57214521222080
:201C000076E7C1EB011105EB810109B2A8E7C1EB011105EB810109B2DAE700BF6BCA5F6B83
:201C2000806967FF80B60020D34D6210044BD3F8003330EA030314BF01200020704700BF76
:201C400080B6002030B40023022515244FF4167140F2D93205808471018130BC4281438052
:201C6000838083817047134B10B400220F2483F80613090A83F8050383F80713C3F808238A
:201C8000C3F80C23C3F8102383F8044303F54170012110F8014F013122440E29D2B2F8D16B
:201CA00083F812230449D3F814035DF8044B102237F0E2BF80B6002084B90020054B002183
:201CC00083F81813C3F81C13D3F8143303B1CAE7704700BF80B6002013B50446FFF740FCED
:201CE00008B300230DF106022046ADF806300DF06BFCC0B10D4C9DF8062094F9CC1084F8F1
:201D0000E120032908BF62F07F024FF00501084808BF84F8E120FFF78BFC062184F8E20021
:201D20000348FFF76DFC02B010BD00BF680400204505002008B5044BD3F8200337F0CCFFD9
:201D4000B0FA80F0400908BD80B600202DE9F84F1B4C05461E2094F824A394F825B394F875
:201D60002663B4F82893B4F82A8394F82C7322F0A3FA30B1B8F1000F03D0C14601264FF067
:201D8000000A94F82E33DA070AD494F833233AB9012F12D0022F03D113F0020F08BF01269F
:201DA00085F800A085F801B0AE70A5F80490A5F806802F722846BDE8F88F3E46F0E700BF11
:201DC00080B600202DE9F84F2DED028BFFF7C8FB002844D0264B93F9CC0001283FDD93F81B
:201DE000E340DFF894809FED238A0FF27C0BDBE900AB15468E1E02EB44094D4504D1BDEC54
:201E0000028B2046BDE8F88F38F8027B26F8027F07EE907AF8EEE77A67EE887A17EE900A1B
:201E200053F024FE52465B4653F078FE41EC100B56F002FF51EC100B54F098F90E2F80B220
:201E40000AD919303223B0FBF3F080B200EB800000EB8000400080B225F8020BCDE70024F7
:201E6000CDE700BFAFF300801655B5BBB16B024068040020CDCCCC3DD8B9002038B50D4675
:201E8000FFF76EFB044638B10C4890F8CF30DB0704D5B0F8D0002880204638BD084A90F9C4
:201EA000CD3092F82C2093FBF2F102FB113201320131E4300DF09CFBEDE700BF6804002072
:201EC00080B6002038B5134C94F8313094F830209A4219D004EBC3030F49D3E90D200023B9
:201EE000984212DC93780D4AC4F868035B081370FCF718FB94F8313006210133B3FBF1F2CC
:201F000001FB123384F8313038BDD55C01F8015B0133E5E780B60020C46A0020F26A002008
:201F2000A1F5AF53B3F5AF7F70B541D8214BD3F86C03A3F86A10B0B94FF47A744C434FF4CE
:201F4000C8714BF0B3F92823B4FBF3F303F03F034FF420610120B4FBF1F1BDE8704043EA54
:201F6000C1114BF0A3B9144C4068A1FB044580214FF014F943F210204BF0F8F90A2037F03C
:201F8000B1F90E4A00232046294654F05FF9C0F30510460129462046094A002354F056F9BE
:201FA00046EA003040F01100BDE870404BF0DEB970BD00BF80B600200084D71740420F0014
:201FC0000000093D13B500230DF106020C46ADF806300DF0F9FA30B1044B9DF8060083F867
:201FE0006C404BF0FBF902B010BD00BF80B60020194B37B593F8682004461D4651B13AB96D
:020000040801F1
:20200000D3F87003012283F8682008B13AF082FE03B030BD002AFBD0D3F8700383F8681033
:2020200008B13AF071FE4FF4AF7037F079FA95F96C1000230DF106022046ADF806300DF0E1
:20204000C3FA9DF806004BF0C9F9B5F86A102046FFF766FFDCE700BF80B600202DE9F04F16
:20206000AB4B1B788BB08046002B40F0B980A94DD5F87463002E00F0B380A74AD2F8E84074
:2020800004F0F021B1F1E02F70D1C2F8E830D5F8782394426AD004930593ADF81830B5F836
:2020A000283395F824E3ADF8143095F825C395F82C3395F826B38DF818300DF1100A8DF817
:2020C00010E08DF811C08DF812B09AE8070007AB03C3924F1A80C4F342533B44C4F3034230
:2020E000997CC5F878438E4502F1010201D1944508D030468DF81C108DF81D200DF078FAAF
:20210000ADF8200030460DF05BFD032804F0070937D0042838D001283AD14F44FB7D9B45A6
:2021200001A9304618BF8DF81E300DF0DBFA48B1019BC4F3001103F001038B4202D030469A
:202140000DF0DEFC0A2207A9504657F01CF868B19DF81E30BDF81C2085F82633BDF8203013
:20216000A5F82423A5F8283345F010FB95F87CA304AF95F87C33032B7CD8DFE803F00B342D
:2021800077A44F44FB7FCAE74F4497F82730C6E70023C4E7394630460DF0AAFA044658B189
:2021A00007A8FFF7D3FD9DF81E109DF810308B4260D030460DF0A7FC95F87C33013303F09C
:2021C000030385F87C330CB99A45D2D195F82E33DB0700D524B1336841461B683046984712
:2021E0000BB0BDE8F08F01A8FFF7B0FD95F82E939DF8044009F00109ECB1B9F1000F39D12A
:202200003A460DF1030130460DF0DCFA044688B307A8FFF79BFD9DF81C109DF803309DF813
:202220001D208B4203D19DF81030934222D030460DF074FCC0E7B9F1000FBDD1394630465E
:202240000DF053FA0446A8B107A8FFF77FFDBDF82010BDF810308B420CD085F87D9385F8E3
:202260007E93336830469B699847A5E795F82E33D80701D500249FE707A930460DF032FA31
:2022800004460028F6D01E2022F016F895F87F3383428146EED085F87F0360B1B5F82A3305
:2022A000002BE7D1079BD907E4D4012130460DF027FC4C4680E7079BDA07DBD50146304660
:2022C0000DF01EFC78E73846FFF740FD97E8070007AB03C31A809DF810309BB10DF11D0201
:2022E00007A930460DF06EFA0DF11E0130460DF0FFF90A2207A9384656F045FF041E18BFEE
:20230000012459E708A930460DF0EFF9ECE700BF726B002080B6002068040020F09B060842
:20232000024B0146D3F8800337F0DABC80B600202DE9F041FD2984B0044600F0DE80F02956
:2023400000F0BD80EF2900F031814AB10346861803AD002003F8010B9E4205F8010BF9D12A
:202360009A4B0B2003F1090501E013F8010F814200F0C880AB42F8D14B1E832B00F2938082
:20238000DFE813F03201390143014E01C0018400580163016F01910091007501750175017D
:2023A0008D018D018D016F01910091009801A001910091009100910091009100910091001F
:2023C0009100910091009100910091009100910091009100910091009100910091009100ED
:2023E0009100910091009100910091009100910091009100910091009100910091009100CD
:2024000091009100B601910091009100910091009100910091009100910091009100910086
:2024200091009100910091009100910091009100910091009100910091009100910091008C
:2024400091009100910091009100910091009100910091009100910091009100910091006C
:2024600091009100910091009100910091009100910091009100910091009100910091004C
:2024800091009100910091001F011F01504BB3F8B013002900F0688101922DF09FFE019AC5
:2024A00080B2ADF80C003AB1224403AB13F8011B04F8011BA242F9D104B0BDE8F081454FEF
:2024C00003214FF00508B844002501370CE0FFF743FA064660193246FFF72AFF70194745A3
:2024E000C5B2E9D017F8011B412981F08003084601D0042BEBD80426ECE7374F0B214FF024
:202500000408E0E7324BD3F8140180060CD4002AD2D0224403AB13F8011B04F8011B944230
:20252000F9D104B0BDE8F08193F88403870742D52A4D287D052834BF02260326142917D996
:202540007C39C8B20628E2D80629E0D801A050F821F000BF41270108412701082B27010887
:202560000F250108512701084B270108572701080929CCD90A390A29C9D801A757F821F0A5
:20258000112701085D2701080F2501080F2501080F2501080F2501080F2501080F250108FF
:2025A0000F25010823270108412701080C4F0C214FF0060887E7094B0B29187DA7D101261B
:2025C000CDE0084B5B6B03936DE700BF209C060880B60020F49B0608F09B0608D8680020D6
:2025E000FC9B0608D85000200192FFF7E9F9019AADF80C0057E76C4BD3EDE87AFDEEE77AD4
:2026000017EE903AADF80C304DE7674B93F8EB02B3F88813002840F0AD80ADF80C1042E7F7
:202620006149B1F8883391F89013B3FBF1F3ADF80C3038E75C4D95F82E33DE0700F19F8042
:20264000B5F8B033ADF80C302DE7574B5749B3F9343481FB0301DB17C3EBA103ADF80C30FA
:2026600021E7514BB3F83634ADF80C301BE7A1F10C034D49DFED4E6AD1EDF47ADBB2143303
:2026800001EB830393EDF47A67EEA67A67EE877AFDEEE77A17EE903AADF80C3003E7424B9C
:2026A00003EB4101B1F8123403EB83035B00ADF80C30F8E63C4B93F82E3303F00103ADF85E
:2026C0000C30F0E6384BB3F8CC13CD055ABFCB4303F00103032311F0440F18BF042311F072
:2026E000020F18BF072311F4806F18BF0923A9E70192FFF765F92F4B019ADB6B43EAC040D2
:202700000390D0E6284BD3F8C033ADF80C30CAE62B8A03EB830303EB83039B00ADF80C3095
:20272000F5E6EB89ADF80C30F1E6EB89224903EBC3039B00A1FB03135B09ADF80C30E6E6A1
:20274000B3F88633ADF80C30E1E66B680393DEE62B680393DBE6AB680393D8E6F6B28DF8C2
:202760000C608DF80D00D2E6D3F8C80380F3100080B296E693F89033B1FBF3F14DE7019237
:2027800021F0AAFFD5EDE87A019AFCEEE77A17EE903A9BB200287FF455AF0849096811F0F7
:2027A000100F18BF00234DE780B600206766666600007A44D85000201F85EB51A0670020D0
:2027C00070B5214D95F83834EA181C4692F83C248AB11E4E09225C1CA6FB04135B0803EBCC
:2027E000C303E31AE918DCB291F83C1409B1013AF1D185F8384402681549561C06600C262C
:2028000016700268561C0660002616700268561C066003EB430603EB8603147019440D2244
:202820003FF0BCFB95F83814084B4A1CA3FB02035B08294403EBC3030120D31A81F83C0432
:2028400085F8383470BD00BF80B60020398EE338C8BA00202DE9F0416A4ED6F8747384B0E1
:20286000044638460D460DF0ABF986F8BD0457B10DF1090202A938460CF0A4FF002840F02C
:20288000838096F8BD040023ADF808308DF80A301A46431EDBB20021FF20FD2B8DF80C20C0
:2028A000ADF80E108DF80B0003D9002004B0BDE8F0819DF80830042B00F09D80052B00F0D6
:2028C0009D80032B00F09C80022B00F09380012B08BF042100F08F809DF809309DF80A10DD
:2028E000D6F87403013B0DF10E028DF809300CF06BFE96F8BD34032B7AD0042B76D0012B8E
:2029000064D0D6F8C024029B3F4F9A420DF108084FD023680D22591C21601A7023680022B6
:20292000591C21601A7023689DF80820591C21601A7023689DF80920591C21601A702368FB
:202940009DF80C20591C21601A7023689DF80A20591C21601A70BDF80E1020463FF066FBA3
:2029600023689DF80B20591C216020461A700721FAF7AAFF98E8030087E803000120C6F890
:20298000C85404B0BDE8F08101A938460CF0AAFE00283FF476AF38460DF10A010CF0A8FEDC
:2029A00000283FF46EAF019B96F8BD0403F001026FE77A68D8F804309A42AAD1D6F8C83461
:2029C000124AEB1A93427FF670AFA2E7104A9DF80A000121002304E00133082B91D012F8B0
:2029E000011F8142F8D38DF80A308AE7094AEEE7094AECE703218DF808106DE70121FAE793
:202A00000221F8E780B6002040BB002080841E00079C0608179C06080F9C06082DE9F041AF
:202A20002A4C2B4AD4F8C033B4F8CC74B4F8C86382FB0352DB17C3EBA2031FFA83F84745F2
:202A400082B00D4603D1B4F8CE34B34233D002680190511C34230160137002680023511CDA
:202A60000160137041463FF0E1FA019831463FF0DDFA019847F6FF713FF0D8FA019847F6AE
:202A8000FF713FF0D3FA019847F6FF713FF0CEFA019847F6FF713FF0C9FA01980221FAF7A8
:202AA00013FF0120A4F8CC84A4F8CE64C4F8D05402B0BDE8F081D4F8D034064ACB1A9342A7
:202AC000C5D8002002B0BDE8F08100BF80B600206766666680841E00026810B57F21541C62
:202AE0000460117002680024511C01600E211470FAF7EAFE012010BD2DE9F04FC24B1B6836
:202B0000804613F0800083B000F07181BF4B93F8840310F0020000F06A81DFF810B39BF831
:202B20001430052B40F26881DBF80030B84D0093002BB8BF5B42A5FB0342B648B649920DAB
:202B400000FB0233C3EB03139B0085FB034502EB8202DC1702EB8202C4EBA55400FB04336F
:202B600004EB8204A4B281FB0321DB17C3EBA111BCB10025A94F2E46A7FB0432D20802EBFB
:202B80008203A4EB4303E8B2A4469BB280008340BCF1090F94B246EA030605F10105EBD8C4
:202BA000340489B2B9B100259C4F2E46A7FB0132D20802EB8203A1EB4303E8B28C469BB208
:202BC00080008340BCF1090F91B246EA030605F10105EBD83443DBF804E08D4D8D4E8E49F8
:202BE0008EEAEE70A0EBEE70A5FB0032920D06FB0200C0EB0010830085FB035002EB820220
:202C0000DD1702EB8202C5EBA05506FB053305EB8205ADB281FB0321DB17C3EBA111C5B133
:202C20000020DFF8F8C10646ACFB0532D20802EB8203A5EB4303C7B2A9469BB2BF00BB4029
:202C4000B9F1090F95B246EA030600F10100EBD8350489B2C1B10020DFF8C0C10646ACFB2C
:202C60000132D20802EB8203A1EB4303C7B289469BB2BF00BB40B9F1090F91B246EA030676
:202C800000F10100EBD83543DBF80830634A0193002B1846B8BF5842A2FB0030604E6149FC
:202CA000030AA6FB0363DB0901FB03F1C1EBD00189B2B9B1002691463746A9FB0132D208DF
:202CC00002EB8203A1EB4303F0B28C469BB280008340BCF1090F91B247EA030706F101066B
:202CE000EBD8B9B2BBF81070DFB10026DFF82CA1B446AAFB0732D20802EB8203A7EB43031D
:202D00005FFA86F938469BB24FEA890903FA09F3092897B24CEA030C06F10106E9D81FFAB5
:202D20008CF7BBF812303D4AA2FB0306F608632E28BF6326092B63D9002093468146ABFB19
:202D40000632D20802EB8203A6EB43035FFA80FAB4469BB24FEA8A0A03FA0AF3BCF1090F72
:202D600096B249EA030900F10100E8D85FFA89F9009B019A002BCCBF392338231616BEF1C1
:202D8000000F26F07F0635DD274A3343964543F00206C8BF43F00606D8F800301622581C08
:202DA000C8F800001A70D8F800300022581CC8F800001A7040463FF039F9214640463FF0E6
:202DC0001DF9294640463FF019F9404639463FF02DF9D8F800305A1CC8F8002083F80090EC
:202DE000D8F800305A1CC8F8002001201E7003B0BDE8F08F1E43CFE7002003B0BDE8F08FE9
:202E00004FF00009B4E700BFA067002080B600206BCA5F6B806967FFD34D6210CDCCCCCC82
:202E2000C55A7C0AA0860100FFC99A3BD86800202DE9F047AB4B1B68064613F0800084B000
:202E400000F09E80A84B93F8840310F0020000F09780A64F397D052940F29780632900F2B6
:202E600092800024DFF898C289B22546ACFB0132D20802EB8203A1EB4303E0B28E469BB29A
:202E800080008340BEF1090F91B245EA030504F10104EBD8EDB2BB68954A82FB0312D917CE
:202EA000C1EB623189B2002900F018814FF0000CDFF84CE26446AEFB0132D20802EB8203C4
:202EC000A1EB43035FFA8CF088469BB280008340B8F1090F91B244EA03040CF1010CEAD8E8
:202EE000E4B2FB8983494FF4F36707FB03F7A1FB0737C7F38F1742F20F739F4249D8CFB1E1
:202F00000020DFF8FCE18446AEFB0732D20802EB8203A7EB4303C1B2B8469BB289008B40FB
:202F2000B8F1090F97B24CEA030C00F10100EBD81FFA8CF7704BD3E9002313433ED14FF0B3
:202F4000FF3833681722591C31601A7033680022581C306039461A7030463FF067F8414681
:202F600030463FF04BF833685A1C32601D7033685A1C326030461C700621FAF7A5FC0120BA
:202F800004B0BDE8F087992585E7002004B0BDE8F0870021DFF868C10F46ACFB0302D2084B
:202FA00002EB8200A3EB40039BB28B400431102947EA030793B2F0D1BFB2BBE701A843F01B
:202FC000A1FF9DF80810002900F08A804FF0000CDFF82CE1E046AEFB0132D20802EB820304
:202FE000A1EB43035FFA8CF089469BB280008340B9F1090F91B248EA03080CF1010CEAD8BD
:203000004FEA08289DF80910E1B10020DFF8F0E08446AEFB0132D20802EB8203A1EB43037C
:203020005FFA80F98A469BB24FEA890903FA09F3BAF1090F91B24CEA030C00F10100E8D8E0
:2030400048EA0C089DF80A104FEA0828E1B10020DFF8ACE08446AEFB0132D20802EB82030B
:20306000A1EB43035FFA80F98A469BB24FEA890903FA09F3BAF1090F91B24CEA030C00F18F
:203080000100E8D848EA0C08BDF80C301B49632BA1FB03214FEA08184FEA51117FF651AF1D
:2030A0000020DFF85CE08446AEFB0132D20802EB8203A1EB43035FFA80F98A469BB24FEAF1
:2030C000890903FA09F3BAF1090F91B24CEA030C00F10100E8D848EA0C0832E70C4600E7D0
:2030E00088468FE7A067002080B60020D868002089B5F814D34D621058BB00201F85EB51C0
:20310000CDCCCCCC08B5A0F10103B3FA83F302284FEA531301D0184608BD0F2021F044F8D0
:2031200030B9064B93F82E3303F00103184608BDBDE808400F2021F0BFB800BF80B6002096
:2031400010B5084CE26D13899907FCD513891B06F9D40A2036F0C6F8206EBDE8104039F0B6
:20316000D9BD00BF301C0020014B1B681B6A18474C5F0020024B186808B183691847704788
:203180004C5F0020024B186808B14369184770474C5F002010B5074C606D40B13AF06AFDEA
:2031A00094F8513013B180F00100C0B210BD012010BD00BF301C002010B5FFF7EBFF0E4C76
:2031C00048B194F82430032B10D8237E0133DBB2072B237603D9002384F8243010BD074AE6
:2031E00001231268626184F8243010BDE06D4FF480714DF0D3FFE8E7301C0020D0240020F2
:2032000030B40A490A480A78531CDBB20525042B00EBC20400F8325008BF00234FF40452A0
:203220000B7062604FF0FF3030BC70471C6B0020206B0020037870B4FBB10446C0F10106A1
:20324000A31914F8015FDBB2002DF9D101335B00DCB2032513800C704D7004785CB1022303
:2032600000255A1CD2B2CC548D5410F8014F0233DBB2002CF5D170BC704702242346E8E7E1
:203280000B0617D401EB810300EBC30310B400EB81000124002283F8764383F8741383F8E9
:2032A0007523426D5DF8044B136843F4001300201360704701F07F0101EB810300EBC30382
:2032C000012200EB810083F81C1183F81E2183F81D2182691368002B01DA43F0804343F4AB
:2032E000001313600020704770B501F07F0505EB850400EBC404282101FB05010126C4F87D
:2033000030310023C4E94A2284F81C5184F81D61C4F8343101F58E711DB9FDF785FF0020A9
:2033200070BDFDF7F5FF002070BD00BF2249F8B5D1F8E0340F2B04D05A1CC1F8E024002016
:20334000F8BD1E4C25780023C1F8E034002DF6D11B4E1C4B3268B2F5006F17D01B689A4207
:2033600027D017D9C2F50063402B15D9403B02F14005C1F8E43401232370356092B240237C
:2033800011490A448121FFF7AFFFD8E71B6835607BB12A469B1AE7E74FF0000502EB03070E
:2033A000C1F8E4540CBF02210121376092B22170E6E700232370C2E780B600204029002095
:2033C000A8240020AC24002044290020AEE700BFF8B51D4C2378012B03D0022B09D000205A
:2033E000F8BD01461948D0F8E43453B923700020F8BD00231A468121FFF776FF00232370D6
:20340000F5E7402B11D9124C2268403B02F14005C0F8E434256092B240230E4C08462244D6
:203420008121FFF761FF0020F8BD094D2A684FF0000603EB0207C0F8E46408BF02202F6023
:2034400092B208BF2070E8E74029002080B60020A82400204429002038B5134602250A46ED
:20346000C0E94E3380F811510021FFF73DFF002038BD00BF10B50C7814F0600413D0202C41
:203480000AD14B78023B092B18D8DFE803F01B21171717171717272E22490122FFF7DCFFF9
:2034A0000024204610BD4B78062B24D00A2BF3D01D4B8A78C3F8F024204610BDFBF764F81B
:2034C0000224EEE719490122FFF7C6FF0024E8E717490122FFF7C0FF0024E2E74B88124A6A
:2034E0001B0AC2F8EC340024DBE70F4B8A78C3F8E8240024D5E74B881B0A222B0CD0212B77
:2035000004D021462246FFF7A7FFCAE7CA880949092A28BF0922F6E7CA880749262A28BF1C
:203520002622F0E770BB002080B600206CBB002068BB00208E0500205405002038B501EB3C
:20354000810400EBC4040D46002184F87453C4F88C1384F87513C4F88833C4F88023C3780C
:203560002821012B01FB050108BFEDB201F55D7108BFC4F884231DB9FDF756FE002038BD4D
:20358000FDF7C6FE002038BD144B9A6870B5044662B1134A1B7B92F8F4542B4316D08121C0
:2035A0002046FFF76DFE022D09D070BD0C4B93F8F45481212046FFF763FE022DF5D120462B
:2035C000064ABDE870401F230121B7E70121FFF757FE20468121BDE8704051E6FC6A0020BD
:2035E00080B6002070B5094A094D1173094B13600021044629700D238121FFF775FE2046B7
:20360000054ABDE870401F23012197E75C6B0020506B002055534253FC6A002010B5064B89
:20362000597B0446FAF7BEFF002800DB10BD20460121BDE81040D5E7FC6A00202DE9F041E8
:20364000314D2C7834B1012C01D1FFF7E7FF0020BDE8F0812D4FDFF8D080B0F8B4337A683E
:20366000C8F804201F2BBA68C8F80820064606D1274B3A689A4202D1797B01291AD9254AAC
:2036800025491378052401F8334001EBC3000133DBB2042B08BF00234FF4005113701F4B92
:2036A00041600222304683F8F424FFF76DFF0020BDE8F081BB7B013B0F2BE0D8FAF772FFDE
:2036C000002819DB2B78013B022BC0D9144B1988B1B1BB68D8F8082088F80C408B4228BF2C
:2036E0000B46D11A0424C8F808100E4A2C7030468121FFF7F9FDAAE73046FFF745FFA6E7C8
:203700003046FFF76FFFA2E7506B0020FC6A0020555342431C6B0020206B002080B6002010
:20372000446B0020288E00205C6B002008B5084B1B78022B07D0033B012B02D80021FFF7FB
:2037400051FF002008BDFFF769FF002008BD00BF506B002010B501EB8101084A00EBC10125
:203760000446B1F88C131046F4F744FD034A204640230121FFF7E2FE002010BD78BB0020E7
:20378000E8E700BF70B50A7812F060050C46064611D0202D16D1CD88D5B113062AD52A4677
:2037A0001F496078F4F750FDE2881D493046FFF753FE00250AE04B780A2B16D00B2B0ED003
:2037C000062B03D13046FAF7DFFE0225284670BD022260781144F4F737FD284670BD8B78D0
:2037E000D3B9104BC3F83855F0E70F490122FFF733FEEBE70D4964780A4AC1F8C8400321E4
:20380000C0E9E45542F8045B2B4680F811110021FFF794FE0025D9E7FAF7B6FED6E700BF73
:2038200084B6002080B60020B8BB0020680400200B7803F00303012B03D0022B04D000201D
:2038400070478B881BB915E68B88832BFBD099E710B50223044640228121FDF761FC2046D4
:20386000022340220121FDF75BFC8221204603230822FDF755FC064B02229A80F4F732FD0D
:20388000044A204640230121FFF758FE002010BDB001002078BB002038B508220D460446DE
:2038A00003238321FDF73CFC29462046FFF7D0FF002038BD82B00023016801930B69019309
:2038C0000E4B03E00A690192013B13D0019A002AF8DA019A094B42F001020192019A0A6133
:2038E0000A69019203E00A690192013B02D0019AD207F8D4002002B0704700BF400D0300F3
:20390000436D064A1A61C278012A06D100F2CC5058614FF0802219681A6070471800086016
:2039200010B5002304220446194680F811211A46FFF7DAFC2046FFF7E3FF002010BD00BF10
:2039400010B5044629B990F81131032B0DD0002010BDD0F8E4359B69002BF8D090F8122121
:20396000032AF4D19847002010BDD0F89013D0F87C33994214D9C078D4F880230128A1EB83
:20398000030104BFD218C4F880238B4228BF0B46C4F890139BB220460021FFF7CFFDD6E760
:2039A000D0F8E4351B691BB190F81221032A03D02046FFF7B5FFCAE79847F9E7F0B50121D4
:2039C00090F8D17590F8D36590F8CFC590F8CE5590F8D03590F8D22580F8111190F8CC1583
:2039E00085B005EB0C2503EB072302EB062201F01F06AFB292B290F8CD558DF808109BB2F5
:203A0000012E0446ADF80A70ADF80C30ADF80E20C0F840218DF8095017D0022E1FD036B176
:203A200001F08001FFF72CFC002005B0F0BD092D0FD8DFE815F0BF00AC000E00D5000E002F
:203A4000EA0085000E007700540090F81221032A2FD02046FAF798FD002005B0F0BD01F0D8
:203A600060012029DAB234D0012D00F02081032D00F00681002DD7D190F81211022900F00B
:203A8000DF800329E5D11B0600F14B8102EB820200EBC20393F87633002B00F04D81BF4BBF
:203AA0000122C3F84C25BE4920460222FFF7D4FCBAE7DAB2012ACCD8D0F8E43502A99B68D5
:203AC0009847BDF80E30002BAED12046FFF728FFAAE7D0F8E43502A99B689847A4E7F9B2B2
:203AE000AE4D012985F83C15B3D890F81231022B00F02781032BACD1002900F0868190F865
:203B000010110129E1D0D0F8E4355B68984795F83C1584F810112046FDF770FA2046FFF78B
:203B2000FFFE81E7012A94D190F81231022B00F01781032B8DD100F58871FFF78DFC73E7BD
:203B40003D0A022DADF8062000F05081032D00F00B81012D7FF47DAFD0F8EC3580781B6886
:203B60000DF106019847BDF80620002A3FF45CAFBDF80E30002B3FF457AF9A4228BF1A46A4
:203B800001462046ADF80620FFF766FC4CE790F81231023B012B3FF65CAF012F7FF444AF18
:203BA000D0F8E43500229B68C0F8182102A9204698478AE790F81231023B012B3FF649AF4C
:203BC000764BD0F818210021C3F8441512B10222C3F84425734920460222FFF73DFC23E764
:203BE000012F00F09880022F7FF41EAF13F0FF0F7FF41AAF02691B0A023B5268032B00F228
:203C00001D81DFE803F0393531241A437FF421AF90F81231032B3FF41CAF036907F07F050B
:203C200080F81451196867F30A120A431A60FFF777FE002D00F0E580022384F81231F3E63F
:203C400051063FF4F1AE1146FFF71AFBECE6052363F30612514B012184F816112046C3F8EF
:203C60004825FFF75DFEDFE6042363F30612F1E7032363F30612EDE7022363F30612E9E789
:203C800090F81231022BDBD0032B7FF4E2AE27B9550602D01146FFF7F3FAD4F8E43502A979
:203CA0009B68204698472046FFF73AFEBCE690F812110229C4D003297FF4CBAE002F7FF462
:203CC000B3AE12F07F013FF400AF180600F1A78002EB820304EBC30304EB810083F87673EE
:203CE00083F8741383F87573282303FB0243416D03F55D73DA780B68023A6FF35553012A25
:203D0000D4F8E42598BF43F080530B602046936802A99847D9E6D0F8E435C0F818719B6837
:203D200044E702F07F0202EB820200EBC20393F81E31002B7FF4B3AE184B0022C3F84C253A
:203D4000B1E600293FF4C1AE0121032380F8101180F81231FDF752F92046FFF7E1FD63E6A3
:203D60001149FFF779FB5FE6FDB2052D3FF671AEDFE805F0342C241C0B03D0F8EC358078BA
:203D80009B690DF106019847EDE6D0F8EC3580785B690DF106019847E5E600BF80B60020FF
:203DA000CCBB0020C4BB0020C0BB0020D0F8EC3580781B690DF106019847D4E6D0F8EC3536
:203DC0008078DB680DF106019847CCE6D0F8EC3580789B680DF106019847C4E6D0F8EC35B7
:203DE00080785B680DF106019847BCE6D0F8E43580789B6A0DF1060198474570C4F8F0055A
:203E0000B1E6012384F812310EE60222D0F8E43580F8101180F812215B68984755E62822C4
:203E200002FB014304EB810083F81E7183F81C1183F81D51816903F58E735BE7012363F397
:203E4000061207E770B5044649B990F81131022B1BD094F81631012B0DD0002070BDD0F818
:203E6000E4355B69002BF8D090F81221032AF4D19847002070BD2A4A2369D2F848255A60A8
:203E8000002384F81631002070BDD0F83831D0F82451AB4217D9C278012AD0F82821A3EBA0
:203EA000050308BF5219C0F8383108BFC0F828219BB20021FFF718FA00231A461946204621
:203EC000FFF73CFBC5E7D0F83C31B3FBF5F605FB163666B99D420AD8D0F84021934206D239
:203EE00033463246FFF700FAC4F84061E4E7D4F8E435DB681BB194F81221032A0CD00023DA
:203F0000052284F8112119461A462046FFF716FB2046FFF7F5FC9CE720469847EFE700BFF6
:203F200080B6002082B000230193019A094B42F010020192C168019A0A610A69019203E064
:203F40000A690192013B02D0019AD206F8D4002002B07047400D030082B000230193019AB1
:203F60000B4B42F020020192019A61F38A120192C168019A0A610A69019203E00A690192C8
:203F8000013B02D0019A9206F8D4002002B07047400D0300F8B50B7813F060050C46064605
:203FA0001CD0202D17D14A78FE2A44D0FF2A3DD14A88002A56D1CD88002D53D11B0651D49C
:203FC0003749384B0D70012183F8F414364A1F23FFF7B4FA00E000252846F8BD4B780A2B36
:203FE0004BD00B2B44D0012BF6D191F904308988002B47DBFFF796FF21792A4F3046FDF745
:020000040801F1
:204000002BF80223217940223046FDF789F897F8F434022B3BD094F90420002ADCDA012BC5
:20402000DAD030460121FFF7DDFAD5E70225FAF7ABFA2846F8BD4D88A5B9CC88012C11D13F
:204040001A060FD5194B1B689B6998471549C0B281F8500530B1224601F5AA613046FFF73E
:20406000FBF9B9E730460225FAF78EFA2846F8BD0C4B4A8883F85125AEE70D490122FFF755
:20408000EBF9A9E701F07F01FFF766FFB4E730468121FFF7F5F8002387F8F4349CE700BF3E
:2040A000506B002080B60020FC6A0020406B0020D1BB002038B50446FDF704F82046022320
:2040C00040228121FDF72CF82046022340220121FDF726F80C4B0D491B680D4A00250D707A
:2040E0001B6882F8F454284698472046FFF71AFF20460121FFF730FF064A20461F230121F2
:20410000FFF71CFA284638BD406B0020506B002080B60020FC6A0020012905D008B50321CE
:20412000FFF71AFF002008BDFFF752B900B583B009238DF80730FDF7A3F98DF807009DF809
:204140000730012BF7D09DF8070003B05DF804FB82B0064B002201920193019B03EB8000BC
:204160000190019B186802B0704700BF5028004082B0064B002201920193019B03EB8000DC
:204180000190019B196002B0704700BF502800400023C0E90033C0E90233C0E90433C0E933
:2041A0000633C0E90833C0E90A33C0E90C338363704700BF0B6870B4D1E90524CD682B439B
:2041C0001343D1E9072523431343D1E909422B43D1E90D652343134304680B4A33432240F3
:2041E0002B4313430360D1E90B3442690D6922F0070223431343D1E901424361456084607D
:2042000070BCC260704700BF3F801CF002683649002310B422F00102212488420260036056
:2042200043608360C3600361446138D02F4B98422ED02F4B98423CD02E4B984240D02E4B36
:20424000984232D02D4B984241D02D4B984246D02C4B984217D02C4B98423CD02B4B9842D2
:2042600016D02B4B984224D02A4B984228D02A4B98421AD0294B984229D0294B98422ED001
:20428000284B984208D14FF03D5243F8AC2C03E04FF4746243F8202C5DF8044B7047224BCC
:2042A0005DF8044B3D229A607047204A43F8642CF2E74FF474125DF8044B43F8382C704779
:2042C0004FF074625DF8044B43F8502C7047184A43F87C2CE0E73D2243F8082CDCE7154ABB
:2042E00043F8942CD8E700BF106002402860024040600240586002407060024088600240B1
:20430000A0600240B860024010640240286402404064024058640240706402408864024055
:20432000A0640240B8640240006002403D000020400F002000003D200B88F0B433BB028C5B
:204340004C880E898B88C98822F001021204120C0284058B028CADB225F0F30592B22B4383
:2043600022F00A0243EA061322439BB242F0010203830284038B23F00C031B041B0C03836A
:20438000038B9BB21943F0BC01837047042B048C2CD0082B4E888A880D89C98851D024F409
:2043A00080542404240C0484838B078C2C0344EA022440F6FF421A4045F6FF733B4043EAFF
:2043C000063322439BB292B243F4805382830384828B22F440621204120C8283838B9BB2BF
:2043E00043EA01239BB2F0BC8383704724F010042404240C4D880F898A88C9880484068B4D
:20440000038C12029BB242EA073423F0A00340F6FF42324043EA051322439BB292B243F038
:20442000100302830384028B22F440621204120C0283038B9BB243EA01239BB2F0BC0383B4
:20444000704724F480742404240C0484848B038CA4B29BB224F0F30423F42063224343EA41
:20446000062342EA05129BB243F4807392B282830384838B23F00C031B041B0C8383838BFF
:204480009BB21943F0BC8183704700BF214A038890429BB212D002F5806290420ED0B0F12C
:2044A000804F0BD0A2F58032904207D002F58062904203D002F58062904203D14A8823F07E
:2044C00070031343144A904218D002F58062904214D030B423F440730C894D6802F56C42CF
:2044E0009BB2234390420C880380C56204850DD18B7A0386012330BC8382704703800B8822
:204500004A68C2620385012383827047034B9842EED0EFE7000001400010004000040140CB
:20452000024A536A23EA00005062704700380240024A136A23EA0000106270470038024009
:20454000484B98422ED0B0F1804F32D0464B984236D0464B98421ED0454B984237D0454BB3
:2045600098423BD0444B98423FD0444B98424BD0434B984240D0434B98424CD0424B9842F7
:2045800051D0424B984256D0414B98425AD0414B98425ED07047404A136A43F004031362DC
:2045A0000420C5E73C4A536A43F0010353620120B6E7394A136A43F0010313620120B7E7D3
:2045C000354A136A43F0020313620220B0E7324A136A43F0080313620820A9E72E4A136A20
:2045E00043F0100313621020A2E72B4A136A43F02003136220209BE7274A536A43F48033B0
:2046000053624FF480308BE7234A536A43F002035362022084E7204A536A43F40033536296
:204620004FF400307CE71C4A536A43F4802353624FF4802074E7184A136A43F040031362EA
:20464000402075E7144A136A43F08003136280206EE7114A136A43F4807313624FF48070F9
:2046600066E700BF000001400004004000080040000C00400010004000140040000401402C
:2046800000400140004401400048014000180040001C00400020004000380240224A936896
:2046A00003F00C03042B10B421D0082B22D01F4B03601D4C1E4AA168C1F30311114491F8A2
:2046C0003811CB404360A168C1F38221114491F8381123FA01F18160A1685DF8044BC1F30B
:2046E00042310A4492F83821D340C3607047114B0360DEE75468516852686302C2F38812C2
:204700004CBF0C4B094B01F03F01B3FBF1F303FB02F3054A5268C2F3014201325200B3FBF9
:20472000F2F30360C5E700BF003802400024F4006804002000127A002DE9F04700230F6835
:2047400001264FF0030C02E00133102B41D006FA03F232EA0704F7D1D0F800E05C000CFA94
:2047600004F52EEA050EC0F800E091F80490D0F800A009FA04FE09F1FF394EEA0A0EB9F1C7
:20478000010FA846C0F800E06FEA050515D8D0F808E005EA0E0585604D79D0F808E0A54041
:2047A00045EA0E058560456825EA020242608A7945689A4092B22A434260C26822EA080253
:2047C000C260CA79C568A24001332A43102BC260BDD1BDE8F0870D4B93F82E23D20703D5D8
:2047E000012283F85225704793F8522562B9D3F874234AB193F82423104493F8252383F8FF
:204800002403114483F82513704700BF80B60020044B93F90C00012806BF02221A730020F7
:20482000704700BF80B60020114AD2F85405A0B1D2F858358BB188420DD88B4234BF0023B8
:2048400001239BB11369C2F85C1599421CBF142382F86035DCE70023F3E7A1F59C53083BBD
:20486000B3F57A7F2CBF00230123EAE7704700BF80B6002007B500230DF10602ADF8063008
:204880000AF0A2FE60B1084BBDF80620998AA3F8622591421CBF142283F86425FFF7B8FF65
:2048A00003B05DF804FB00BF80B6002013B50446262001911FF000FD019948B9054BD3F830
:2048C00014332BB1204602B0BDE81040FDF7CBB902B010BD80B60020B1FA81F14909492083
:2048E000E4E72DE9F341BE4C94F90C3001330D4600F06681D4F81433002B00F0B3800227E8
:2049000000264FF00108D4F8140335F0E5F9002800F0A880D4F8140335F0D6F9D4F81C3311
:204920005A1C2344C4F81C2383F8650594F81833012B09D0022B15D063B90F280CBF84F832
:204940001883C4F81C33DEE7A0F17203012B06D9762804D084F81863C4F81C63D3E784F801
:204960001873D0E7102ACED19E490023012211F8010F013203440E2ADBB2F8D194F87325AA
:2049800084F818639A42C4F81C63BCD194F87435002BB8D194F86635732B59D0762B1BD019
:2049A000722B5FD194F8682594F8673594F90C1053EA022356D0C4F854350029B4F8693500
:2049C000C4F858354EDC94F8822501232373002A48D184F8823545E094F8682594F867359B
:2049E00053EA02233ED0D4F8782594F86A1594F86E05236193421CBF142284F8602594F8DD
:204A00006925C4F8783542EA0122B4F87C15A28291421CBF142184F8641594F86B15617337
:204A200094F86C15A17394F86D15A4F87C2541EA0021A4F87E15D4F85C1509B9C4F85C3543
:204A4000B4F862350BB9A4F862250223237309E094F86C2594F86B3543EA02231AB20BB165
:204A6000A4F8802594F90C30022B35D00FDCDAB2012A15D9636E13B1A369002B6CD15A49BE
:204A80005A481F2202B0BDE8F04154F0E2BB032BF0D1D4F88435564AEB1A9342EADD13E022
:204AA000D4F884255349AA1A8A42E3DD2BB97220FDF704F9C4F88455DCE7D4F888355A1CD7
:204AC000D907C4F8882503D47620FDF7F7F8F1E77320FDF7F3F8EDE7D4F85C15D1B194F8D4
:204AE0006035BBB12369994214D0637BDA0703D489B24620FFF7DAFE94F86035013B84F88C
:204B0000603505F59225032305F578752373C4F88455AFE7B4F86215A38A81B194F86425EA
:204B20006AB18B420BD0637BDB0702D45020FFF7BDFE94F86435013B84F86435E1E701229A
:204B40002273A4F862352269C4F85C25002384F8643584F860358DE7274DD4F874732A2394
:204B600085F848310DF1070220230DF10601384685F849310AF026FE30B19DF806109DF83C
:204B8000076051EA06031ED1552385F84A31462385F84B3122691948202385F84C31002A56
:204BA00034D0174946F0CEFDB4F87E3515488BB3A28A15499A420CBF20222A2246F0C2FDE2
:204BC00002B0BDE8F08138460AF07AFD314685F84A0138460AF060FD037885F84B31D9E7D6
:204BE00080B60020E5BB002022220708B0050020400D030040420F0068040020B505002030
:204C0000DD5B0708B90500203C220708034946F099FDC9E7024946F095FDD1E744220708FA
:204C20004322070810B50E4C40F0080284F86B2194F9CC20022A06DD420704D583071CBF90
:204C4000012384F8D43005210648FCF7F1FC062184F86C01BDE810400248FCF7D1BC00BFCE
:204C600068040020CF05002010B5FCF779FCA8B31B4C94F9CC30012B30DD59B3022B2DD0CD
:204C800094F8D4309BB971B180230521154884F87131FCF7CDFC062184F87201BDE8104003
:204CA0001048FCF7ADBCBDE810400420BAE7002914BF0020042094F8CF301A0748BF40F063
:204CC00002005B0701D411B108B940F00100BDE81040A7E7022BD3D10420ECE710BD00BF10
:204CE00068040020D5050020F8B5224C04F27317030A84F8780105460621384684F877317D
:204D0000FCF796FC94F8CF3084F87901DB072AD4B4F8D020AA4226D1174DD4F87331C5F89D
:204D20008C35C3B285F8923541F26F714FF6FF738A4218BF0123134405F28C56C3F3072259
:204D40000621304685F8902585F89135FCF770FC072185F892053046FCF752FC052104F5D0
:204D6000BD70FCF74DFCBDE8F84004480721FCF747BC00BF6804002080B60020DB050020E2
:204D800008B5FCF7EDFB48B1A1F59C53083BB3F57A7F03D2BDE808400846A5E708BD2DE9A2
:204DA000F0476B4E3368002B3AD06A4D6A4C05F1CC07306834F090FF002833D1674B198833
:204DC00009291D4609D95F8864227A43B2FBF1F2452A40F3A4811880588094F8CD35012BB1
:204DE00000F0C881022B00F0E38133B95C480521FCF706FC012384F8CD355A4B1D685A4BDD
:204E00001B78002B00F0DE81584B1B68EB1A782B40F2D881D4F86803F9F784FBC4F8D055A5
:204E2000BDE8F087306834F04FFF94F893358046052BBED8DFE803F00309171D3745AA2824
:204E4000B7D1012384F89335B3E7552803D1022384F89335ADE7414A93880133938000236A
:204E600084F89335A5E7032384F8940584F893359FE7132884F89505C4F8B00507DD374A36
:204E8000D3880133D380002384F8933591E718B9052384F893358CE70023C4F8B4350423B2
:204EA00084F8933585E7D4F8B435E218013382F89605D4F8B025C4F8B43593427FF479AF94
:204EC000E6E7D4F8B0352A4803F1020A4FFA8AF1FCF7AEFB804594F8949540F017812620FA
:204EE0001FF0EAF9204B48B100221A701B4A538801335380002384F893355AE71A784A45A0
:204F000019D100221A7009F1FF33102B00F2F980DFE813F030008E008E00E1008E00F700AD
:204F2000F700F7003000F700F700F700F700F700F700F7003000B9F1090F02D0B9F1110F04
:204F400001D1012ADDD0054A538901335381DAE7C06A00206804002080B60020E46A002019
:204F6000E2050020D0240020F26A0020F46A002014BC0020BAF1060F5ADDB9F1010F06D0A5
:204F8000B9F1090F0CBF4FF002094FF0030994F8990594F89A1594F8982594F996E594F9AC
:204FA00098C594F8973585F8CC9041EA002109B2900785F8CDE085F8CFC0A5F8D01006D537
:204FC00012F00C0F14BF0122002285F8D420B9F1030F13D1BAF1090F2ADD94F99C25082A41
:204FE000A8BF082222EAE27285F8E320002043B29A4200F101005CDC94F89B35D4F818A045
:20500000002002469BB2524590465ADB7D4B85F8CE001B78232B0BD109EB89037A4A03EB37
:2050200083030CEB83031380A2F802E09180D080764977480A2254F0A6F810B1002384F811
:20504000C235724B3A681A607A685A603A891A8194F8C23543BB95F8D43094F8242384F825
:20506000C425002B14BF0223012384F8C23595F8CF3094F8260384F8C80513F001031CBF21
:20508000B2FA82F35B0994F8252384F8C525D9B2B4F8282384F8C315A4F8C62513B10AB175
:2050A000A4F8CA2584F8CC150FF0E6F90FF0E4F91CE704EB4308234493F89E35A8F8583321
:2050C00095E704EB48080132B8F81C8052B2984508BF104697E7BAF1040FA9DD94F896258F
:2050E00094F8973543EA022359041AB204D5C3F30D03A5F8D2309BE7002AF8DBA5F8D03083
:2051000096E7444A938901339381EFE619F0010F7FF4F0AE3F4A138901331381EAE63E4BDB
:20512000D3F88021B3F88411012A1AD141F25632914203D14FF0FF32C3F88021D3F8802113
:20514000306802EB820202EB820201EB420189B2A3F8841103681B69984700232B806B80B4
:205160003BE60132EAD1B1F5965F04BF0122C3F88021E3E7284D95F9CC60002E3FF43DAEFE
:20518000022E11D14FF48040FFF7AEFD84F8CD6595F9CC30012B7FF730AE95F8CF30C3F35F
:2051A000400385F8D43028E6032384F8CD35EFE7194BB3F8D230002B3FF41FAE032384F8C5
:2051C000CD351AE694F8302094F831309A4204D0FCF778FEC4F8D05522E6D4F8D035EB1A2C
:2051E000B3F57A7FBFF41CAE0C4B1B68ED1A952D7FF616AE0A480521FCF702FABDE8F04772
:20520000FCF760BEA9280020AC28002038BC002034050020E46A002068040020F46A0020B3
:20522000E205002010B5134CD4F8740300B394F8241359B194F825230AF0DAF9B4F82833D8
:2052400083421ABFA4F8280301210021B4F82A2362B141F288339342B8BF13469A4205D056
:20526000A4F82A33BDE8104042F090BA0029F9D110BD00BF80B6002010B40144044600207C
:2052800014F8013B08225840430010F0800F08BF400083F0070314BFD8B2C0B2013AF3D1E0
:2052A0008C42EDD15DF8044B704700BF30B54FF4806085B02DF00CF940B3154C90F9040008
:2052C00094F8D435134A002B18BF08234FF4E1310125CDE90153009100234FF480612DF035
:2052E00058F9FF232067003818BF012084F88C3084F89C3084F8AC3084F8BC3084F8CC30CC
:2053000084F8DC3084F8EC3084F8FC3005B030BD80B6002029190108364B1A6812F000621B
:205320005CD0354B93F86EC0604559D3FF2855D1324A92F8DC20002A56D000212DE9F04F22
:20534000C3F8D815C3F8DC15C3F8E015A3F8E415BCF1000F4AD003F18C020C460D4608466A
:205360000E460F4602EB0C1BE246B2F802E0B2F80CC092F8009092F90180704461444F4533
:20538000D2E901EC38BF4F4610324645B8BF4646934500B209B275446444E6D190FBFAF037
:2053A00091FBFAF183F8D87583F8D965C3F8DC55C3F8E045124AA3F8DA0512780F48A3F8D7
:2053C000E415092A4FF0000180F8DC1003D10D4A93F8D835D3800C48BDE8F08F0020704798
:2053E0008C3303EB001070470748704761466046E0E700BFA067002080B600206804002057
:20540000A9280020AC28002058BC00200268F8B53A4E3B4CB6F9E835511C01607E21117093
:205420000168054603EBC30384FB0302481CDC17002328600B70FF20C4EB6204FFF76CFF6E
:205440002034304BA4B200284DD01B78B0F90C102BBB2D4BA1F57A729A4246D82B48B0FB92
:20546000F1F189B228463CF0BBFD96F8EB32B6F8881383B196F89033B1FBF3F128463CF01A
:20548000AFFD214628463CF0ABFD28460821F8F71BFA0120F8BD28463CF0A2FDF1E796F8A7
:2054A0006E70002FD5D01A48002300EB830201339289BB421144F8DB164B9FED176A9B7E4A
:2054C00007EE103A07EE901AB8EEC77AF8EE676AC6EE077A67EEA67AFCEEE77A17EE901AAC
:2054E000B1FBF7F1B5E71B7813B94EF69C21B9E796F86E70002FF8D00146D4E780B60020C1
:20550000676666663166002017839303008793036CBC002078310020000048432DE9F84301
:205520004A4C427894F8703602F00F05C3B9EDB92B46002184F87416EB1AD9B20E290BD87F
:20554000234493F8EC1239B102F0F002802A4AD0902A5FD0A02A0DD000273846BDE8F88374
:205560000021AB4284F87416F6D8E5E784F870562B46DEE7412966D081F08003042B62D907
:205580000846FCF7E9F9031D0246DBB2304884F8743665F05F0584F87556FCF7C9FE94F80F
:2055A0007476002FD8D0BE1E16F0FF0024D1FF25A946022756B1DFF89C80464418F8011B68
:2055C000D4F8980634F08CFB4645F7D1D4F89806494634F085FBD4F89806294634F080FB4E
:2055E0003846BDE8F88365F07F050427022684F8755684F874763046164A4FF6FF71104455
:2056000012F8015B491B904289B2F9D15FFA81F90D0ACFE7412914D081F08003042B10D9EF
:205620000846FCF799F965F06F050627042684F8770684F8755684F8761684F87476304653
:20564000DAE70420EFE7082304229FE780B60020F6BC0020F4BC00202DE9F047C31DDFF8BC
:20566000348182B003F4FC7300AFD8F82C61ADEB030DC7F800D03268D8F8243168449A4253
:205680000C4698F89C3678606D4658D0591C0DF1010203F00F0388F89C168DF800303A60A7
:2056A000A0EB0209D6E900125FFA89F9521A09F107035FFA82FA03F4FC73CA45ADEB030D46
:2056C00055D25246684653F025FD3368534433605246694638463CF061FCD8F82C21D8F8F8
:2056E00024313068117A7060C21A4A40D2B28342336088F89D2609D00133336013F8011C15
:20570000984282EA0102F7D188F89D263B68591C39601A70D7E90032D21A012A08DD0021EB
:205720005A1C3A601970D7E90032D21A012AF7DC2846A04700200837BD46BDE8F087B6F972
:205740000C20591C03F00F0343F01003002A2A46B8BF43F0200302F8023B88F89C16691C08
:205760003960D6E900135B1A3A606B7098E74A46684653F0CFFC33684B4433604A4669460D
:2057800038463CF00BFC2846A04701200837BD46BDE8F08780B600202DE9F04F7A4C83B0E0
:2057A000D4F82C51D5E900535B1B002B00AF83460D46164628DD002384F89E36FCF740F923
:2057C00000200BEB05030BF1010AC4E946A39BF80050D4F828816909012940F09D8005F0D8
:2057E0000F0915F0100514D150B194F8A026013202F00F024A4500F0988084F89E56284694
:205800000C37BD46BDE8F08F94F89E060028D8D1D4E70BF10203C4F818310BF103029BF8C8
:205820000130D4F82001C4F818219BF80250C8F80000C218C8F804206B4084F89F36D4E939
:2058400046A34FF0000C84F89E16A8F80850A8F80CC0A3EB0A03DDB2121AEB1D5FFA82FB4C
:2058600003F4FC73AB45ADEB030D6BD25A465146684653F04FFC0AEB0B035A4640466946A2
:20588000C4F818313CF08AFBD4F82031D8F8000094F89F268342C8E900300AD00133C8F8A0
:2058A000003013F8011C984282EA0102F6D184F89F26D4F818311B78934239D1B8F90830CF
:2058C000FA2B54D0D8F80020D4F82031D4F82811D4F8D402C8E90032D4F82C21D4F82431AE
:2058E00053600025158195813B1D84F89E567D602DF060FA01303FD07B680BB1002098472A
:20590000D4F82C31D4F82421196801200C37C3E90021BD46BDE8F08F00210846FCF774F8A6
:2059200001200C37BD46BDE8F08FD8E9000290E700230120B8F9081084F89E36FCF764F8F6
:2059400001205DE72A465146684653F0E3FB0AEB050340462A466946C4F818313CF01EFB20
:2059600000200C3784F8A096BD46BDE8F08F002EA8D005233370A5E7D4F82C211368022137
:20598000581C10601970B7E780B600200B4B93F8AE2312B1B3F8FC224AB9B3F93434084AFF
:2059A000D81782FB0323C0EBA30000B27047D3F8C80390FBF2F000B2704700BF80B600201D
:2059C00067666666F8B5184CC6B205463146D4F8A40634F085F994F8A816D4F8A406C5F353
:2059E00007274E40394684F8A86634F079F994F8A816D4F8A406C5F307464F40314684F805
:205A0000A87634F06DF994F8A816D4F8A4062D0E4E40294684F8A86634F062F994F8A81693
:205A20004D4084F8A856F8BD80B6002070B50C4DC6B231460446D5F8A40634F051F995F82B
:205A4000A816D5F8A406240A4E40214685F8A86634F046F995F8A8164C4085F8A84670BD91
:205A600080B6002038B50B4C002305462421D4F8A40684F8A83634F033F9D4F8A4065421CE
:205A800034F02EF9D4F8A4062946BDE8384034F027B900BF80B600202DE9F047DFF85CA37D
:205AA0002DED028B9AF8A94682B00F461646002C00F0E981013C8AF8A946DFF844839FED7D
:205AC000C88ADFF840933B78002B00F090809AF8A946002C40F08B8036B133F0A3FC3368C0
:205AE000C01A002880F2DD839AF8AA16002940F07C839AF8AB56062D40F28681B94B93F89A
:205B00008D0193F88C21824200F0AD81D3F888219AF8AC1632F810400C440135013003F5EC
:205B2000C473A4B2EDB2C0B2B4F5C06F8AF8AB56587100F080817CD8B4F5806F00F02B8229
:205B400024D8B4F5067F4FD8B4F5007F54D3A4F50073182B48D8DFE813F0E901E001E001C0
:205B6000E001E001E001E001E001E0014700470047004700470047004700C801AD01AD01C9
:205B8000AD01AD01AD01AD01AD01AD01B4F5846F00F0E88140F2E280B4F5A06F00F06682D8
:205BA0006FF4A06C04EB0C03072B1DD8601EC0B2FFF7B2FBC0B1B0F90C308B4AADF80140AD
:205BC000917EDAF8D82203EB830303EB830349089B0093FBF1F31021CDF803308DF80010E6
:205BE0006846904700233B70002E7FF46CAF02B0BDEC028BBDE8F087B4F5807F00F0FF817A
:205C0000B4F5887FF0D1BAF93634CDF80330012210238DF800308DF801308DF80220DAF8C4
:205C2000D8326846002498473C70002E7FF44BAFDDE7B4F5046F00F0A68265D8B4F5006F15
:205C400000F084821AD9B4F5026F00F0F381B4F5036FC9D19AF884339D07C5D5634BDAF821
:205C6000D822D9894FF4F36303FB01F3A8FB03135B091020CDF8033030218FE2B4F5E26F3C
:205C800000F03982B4F5E46F1FD1594BDAEDF47A93ED000A20EE270A002420EE080A51F046
:205CA0006DFC102320228DF800300723CDF803008DF802308DF80120DAF8D8326846984799
:205CC0003C70002E7FF4FFAE91E7B4F5E06F8BD1484BDAEDF47A93ED000A20EE270A002449
:205CE00020EE080A51F04AFC10220723CDF803008DF802308DF80020DAF8D8328DF80140DB
:205D0000684698473C70DCE740F678339C4248D8B4F5376F00F2E481B4F5116F00F08281E6
:205D2000B4F5376F7FF460AFFF20FFF7F5FA00283FF45AAF90F90130CDF8033010217022B5
:205D40000B238DF802308DF80010DAF8D8328DF801206846002498473C7066E740F2014327
:205D60009C4200F02A82B4F5826F7FF43DAFDAF81431980600F148821F4B1B681B0640F101
:205D800096820024102304228DF800308DF801308DF803408DF804408DF805408DF80640DD
:205DA000BDE145F230239C4200F0868145F240239C427FF419AFBAF93034CDF803301021F3
:205DC000402252238DF802308DF80010DAF8D8328DF801206846002498473C7025E700BFF6
:205DE0000000C8426804002078310020D8680020A8BA0020A0BA0020A067002080B600206B
:205E00001F85EB51C5B3A2910135CA4BEDB293F8952193F89411914220D0501CC0B25200A9
:205E2000D3F89011C44B8C5A8AF8AB56B4F5C06F58717FF480AEDAF8C833CDF80330102245
:205E4000002406238DF802308DF80020DAF8D8328DF80140684698473C7032E7002283F808
:205E600095210120DCE79AF8AC269AF86E0083F88D110132D2B2013082428AF8AC2600F01B
:205E8000B0810125C3E700283FF417AE0378303B012B3FF612AE01300AF2A9620621FFF785
:205EA0007BFC9AF8A9368AF8AA06002B3FF405AE3C7002E6A4F11100C0B2FFF72DFA0028C6
:205EC0003FF492AEB0F90230CDF8033010238DF80030ADF80140DAF8D83268469847002322
:205EE0003B70002E7FF4EFAD81E69AF8EB22BAF88833002A40F0CF8110220221CDF8033050
:205F00008DF80020DAF8D8328DF801208DF802106846002498473C7087E6601EC0B2FFF713
:205F2000FBF900283FF460AE4368CDE7DAF8C0338249DAF8D82281FB0301DB17C3EBA10385
:205F400000241021CDF8033002238DF800108DF801408DF80230684690473C70002E7FF4EB
:205F6000B2AD44E69AF884339A077FF53DAEBAF88633CDF803301021202204238DF802309B
:205F80008DF80010DAF8D8328DF801206846002498473C7049E69AF8B4360133DAB2042AF4
:205FA00000F06E8142F210738AF8B42603FB02F3DAF8B826002A00F0258102339AF82E2374
:205FC000D507BAF8CC2348BF0433D40748BF0A33900748BF1433D10548BF2833550748BF67
:205FE0006433540648BF03F57A63102100240422CDF803308DF800108DF801408FE0DAF8C5
:020000040801F1
:20600000B036CDF803301022002401238DF802308DF80020DAF8D8328DF80140684698479D
:206020003C704EE69AF89033002B40F02F811022092163E79AF884339B077FF5D5AD404A0F
:20604000DAF8D8329268CDF80320102220218DF8002008228DF801108DF802206846002431
:2060600098473C70002E7FF42EADC0E5FF20FFF753F900283FF4B8ADB0F90C303149DAF822
:20608000D822897E03EB830303EB83031020490800249B0093FBF1F305218DF80000CDF8F5
:2060A00003308DF801408DF80210684690473C70002E7FF408AD9AE5BAF93234CDF8033039
:2060C0001021302252238DF802308DF80010DAF8D8328DF801206846002498473C70A4E514
:2060E000A4F17100C0B2FFF717F900283FF47CAD90F90130E8E6144BDAEDF47A93ED000AF8
:2061000020EE270A002420EE080A51F037FA1023CDF8030007228DF800308DF80130DAF829
:20612000D8328DF80220684698473C70002E7FF4CAAC5CE568040020F805002067666666DB
:20614000D868002078310020A4BA00209AF884339C077FF549ADC107814B40F1B5805A6886
:2061600082EAE273A3EBE27303EB5303A8FB0313DB08002AACBF43F0004343F040431021A9
:206180000024082234E7BAF93434DAF8D82203EB83035B001020CDF80330402108238DF8A7
:2061A00000008DF801108DF802306846002490473C70002E7FF487AC19E5BAF9E835CDF8D6
:2061C00003301021012204238DF802308DF80010DAF8D8328DF801206846002498473C70E6
:2061E00023E58AF8AC16012511E65E490620FFF733FA00238AF8AA063B7002B0BDEC028B5E
:20620000BDE8F0870133D9E6554A9AF88413538A643BC3EB4370C3EBC00389FB0340184436
:20622000DB17C3EB20230933092BA8BF092323EAE37303EB830311F0020F03EB830314BF48
:206240004FF47A7000209B00C90748BF00F5FA60117DDAF8D8229BB203440B44042010219E
:206260008DF80200CDF803308DF800108DF801106846002490473C70002E7FF424ACB6E414
:2062800001238AF8B43642F2107391E6BAF88823B2FBF3F3CBE69AF89023002A57D11346AF
:2062A0002AE63C7002B0BDEC028BBDE8F0879AF8EA32002B3FF498AC9AF8BC36032B49D8FB
:2062C000DFE803F03B3122111A6882EAE273A3EBE27303EB5303A8FB0313DB08002AB8BFBE
:2062E00043F080434BE7DAF8C026537A907AD17A03F1407303EB0023002203EB01438AF80E
:20630000BC2610220421F9E5174A11688A7D087C897A120402EB00220A44591C8AF8BC16C2
:2063200002EB0363EDE7104A11684A7DC87B497A120402EB00220A44EFE70B4A11680A7DF8
:20634000887B097A120402EB00220A44E5E7B3FBF2F3D1E55A1C8AF8BC261B06D1E700BFBD
:20636000D8680020811A0108F8690020CA4A38B50820002382F89531FBF758FC002800F0AE
:206380008C80D2F890314FF4806102204FF48264198082F8950101465C804FF40020FBF7D6
:2063A00045FC50B14B1CD2F89001DBB240F2014482F8953120F811401946B84C94F8AD335D
:2063C000002B6CD194F8AE33002B40F088804FF40070FBF72BFC50B14B1CD2F89001DBB269
:2063E0004FF4046582F8953120F811501946D4F81441A50700F10181600700F1DB80A84BF3
:206400001B681B0600F1938000234FF4803082F8941182F8953182F88D31FBF707FCD0B3AF
:20642000D2F8883101214FF4047082F88D1118804FF40040FBF7FAFB50B14B1CD2F888012B
:20644000DBB24FF4007482F88D3120F8114019464FF40030FBF7EAFB50B14B1CD2F88801F3
:20646000DBB24FF4A06482F88D3120F8114019464FF48020FBF7DAFB38B1D2F888014FF41F
:2064800037644B1C20F81140D9B2002382F88C1182F88D3138BD0146CAE701467DE70120DB
:2064A000FBF7C4FB00288DD04FF48030FBF7BEFBD2F8905128B94FF4047325F81130013132
:2064C000C9B20BB2481CC1B24FF4116082F8951125F8130094F8AE33002B3FF478AF022095
:2064E000FBF7A4FB00283FF472AF4FF40040FBF79DFB50B94B1CD2F89001DBB24FF4007572
:2065000082F8953120F8115019460420FBF78EFB00283FF45CAF4B1CD2F89001DBB24FF4CC
:20652000C06582F8953120F8115019464FE74FF40050FBF77BFB50B14B1CD2F89001DBB29D
:206540004FF4036482F8953120F8114019464FF48050FBF76BFB68B1D2F890014B1C4FF400
:206560000064DBB28D1C20F81140E9B282F8951120F813404FF48040FBF758FB50B14B1C42
:20658000D2F89001DBB24FF4846482F8953120F8114019464FF48060FBF748FB00283FF42D
:2065A00033AFD2F890014FF402644B1C20F81140D9B229E74FF48060FBF738FB50B14B1CDA
:2065C000D2F89001DBB24FF4807482F8953120F8114019464FF40060FBF728FB00283FF481
:2065E0000EAF4B1CD2F89001DBB24FF4887482F8953120F81140194601E78020FBF716FBBD
:2066000050B14B1CD2F89001DBB245F2302582F8953120F8115019464FF48070FBF706FB60
:2066200050B14B1CD2F89001DBB245F2402582F8953120F8115019461020FBF7F7FA50B142
:206640004B1CD2F89001DBB24FF4E06582F8953120F8115019462020FBF7E8FA50B14B1CCF
:20666000D2F89001DBB24FF4E26582F8953120F8115019464020FBF7D9FA00283FF4BCAEA6
:206680004B1CD2F89001DBB24FF4E46582F8953120F811501946AFE66804002080B6002090
:2066A000A067002030B5A0F17D03012B044683B00D46104608D9214633F012FB15B128887D
:2066C00004442C8003B030BD7D21019233F008FB019884F0200133F003FBEFE730B50F4B6B
:2066E00085B0D3F8202300230446C51DADF80E3014F8010B01920DF10E01FFF7D3FFA542BE
:20670000019AF5D10DF10E0014F0BCFD019A9DF80E000021FFF7C6FF05B030BD80B600203D
:206720007E28F8B50F4652D0324E96F8984164B9314D95F8CC1651B11B2885F8CC463DD0BD
:206740000D2837D0012386F898310020F8BD7D284AD095F8D0261AB180F0200085F8D016BD
:2067600095F8CB26062A14D8B5F8CE46511C2A440444C9B2A5F8CE4685F8CB1682F8C406CD
:20678000002BE2D10729E0D101231C4886F89831F8BDB5F8CE361844C0F3072353FA80F00F
:2067A000FF284FF00103A5F8CE0686F89831CCD11248F8BDA5F8CE462046F8BD9047002840
:2067C000C0D0012320463B7086F89831F8BD0A4B084A0024012183F8CB4683F8CC163C7076
:2067E00082F898412046F8BD0123084685F8D036F8BD00BF6804002080B6002044BD0020BF
:20680000044AD2F8D43643F4DF2343F48063C2F8D436704780B60020013070B5094EC4B20F
:2068200003E044F0C5FF013448B9E5B2152D21463046F6D9162D04BF034B93F8D856284647
:2068400070BD00BF54BD002080B6002000B1D7E7044AD2F8D43623F4DF2323F48063C2F867
:20686000D436704780B6002070B5114C84B00546D4F8DC060E462BF0FDFD94F8E42294F8CB
:20688000E532003A18BF01220BB142F00802CDE9016200234FF4964195F9000000911A46E0
:2068A00008212BF076FEC4F8DC0604B070BD00BF80B6002010B5064C03E0D4F8DC0633F0C1
:2068C00003FAD4F8DC0633F007FA0028F5D110BD80B6002010B50D4CD4F8E0361B791E3BEB
:2068E000012B0DD9D4F8DC0601213830FFF7BCFF0023C4F8E43684F8E836BDE81040D9E755
:20690000D4F8DC06012133F0D7F9F1E780B6002070B5C54C94F8F036D4F81411C4F8EC06FF
:206920000133880784B084F8F03612D411F0340F33D1090794F8F02640D412F0070559D093
:20694000282A00F0B980D4F8DC325E20984704B070BD7020FBF76AF90028E7D004F58466FD
:206960002425F6EC017A94EDF47A67EE877A2846FDEEE77A013517EE901AC1EB411301EBA1
:206980008301C90009B2EDB2FBF7B2F8272DE8D1D4F8141111F0340FCBD04FF40060FBF742
:2069A00045F9002840F0058194F8F02612F0030100F0DB80D4F814110907BED54FF4007081
:2069C000FBF734F90028B8D012F00305B5D1974AB4F93434D91782FB0323C1EBA30109B2C4
:2069E0001420FBF785F829461C20FBF781F894F8F026A2E7FF20FEF78FFC002800F0DF809D
:206A00000378FF2B7AD090F901100220FBF770F8FF20FEF781FC002872D00378FF2B6FD092
:206A2000B0F90C20824B8148997E02EB820202EB82029300490893FBF1F3D91780FB03200E
:206A4000C1EBA00001B20320FBF752F894F8AD33002B5DD1D4F814319A067AD54FF4005080
:206A6000FBF7E4F8002840F0C980724D4FF48060FBF7DCF8002840F049816B8A94F8F02646
:206A8000297DB3F5967F02D9100740F10E8194F8E732002B40F0958009B20520FBF728F8DA
:206AA0004FF48050FBF7C2F8002840F0D58094F8F026282A7FF447AF5F4A604B1568604993
:206AC000A3FB0535AD09A1FB05367609A1FB06314909C1EB0111A6EB81010902C6EB061604
:206AE000002309B21720A5EB860684F8F036FAF7FFFF31B21820FAF7FBFF24E7294684E7E9
:206B000000210320FAF7F4FF94F8AD33002BA1D00120FBF78BF8002840F00A8194F8AE335F
:206B2000002B97D00220FBF781F8002840F059810420FBF77BF800288CD0B4F8B033002B3D
:206B400000F05C8129F04AFB01B20420FAF7D0FF80E71B07ABD53B4B93E8030002AB83E84E
:206B600003001846FAF7DAFFA1E74FF48060FBF75DF800283FF41EAF334BD4F8EC26D4F8A8
:206B8000B0569A4240F20A81304BE91783FB0523C1EB6313642101FB13510DB219B2102074
:206BA000FAF7A6FF29462120FAF7A2FF94F8F02600E7B4F936143020FAF79AFFF4E6014682
:206BC00023E7A1F1200307EE903A9FED217AF8EEE77AF6EE006A67EE877ABEEE007AF5EE1C
:206BE000C07AF1EE10FA58BFB0EE667A77EE877AFDEEE77A17EE903A19B24EE794F8843319
:206C00009B0758D44FF48060FBF710F8094D00283FF433AF002631460120FAF769FF314668
:206C20000920FAF765FF28E780B600206766666678310020D8680020D0240020D34D621009
:206C4000898888882C9C06083F4B4C001F85EB51E4380E3F0050C34794F8842300239207D5
:206C6000CDE9003347D494F8F436012B43D0B4F9E0325FED086A07EE103AB4F9E23207EEA9
:206C8000903AB8EEC77AF8EEE77A27EE267A67EEA67ABDEEC77AFDEEE77A02A88DED027AFA
:206CA000CDED037AFAF73AFF01E742F20F719942A8BF1946EBE6544D544BE9894FF4F36617
:206CC00006FB01F14909A3FB0131C9091120FAF70FFFE9894E4B06FB01F1A3FB012149098D
:206CE000A3FB01235B09642202FB131109B21920FAF7FEFEBAE6D5E9002301216846CDE9DF
:206D0000002384F8F416FAF709FFD0E694F884339E077FF57FAFAB683D4AD91782FB030285
:206D2000C1EB6211642606FB113636B209B273E794F8901300293DD10B460620A4F8F236C4
:206D4000FAF7D6FEB4F8F2360133A4F8F23629F039FA94F8E83294F89023012B94F8EB329C
:206D60001ED000EB800086B213B10AB1B6FBF2F6274BA3FB062343F34F113A205D09FAF7EA
:206D8000B7FE642101FB1561224B89B20531A3FB0131C9083B20FAF7ABFEBFE60D46FEE6F7
:206DA0001BB112B1B0FBF2F080B201B23920FAF79FFEB3E6B4F8F206B4F88823B0FBF1F3C8
:206DC00001FB1303642000FB02129BB24900B2FBF1F2110241EA0311C2F30322114309B2AD
:206DE000ABE7D4F8C0330C49DA1781FB0313C2EBA30319B22820FAF77BFE99E6D4F8C83354
:206E000083F3100319B2A0E6D8680020C55A7C0A1F85EB51CDCCCCCC676666660B2814D8CA
:206E200010B401EB4103094C01EB83032344184490F84834934205D02144002380F84824BA
:206E400081F83C345DF8044B7047704780B60020F0B5454C94F8F536012B83B005464FD922
:206E600094F8F6064149424E94F8F776421CA1FB02C1184406EB800001F4FE7606EB910101
:206E8000521A466C84F8F6262FB1D4F8F81604F2FC6291420DD06EB9364A0133A2FB0312F1
:206EA00022F0010101EB52029B1A84F8F53603B0F0BD314E94F8103793B9304B019348F2DB
:206EC000A501123B15226F46A4F81417009384F8162729463846B04758B994F8F536DBE752
:206EE0006F46384611F0C2FD29463846B0470028F3D094F8101751B1384611F031FDECE79B
:206F00001B4A02EB8302566C002EC5D0D2E7009E1B4A964214D9013A013E41F2210512F8B7
:206F2000013F81EA0321082311F4004F85EA41000ABF490081B289B2013BF5D19642EED13A
:206F400038463BF073F80F49009D6D1A152DA8BF15252A4601F1180052F0DCF894F8F53677
:206F600084F8415798E700BF80B60020CDCCCCCCF09B0608ABAAAAAAC1270108A9BD00207F
:206F800097BD002094BD002070B50B4E054606F2467140F061FA2C686C6006F24471641A7E
:206FA000402CA8BF40242960224606F2847052F0B1F886F8C44770BD80B6002030B50C4B8A
:206FC0000C4AC3F8442783B0C822014603F2847503F2497483F8482768463A22CDE9004542
:206FE0003AF0DCFF6846FFF7CFFF03B030BD00BF80B60020C83E7BEA03685A0607D513F44C
:20700000057F04D007298CBF00200120704703F48253B3F5825F03BFC81FB0FA80F0400944
:207020000020704770B5BC4C94F8C537012B84B000F04C8194F8D107FCF764F894F8D2375F
:20704000834205461FD0002800F0D580D4F8E036CBB194F8E52293F90400002A18BF082218
:207060004FF4964100230325CDE9015200911A4608212BF08EFAC4F8DC0620B1FFF72AFC5A
:20708000012384F8D23794F8D337012B00F0C080D4F8DC673EB1A14B30465978FFF7ACFF83
:2070A000002840F0F18094F8E107FCF72BF894F8E0378342054621D0002800F0F580EEB1AD
:2070C000337A002B00F01781954A02EB83031B6E94F8E42296F904000093003A18BF012289
:2070E00002210023CDE901121A4610212BF051FAC4F8A40610B1012384F8E037D4F8E46795
:207100003EB1864B30465978FFF776FF002840F0AB8094F8F007FBF7F5FF94F8E8378342A1
:20712000054622D0002800F0C880F6B1337A002B00F0E4807A4A02EB83031B6E94F8E4228D
:2071400096F904000093003A18BF012202210023CDE901121A464FF400712BF01AFAC4F8C7
:20716000EC0710B1012384F8E83794F8F107FBF7C9FF94F8F2378342054630D088B3694BAA
:20718000D4F8F4674FF47A72C3F8AC263EB34FF48052402130462BF087F90546F8B994F80C
:2071A000E43296F90400002B14BF0921082103224FF4E133CDE9012100932A462B464FF4CA
:2071C00080512BF0E6F9C4F8F80740B10123C4F8980684F8705684F8FC5784F8F23704B050
:2071E00070BDD4F8F8072BF045F9C4F8F85784F8F25704B070BDD4F8DC062BF03BF994F804
:20720000D337C4F8DC56012B84F8D2577FF440AF94F8D407FBF776FF0546002871D0D4F8F5
:207220002033002B7FF434AFD4F8D827002A3FF42FAF94F8E55294F8E41292F90400002D73
:2072400014BF08220022002908BF42F0010203254FF46141CDE9015200911A4620212BF087
:2072600098F9C4F8200313E794F8E837002B7FF47CAFD4F8CC37002B3FF477AF0122C4F8FE
:20728000EC3784F8E82770E794F8E037002B7FF435AFD4F8CC37002B3FF430AF0122C4F8D9
:2072A000A43684F8E02729E7D4F8A4062BF0E2F8C4F8A45684F8E05720E7D4F8EC072BF0AC
:2072C000D9F8C4F8EC5784F8E8574EE7D4F8C857124B28465978FFF78FFE28B3D4F880338A
:2072E000002B7FF4A7AED4F8CC37002B3FF4A2AEC4F880339EE64FF49643E9E64FF4614359
:207300001CE7D4F8200300283FF4C2AE2BF0B2F8C4F82053BCE600BF80B600201C63002066
:20732000F09B06086804002094F8D007FBF7EAFE0646D8B1D4F88033002B7FF47BAE002DA3
:207340003FF478AE94F8E42295F90400B2FA82F252094FF416510225CDE9015200911A466A
:2073600004212BF016F9C4F8800363E6D4F8800300283FF45FAE2BF07DF8C4F8806359E611
:2073800070B5B14C94F8C537002B00F0218108202BF09EF8C4F8E00600283BD008212BF094
:2073A0008DF800260346A949A94884F8D137C4F8046836F061FE41F208530122A448A4F88C
:2073C000083884F80C280DF0D5FF31462B22A14851F001FF48F67C607D25E02331462B227B
:2073E000A4F814089C4884F8173884F83F5851F0F2FE48F67C21A0224EF27B0384F86B5848
:2074000084F86E6884F81759A4F8401884F84328A4F86C3894F8D337002B00F0C3801020EF
:207420002BF056F81021C4F8DC072BF047F88B4B84F8E1073A2140F23B1094F8AD231880B3
:207440009F254AF21E40197100219D7198601973002A40F08E8094F8AE33002B48D1D4F8AC
:20746000143158077ED4990773D41A076AD47C4D2868C0F3C010FFF7E9F90020FFF7CCF941
:2074800003464FF4007084F8D8362BF021F84FF40071C4F8E4072BF011F8D4F8183984F81A
:2074A000F007002B14BF0123002384F81C3926D1D4F88C290023C4F88839002A69D0012221
:2074C00084F8103784F890294FF480502BF000F84FF48051C4F8F4072AF0F0FF002384F81B
:2074E000F10784F8F237FAF7ABFABDE8704099E5D4F8D43643F00403C4F8D436AFE7D4F84E
:207500001421002312F0020284F81D3984F81E3940F0828094F8AD3323B10120FAF786FB63
:20752000002873D194F8AE33002B6AD1A3182868042183F82019030602F1010175D484F825
:207540002419B5E7D4F8D43643F48073C4F8D4368DE7D4F8D42642F4601242F0C002C4F8FA
:20756000D42682E7D4F8D42642F40272C4F8D42679E7D4F8D43694F8AE2343F00201C4F8FD
:20758000D416002A3FF46BAF43F03603C4F8D43665E7D4F894397BB3012384F8903984F860
:2075A000103791E720202AF093FFC4F8D80700283FF435AF20212AF081FF2A4BC4F8D83230
:2075C00084F8D407FEF7D2FE012384F8D33726E704202AF07DFFC4F8C80700283FF4D7AEB3
:2075E00004212AF06BFF204A84F8D0070123C4F8DC2284F8C537CAE684F8903984F8103717
:2076000062E70620FAF712FB00288FD0A318022183F82019013289E74FF46070FAF706FB3C
:2076200078B1012284F8202974E74FF45850FAF7FDFA002883D063180820911C83F820099C
:207640007DE7024666E700BF80B60020909C060880BE002094BE0020C0BE0020B06800203C
:20766000A0670020DD66010821230108094BB3F8A623B3F8A433801A9B1AC00090FBF3F083
:207680000628A8BF062020EAE070C0F19600C0B2704700BF80B6002010B5094B0022D3F84A
:2076A000981903F69C13914201D1002010BD13F8014B844201D00132F5E70120F6E700BF25
:2076C00080B600201B4B2DE9F04103EB81038EB0D3F8F07006460D4647B3174B03EB41039F
:2076E0001C22B3F8D849002319460DEB0200069304F01F0851F06FFDC4F3441401228DF8EC
:20770000085006AD8DF81420CDE903568DF809808DF80A4002A8B8479DF8142000232AB149
:2077200000952246414602A806F0B0F80EB0BDE8F08100BFF09B060880B600200A4B03EBB8
:207740004002B2F8D819094A92F85C2902EAD122520707D0D3F89829511CC3F8981913441F
:2077600083F89C09704700BF80B600206804002010B5164B42681B7803F00303032B21D115
:20778000134B1B88DBB1134B1349B3F90030B1F904100A2491FBF4F15B1A1B0103F5B953D4
:2077A00014334FF4B471B3FBF1F3C3F1080303F00F0360331370436800225A7010BD052322
:2077C0001370F8E72D231370F5E700BF04BA002006BA0020ECC10020B0BA00204368722285
:2077E0001A70436873225A70436874229A7043680022DA7070470F4B4268B3F904300A21CD
:2078000093FBF1F31B0110B503F5B9530A4C4FF4B4711433B3FBF1F303F00F03E118E35841
:2078200013604B6853600B7A1372436800225A7210BD00BFB0BA0020009E0608084B5B7AE2
:2078400033B942F210735843064B90FBF3F07047242358434FF47A7390FBF3F0704700BF7E
:20786000ECC1002040D20600044B5B7A2BB94FF4A4735843642390FBF3F07047ECC10020AD
:20788000831E00F17402EA2123F8021F9342FBD143F649134385CD2383804E23C380CE2303
:2078A00003812323A0F87230704700BF08BB1F48B0F86C3003F001036BBB30B490F87040A7
:2078C000ACB11B4A02F1F00502E00133A3420ED052F8041B4904F8D590F85C1100EB810140
:2078E000D1F8F41045F823100133A342F0D130BC70470E48B0F86C20032A4FEA52030BD9A5
:207900000A68A0F86C3002F5C332A03203F001030A60002BD1D070470B6803F5C333A033EB
:2079200048F205020B60A0F86C207047ECC1002060C200202DE9F04100283AD12D4A92F836
:20794000700080B32C4A2D4B92F800E092F901C092F90280CEF1FF07AEF17F06FFB2F6B291
:2079600003EB800003F1F002002403E0834202F1040218D053F8041B8904F7D5E1B2A1EB24
:207980000C0181EAE175A5EBE175012D0DDC71B1414514BF394631468342D17004F10104AB
:2079A00002F10402E6D1BDE8F0810821F4E77146F2E7114B1A78F02A09D802F10F000D4A2B
:2079C00018700B6803F582431A330B60B7E7094A93F9014092F872007F2584421D70987876
:2079E00005DB4042C0B2987020445870E9E7002CFADAF6E7ECC10020C80D002060C20020CE
:207A0000F0B5364E78B196F8E431002B46D0344A013BDBB286F8E4311378DC0741D4314B57
:207A20000A681A440A6096F870404CB32E4B2C4F03EB840403F1F001002503E09C4201F1A8
:207A400004011DD053F8042BC2F303200628F5D13878C00715D596F8E40196F873E000EB4E
:207A6000050CBCFBFEF00EFB10C00128CCBF0020012058B99C4205F1010501F10401E1D1EE
:207A8000F0BDE84300F001000028F3D0C2F3834206EB8202D2F8F4200A60EBE796F87330F8
:207AA000B5E7124A124BB2F906201248A2F57A74642202FB04F283FB0234D317C3EBA41345
:207AC00003EB4303C3EB031380FB0302DB17C3EB62130533084A92FBF3F3A1E7ECC10020C7
:207AE000AEB90020400D030060C200209C6A0020D34D62101F85EB5140420F00F0B4524C02
:207B0000002868D194F8E501002856D04F4BD3ED007AB3EE097AF4EEC77AF1EE10FA4EDC16
:207B2000BBEE097AF4EEC77AF1EE10FA4CBF08270027D3ED017AB3EE097AF4EEC77AF1EE4B
:207B400010FA3EDD47F0010794F87050ADB3404ADFF808C102EB850502F1F00014E094F910
:207B6000E861B142ACBF0221002194F9E961B3421CDB41F004010F421CBFDCF8243003606A
:207B8000954200F1040018D052F8043BD903F7D594F9E76103F00F01B142C3F30313DEDCAF
:207BA00094F9E961B3424FF00101E2DA94F9EA61B342D8BF41F00801DDE7F0BC704704270C
:207BC000B7E7BBEE097AF4EEC77AF1EE10FA48BF47F00207B8E794F8E63163B31B4B1D4D60
:207BE000D3ED007A93ED017A0A6894F8E501F0EEE77AB0EEC77AF4EEC77AF1EE10FAB8BFCB
:207C0000F0EE477AFDEEE77A80F0010017EE903A193B03EB4303C3EB031385FB0365DB1713
:207C2000C3EBE51305330C4DB5FBF3F31A440A6084F8E50168E70B6894F8E50103F54333AB
:207C400003F5A0730B605FE7ECC1002014BA002060C20020353AFC4440420F00009E06087F
:207C6000F0B40B4F97F8706086B107F17402054607F5B277002352F8044B35EA040004BFF0
:207C8000086847F823000133B342F4D1F0BC7047ECC1002030B42A4B60B92A48027DCAB90E
:207CA00093F85D312849203301EB830130BC4FF4A060D5E793F8EB21F2B1013A214883F833
:207CC000EB210A6802F5C32202F520720A60027D002AE5D01D4A12689106E1D51C4A93F8DA
:207CE000EB11127892071AD511BB93F85F311649203301EB8301D9E7124893F8EC41057D19
:207D0000A54205D8042483F8EC2183F8EB41D8E70134012283F8EC4183F8EB21D1E7002921
:207D2000BED193F85E310849203301EB8301BDE793F85B310449203301EB8301B6E700BF5F
:207D4000ECC10020D868002060C2002094B7002004BA002010B41E4A48B91E4C92F8ED015C
:207D60000B6823440B6098B15DF8044B704792F8EE3103B3012B16D092F8ED010B68164C5C
:207D800080F00100234482F8ED010B600028EBD192F85B3111495DF8044B203301EB83017D
:207DA0004FF440705CE792F8ED010D4C80F0010082F8ED01D4E70B685DF8044B03F5742382
:207DC00003F5107301200B6082F8ED01704700BFECC1002040420F0048E8010060C20020ED
:207DE00020A107003C4AA0B992F8EF316BB192F8F0118A081341DB070AD501F00101032AC4
:207E000006D8DFE802F05048403892F8F23153BB704792F8F031013303F00F0382F8F031CA
:207E20003BB192F8EF31086800F5C330A0300860DCE72A4882F8EF31437A002B44D12848E0
:207E4000C07818B143F0040382F8EF3125480078C00730D592F8F1010028E4D043F0080306
:207E600082F8EF31DFE792F8FE311F4901EB83014FF40030F4E61C4B03F13002002914BF3B
:207E800019461146F4E7194B03F1180200290CBF19461146ECE7144B03F10802002914BF09
:207EA00019461146E4E7104B03F11802002914BF19461146DCE70E4800680028CAD043F0B0
:207EC000010382F8EF31C5E792F8EE31002BB6D0022382F8EF31B2E7ECC1002024BA0020DB
:207EE000B0B90020AEB90020189E0608289E060838BD002030B4022340F203154FF4FA74C1
:207F000032210122C37000238580C480018130BC82720380704700BF90F8603043B9426932
:207F20000121072082F84430A2F8460082F84810704700BF034A0123E021C373517018461B
:207F4000704700BFECBE00204FF0FF30704700BF4FF0FF30704700BF704700BF00207047CC
:207F60000020704770B4067AAEB1427A0B4800212025002352B1142B05DC072903DCC45C3D
:207F8000202C18BFC55401339342F4D101318E4200F11500EDD1002070BC7047EFBE002041
:207FA00010B50024C473FFF7DDFF024B01225A70204610BDECBE002070B403980378ABB102
:207FC0000C4C02EB4205C5EBC5052544142901F1010406D8072A294403D8CE789E4218BFAA
:207FE000CB7010F8013FE1B2002BEFD1002070BC704700BFECBE002014299DF800000CD83E
:020000040801F1
:20800000072A0AD8064B02EB4202C2EBC2021A441144CB78834218BFC8700020704700BFFA
:20802000ECBE0020027A407A02FB00F0704700BF027A407A02FB00F0704700BF002070476D
:20804000002070474FF0FF30704700BF034B93F82923027293F82A3343727047ECC10020AB
:20806000002070470120704700207047027A407A02FB00F0704700BF002070470123C373B0
:20808000184670470123C373184670474FF0FF30704700BF704700BF002070470120704753
:2080A00000207047027A407A02FB00F0704700BF002070474FF0FF30704700BF704700BF1F
:2080C000002070470120704700207047027A407A02FB00F0704700BF0020704700207047D3
:2080E000002070470120704700207047014B1878704700BFD4240020914201D0012A01D9E7
:20810000002070470129FBD808B5074BC1EB0110C2EB021203EB421103EB40104FF4F072DA
:2081200050F0F8FF012008BDD824002001299DBF024B012083F82C1300207047ECC10020B4
:2081400001298CBF00200120704700BF4FF0FF30704700BF002070470020704730B41D2937
:208160009DF808000DD80F2A0BD8074B074D93F82C431E23C4EB041413FB021202EB441254
:208180005055002030BC7047ECC10020D8240020014B9888704700BFC80D002000207047E0
:2081A000024B0020C3F83003704700BFECC10020074BB3F88614B3F88824034610B4054CD5
:2081C0001C6001205DF8044B19815A81704700BFECC10020509E0608064AB2F87C340BB93C
:2081E0001846704792F88434037292F88534437201207047ECC1002000207047034B93F866
:20820000850493F8843400FB03F07047ECC10020002070477047037913F0020308D00369CA
:20822000D0E90920013B101A1840C0B2181A70471846704701717047704703799B070AD551
:20824000436A8269D154436A01690133B3FBF1F201FB123343627047037913F0010306D08F
:20826000D0E90732C0689B1A0138184070471846704710B5037913F0010301460DD0FFF770
:20828000EBFF60B10A6A4B69CC689B5C0132B2FBF4F004FB1022DBB20A62184610BD03462E
:2082A000FBE790F84F3830B53BB990F84D1890F84E380124DAB2914200D830BDB0F856585A
:2082C00004FA03F22A43A0F856280133F2E7D0E90920131A58425841704700BF014BD3F84C
:2082E000A0047047ECC10020034B002283F8A42483F8A524704700BFECC10020024B6FF070
:20830000020298689A607047C80D002070472DE9F04F744C89B094F8A6340490002B40D079
:2083200094F8A73403F0FF07002B3AD16E4BD4F8A8C41A7B0593002A0CBF63462023019314
:20834000B4F8B03403934FF03C0EB4F8B23494F8ACA494F8AD2494F8AE1407970293754667
:208360004FF00109019BBB421ED184F8AD24059A84F8AE1400235D491373012284F8A72449
:208380004A6E896E84F8ACA440F22A3050604B620B889BB243F001030B80136843F0010325
:2083A000136009B0BDE8F08F674536BF504B07AE03EB8706B378F078C3F1FF039BB2002B40
:2083C00000F08A80C3F1FF0343433688B6FBFEFB1B12BBF1050F00F28280DFE80BF0032B2E
:2083E0003C4B5C6DC21A7243B2FBF5F252FA83F2D9B2D2B2049B3F4E012B0BBF13020302FC
:2084000043EA004343EA024343EA0108602303FB076A1726039B09FA06FB1BEA080F9B4676
:20842000029B18BF9B46013E4AF804BBF2D20137824697E7B6FBF5F205FB1266B6B2C21A11
:20844000C6F13C06D9B27243B2FBF5F252FA83F30246D8B2CEE7B6FBF5F205FB1266C11A1B
:20846000B6B27143B1FBF5F151FA83F10246C9B2D8B2BFE7B6FBF5F205FB1266B6B2C21A48
:20848000C6F13C067243B2FBF5F252FA83F20146D2B2D8B2AEE7B6FBF5F105FB1166A0EB56
:2084A000030AB6B2DAB206FB0AFABAFBF5FA5AFA83F30146D8B29DE7B6FBF5F105FB1166E5
:2084C000B6B2C6F13C06C11A7143B1FBF5F151FA83F1DAB2C9B28DE7014602468AE750464A
:2084E00088E700BFECC10020C80D0020E4D2002050C30020A0C60020074910B5024600237D
:2085000001F5B274D1F8A804984200D810BD106844F823000133F5E7ECC10020034B5A7B74
:208520000AB901225A730020704700BFC80D0020034B0449B3F90E304068012243F002B9BF
:20854000C80D00203D220708064B07491A88074B40681B68534342F2107293FBF2F243F007
:20856000F1B800BF08BA00206123070840BA0020044A05495378127840680133013243F0D1
:20858000E1B800BF5C620020662307081C4B1A6812F0200F13B502F00403446829D0194A2A
:2085A0001278910725D5184BB3F90000FFF75CF96421002890FBF1F301FB13014FF00A00D0
:2085C00091FBF0F11148407AB4BF762275220029B8BF494200280CBF99209F20002BCDE902
:2085E0000010B8BF5B420A49204643F0ABF802B010BD002BD7D12D22227042685370F6E74B
:2086000094B7002004BA0020B6BA0020ECC100206C2307080B4B4068B3F904300A2293FB7E
:20862000F2F31A0102F5B9524FF4B4711432B2FBF1F2C2F1080202F00F020349603243F029
:2086400081B800BFB0BA00207A230708034A044992684068072343F075B800BF40BA00204D
:208660008123070807B5114A406892F86E30B2F86C10012B09D1009192F86F300C497B2288
:2086800043F060F803B05DF804FB0A234B4340F2FF32B3FBF2F39BB2092B064928BF0923B4
:2086A0007B2203B05DF804EB43F04CB8E4D2002087230708912307081E4B1A6812F020028E
:2086C00013B501461AD01C4B1A7812F0010215D01A4B1A7812F0020210D0194BDB89632B8B
:2086E0001FD964205843FFF7A9F8002819DD154B1B684FF47A725A4392FBF0F2124B486883
:208700005B7A541E002B42F20E710CBF7E237D238C4208D800930D49072343F013F802B077
:2087200010BD0022EAE70A49072202B0BDE8104043F008B894B70020AEB9002004BA002093
